:100000000C9457060C9476060C9476060C9476069F
:100010000C9476060C9476060C940B070C944A0705
:100020000C9476060C9476060C9476060C94760660
:100030000C9476060C9476060C9476060C940809BB
:100040000C9476060C9476060C9476060C94760640
:100050000C94DC410C94F3380C9476060C947606E0
:100060000C9476060C9474390C9476060C946839CA
:100070000C9476060C9476060C9476060C94760610
:100080000C94A1500C9476060C9476060C9476068B
:100090000C94B2390C9476060C94A6390C9476061E
:1000A0000C9476060C9476060C9476060C947606E0
:1000B0000C9476060C9476060C9476060C947606D0
:1000C0000C9476060C9476060C9476060C947606C0
:1000D0000C9476060C9476060C9476060C947606B0
:1000E0000C9476060C9495410C949F410C948B4192
:1000F0000C94F3410C94D0410C94C1410C94B54143
:100100000C94A9410C9476060C9476060C94760611
:100110000C9476060C9476060C9476060C9476066F
:10012000256300256300256300545F52483D252D5B
:10013000342E3166200052483D252D342E31662064
:1001400000256300256300507772312069732025F4
:10015000730A0044656275673D3078252D780A0082
:1001600048554D5F5057525F414C574159533D25BB
:10017000730A0025730A006175746F0A004C6F677B
:10018000206D6F64652069732000546F74616C206A
:10019000696E74723A2050303D252D6C64205031C8
:1001A0003D252D6C640A005553425F5057523D2542
:1001B000730A00565F4D43553D252D352E32660A94
:1001C00000565F494E3D252D352E32660A0052619C
:1001D00064696F205265706F7274204D61736B3D5E
:1001E0003078252D780A00526164696F205265705D
:1001F0006F727420496E74657276616C3D252D6452
:100200000A0052494D4520616464723D252D642EDB
:10021000252D640A004E65696768626F72207461FB
:10022000626C652073697A653D25640A00537461C8
:100230007475732053756D6D6172790A49443D0080
:1002400025630025630043757272656E74207265C4
:10025000706F727420696E74657276616C3D252DC5
:1002600064207365630A004E6577207265706F7253
:100270007420696E74657276616C3D252D642073FF
:1002800065630A00256300525F54313D09093078E7
:1002900025780A00525F41323D0909307825780AF5
:1002A00000525F41313D0909307825780A00525FDC
:1002B000565F494E3D0909307825780A00525F5251
:1002C000483D0909307825780A00525F5550544955
:1002D0004D453D09307825780A00525F50313D097F
:1002E00009307825780A00525F50305F543D090983
:1002F000307825780A00525F50303D090930782562
:10030000780A00525F565F4D43553D093078257895
:100310000A00525F545F4D43553D09307825780AF5
:1003200000525F543D0909307825780A00525F4930
:10033000443D0909307825780A005573696E6720B5
:100340007265706F72743D307825580A004E65777B
:10035000207265706F72743D307825580A002563ED
:1003600000256300256300256300204F534343416C
:100370004C3D2564200020467573653A2065653D37
:10038000253032782068663D25303278206C663D15
:1003900025303278206C623D25303278004D43554F
:1003A0003D2530366C7800256300252D31306C7585
:1003B00020252D31306C7520252D31306C75200AAB
:1003C000007268206D69737320202020726820738A
:1003D00074616C652020207268206D6973630A0067
:1003E0002563004F4B0A0025630025630025630049
:1003F000445F5057525F313D307825780A00445FA2
:100400004145533D307825780A00445F50315F4CB8
:1004100045443D307825780A00445F50305F4C45B4
:10042000443D307825780A00445F4556454E543D9A
:10043000307825780A00445F504F5745523D307858
:1004400025780A00445F4C45443D307825780A0001
:10045000445F4F573D307825780A00445F504B5435
:100460003D307825780A00445F54583D307825782F
:100470000A00445F52583D307825780A00445F4FA7
:100480005045523D307825780A0043757272656E8A
:10049000742064656275673D307825580A004E65A2
:1004A000772064656275673D307825580A002573AA
:1004B0000A0025372E33662025372E336600253572
:1004C0002E326620004572726F72203020566F6C9B
:1004D00074004572726F72203020566F6C74004544
:1004E00072726F72203020566F6C740025730A0090
:1004F00025730A0025730A0025730A005854414CDD
:100500005F5452494D3D256400253032780025372F
:100510002E33662025372E33660025352E32662091
:1005200000204E657665722D757365642073746165
:10053000636B203E2025642062797465730A005540
:100540007074696D6520256420646179732C2025A1
:100550003032643A253032643A253032640A00750C
:1005600070677220202020202020202020202020A2
:1005700020202020202020202020202D2072656295
:100580006F6F742076696120626F6F746C6F616445
:1005900065720A0D00626F6F7420202020202020D9
:1005A000202020202020202020202020202020204B
:1005B000202D207265626F6F740A0D00726573746E
:1005C00020656570726F6D20202020202020202063
:1005D00020202020202020202D20726573746F722F
:1005E0006520656570726F6D0A0D0070777231203D
:1005F0005B6F6E7C6F66665D2020202020202020AF
:10060000202020202020202D2070696E312070773E
:10061000720A0D007373202020202020202020202B
:1006200020202020202020202020202020202020CA
:100630002D207374617475732073756D6D6172799B
:100640000A0D00727320202020202020202020204E
:100650002020202020202020202020202020202D8D
:1006600020726164696F2073746174730A0D007283
:1006700069205B696E745D202020202020202020CE
:1006800020202020202020202020202D2072657076
:100690006F727420696E74657276616C0A0D0072F7
:1006A00065205B6D61736B5D202020202020202061
:1006B00020202020202020202020202D206D6F743D
:1006C00065207265706F72742073657474696E67EB
:1006D0000A0D006F772020202020202020202020BD
:1006E0002020202020202020202020202020202DFD
:1006F000206F6E652D776972652073656E736F72FA
:10070000730A0D006C6F67205B6175746F7C6F6E90
:100710007C6F66665D202020202020202020202065
:100720002D206D6F7465732064617461206F6E207D
:100730005553420A0D006E65205B666C7573685DEB
:1007400020202020202020202020202020202020A9
:1007500020202D206E65696768626F722074616267
:100760006C650A0D006D637520202020202020205C
:100770002020202020202020202020202020202079
:10078000202D206D637520696E666F0A0D00696407
:10079000205B72657365745D20202020202020205E
:1007A000202020202020202020202D206964206867
:1007B000616E646C696E670A0D0068756D70205B10
:1007C0006F6E7C6F66665D20202020202020202018
:1007D0002020202020202D2068756D69646974799F
:1007E000207065726D2073656E736F722070777202
:1007F0000A0D0068756D2020202020202020202058
:100800002020202020202020202020202020202DDB
:100810002068756D69646974792073656E736F7291
:100820000A0D006465205B6D61736B5D20202020E4
:100830002020202020202020202020202020202DAB
:100840002064656275670A0D0063616C69205B5BFB
:1008500061317C61327C765F696E5D20766F6C748D
:100860006167655D202D2063616C696272617465EA
:100870000A0D00616573205B6F6E7C6F66665D209C
:100880002020202020202020202020202020202D5B
:1008900020696E746567726574790A0D0075202091
:1008A0002020202020202020202020202020202048
:1008B0002020202020202020202D20757074696D9C
:1008C000650A0D00762020202020202020202020D6
:1008D0002020202020202020202020202020202018
:1008E0002D2076657273696F6E0A0D0068202020D6
:1008F00020202020202020202020202020202020F8
:1009000020202020202020202D2068656C700A0DDA
:1009100000256300756E6B6E6F776E20636D640AE1
:1009200000202573002025362E3266200025303227
:100930007800202573002025362E3266204F6E2D3C
:10094000426F6172640025303278000A004520252C
:10095000642E256420636C6F636B20256C752063A7
:10096000707520256C75206C706D20256C75206964
:10097000727120256C7520676C656420256C75206C
:10098000796C656420256C7520726C656420256C1B
:100990007520747820256C75206C697374656E20E1
:1009A000256C752073656E736F727320256C7520CE
:1009B00073657269616C20256C750A00532025648B
:1009C0002E256420636C6F636B20256C7520747812
:1009D00020256C7520727820256C75207274782023
:1009E000256C752072727820256C75207265786D83
:1009F000697420256C752061636B747820256C7593
:100A0000206E6F61636B747820256C752061636B59
:100A1000727820256C752074696D65646F7574201B
:100A2000256C752062616461636B727820256C753A
:100A300020746F6F6C6F6E6720256C7520746F6FFC
:100A400073686F727420256C752062616473796EAF
:100A5000636820256C752062616463726320256C75
:100A60007520636F6E74656E74696F6E64726F70FB
:100A700020256C752073656E64696E6764726F7093
:100A800020256C75206C6C747820256C75206C6C3E
:100A9000727820256C750A00257325730A004F6E45
:100AA0006C696E650A000A002C20636865636B2020
:100AB0007261746520257520487A0025732025739E
:100AC0002C206368616E6E656C20257520706F77D1
:100AD0006572202575000A0025783A004D414320B3
:100AE00061646472657373200052616E646F6D207F
:100AF00045554936342061646472657373206765B7
:100B00006E6572617465640A000A2A2A2A2A2A2AF2
:100B10002A426F6F74696E672025732A2A2A2A2A4F
:100B20002A2A0A00020000FFFE00000141544D4540
:100B3000474131323872666131006C6F63616C68B5
:100B40006F737400454550524F4D20697320636F99
:100B500072727570742C20726577726974696E6731
:100B600020776974682064656661756C74732E0AF9
:100B7000006E616E00696E660000407A10F35A00E4
:100B8000A0724E18090010A5D4E80000E8764817B6
:100B90000000E40B54020000CA9A3B000000E1F59B
:100BA00005000080969800000040420F000000A061
:100BB0008601000000102700000000E8030000008C
:100BC000006400000000000A0000000000010000B6
:100BD0000000002C76D888DC674F0823DFC1DFAE29
:100BE00059E1B1B796E5E3E453C63AE651997696F2
:100BF000E8E6C28426EB898C9B62ED407C6FFCEFBB
:100C0000BC9C9F40F2BAA56FA5F490055A2AF75CE8
:100C1000936B6CF9676DC11BFCE0E40D47FEF5209A
:100C2000E6B500D0ED902E03009435770500808462
:100C30001E080000204E0A000000C80C3333333376
:100C40000F986E12831141EF8D2114893BE65516E2
:100C5000CFFEE6DB18D1844B381BF77C1D901DA41A
:100C6000BBE424203284725E228100C9F124ECA10D
:100C7000E53D27494E46494E4954594E414ECDCC4B
:100C8000CC3D0AD7233C17B7D13877CC2B3295957A
:100C9000E6241FB14F0A000020410000C842004076
:100CA0001C4620BCBE4CCA1B0E5AAEC59D741124F6
:100CB0001FBECFEFD1E4DEBFCDBF15E0A0E0B2E0B4
:100CC000EEE9F5ED00E00BBF02C007900D92A43DE8
:100CD000B107D9F718E2A4EDB5E001C01D92AE3717
:100CE000B107E1F70E945D370C94CD6A0C940000C7
:100CF000EAECFEE11182108236968FE1E630F807C9
:100D0000C9F70895CF93DF93CAECDEE1E881F9815A
:100D1000309761F18091DC059091DD05A091DE05B1
:100D2000B091DF052A813B814C815D81281B390B05
:100D30004A0B5B0B8091F5059091F605A091F705A4
:100D4000B091F805280F391F4A1F5B1F2A833B8388
:100D50004C835D8312161306140615063CF00995A4
:100D6000198218821A821B821C821D8226968FE1AC
:100D7000C630D80759F68091DC059091DD05A09129
:100D8000DE05B091DF058093F5059093F605A093FD
:100D9000F705B093F805DF91CF910895CF93DF93D6
:100DA000EC01EAECFEE120E030E080819181892BCA
:100DB000B1F4F901EE0FFF1FE20FF31FEE0FFF1F5B
:100DC000DF01A453B14E4D935D936D937C931397C4
:100DD000E653F14ED183C08321E030E008C02F5F9D
:100DE0003F4F36962A30310501F720E030E0C90147
:100DF000DF91CF910895882369F06D987598ED9AE9
:100E000080916A00886080936A00809168008160A8
:100E10008093680008951F920F920FB60F921124CD
:100E20008F939F93AF93BF938091680080FF29C0F9
:100E30008091C61E9091C71E01969093C71E809305
:100E4000C61E8091BE1A9091BF1AA091C01AB0918F
:100E5000C11A0196A11DB11D8093BE1A9093BF1AAD
:100E6000A093C01AB093C11A8091D4059091D50572
:100E700090FF07C0749882E090E09093CE03809337
:100E8000CD03BF91AF919F918F910F900FBE0F90A7
:100E90001F9018951F920F920FB60F9211248F93E7
:100EA0009F93AF93BF938091680080FF29C080918A
:100EB000C81E9091C91E01969093C91E8093C81EAA
:100EC0008091C21A9091C31AA091C41AB091C51A08
:100ED0000196A11DB11D8093C21A9093C31AA093CD
:100EE000C41AB093C51A8091D4059091D50591FF8D
:100EF00007C0739882E090E09093CE038093CD0377
:100F0000BF91AF919F918F910F900FBE0F901F9047
:100F1000189580937C0080917B00877F80937B0075
:100F200080917C00806C80937C0085E080937A00C7
:100F300080917A00806880937A0080917B0087FF9F
:100F4000FCCF80917B0085FFFCCF80917A0080648C
:100F500080937A0080917A0086FDFCCF1092790010
:100F60001092780060E070E020E030E080917A003C
:100F7000806480937A0080917A0086FDFCCF809116
:100F8000780090917900680F791F2F5F3F4F2430D0
:100F9000310561F710927C0080917A008F77809301
:100FA0007A00769567957695679580E090E00E9447
:100FB000D962089580E00E9489072091CF03309183
:100FC000D0034091D1035091D2030E948B6321EE54
:100FD0003AE744E95EE30E940962089580E1809364
:100FE000510190E1909351018091510185FF03C01F
:100FF0009F5F9F31B9F76BE4969FB001112488275A
:1010000077FD8095982F0E94DB6220E030E64FE963
:1010100054E40E94096220E030E04AE754E40E9470
:10102000716208958091F20382FF4BC080917B0032
:10103000886080937B0089EC80937C0085E08093BE
:101040007A0080917A00806880937A0080917B009A
:1010500087FFFCCF80917B0085FFFCCF80917A00D9
:10106000806480937A0080917A0086FDFCCF809125
:101070007A00806480937A0080917A0086FDFCCFAC
:10108000609178007091790080E090E00E94D962D0
:1010900027ED33EA40E95FE30E948B6326E636E6FC
:1010A00048E853E40E9408626093F0117093F111D4
:1010B0008093F2119093F31180917A008F7780934F
:1010C0007A0008958091FC1190917D1A891B0895F2
:1010D0009091FC1180917D1A981719F42FEF3FEF32
:1010E0000FC0E0917D1AF0E0EF71F070E75BFD4E0C
:1010F0008081282F30E080917D1A8F5F80937D1A48
:10110000C901089578948091D7059091D805892BCD
:1011100019F483B7817F03C083B7817F866083BF63
:10112000F89483B7816083BF7894889583B78E7F66
:1011300083BF78940895F89461E2E0E0F0E0609372
:1011400057008491E2E0F0E0609357002491E4E0DE
:10115000F0E060935700649190E0A0E0B0E0DC0123
:101160009927882730E040E050E0542F432F322F5A
:101170002227820F931FA41FB51F860F911DA11D4B
:10118000B11D8093451290934612A0934712B093DD
:101190004812789408950895CF93DF93EC018881E5
:1011A0009981009719F08055974089F40E94820830
:1011B00080918E0990918F0965E840E050E00E948F
:1011C000F72A80E597E09983888381E003C019823C
:1011D000188283E0DF91CF910895E091FC11F0E057
:1011E000EF71F070E75BFD4E80838091FC118F5FA3
:1011F0008093FC118091161F88608093161F42E334
:1012000054E0CA0161E10E94F72A80E090E008956D
:101210001F920F920FB60F920BB60F9211242F93BD
:101220003F934F935F936F937F938F939F93AF936E
:10123000BF93EF93FF938091161F82608093161FD8
:101240008091CD039091CE031816190614F4749A68
:10125000739A8091D4059091D50585FF02C074984A
:1012600073988091DC059091DD05A091DE05B09129
:10127000DF050196A11DB11D8093DC059093DD056E
:10128000A093DE05B093DF058091880490918904D6
:1012900001979093890480938804892B09F05EC09C
:1012A000E091F305F091F4053196F093F405E093A5
:1012B000F30580916D1A90916E1AA0916F1AB091FA
:1012C000701A0196A11DB11D80936D1A90936E1A2C
:1012D000A0936F1AB093701A80E190E09093890404
:1012E000809388048091F60380FD02C01D9B05C099
:1012F0001092D8051092D70506C081E090E0909337
:10130000D8058093D7052091F4033091F50321157A
:10131000310521F1CF010196B9010E940D64892B9D
:10132000B9F477988091D4059091D50593FF10C0BA
:10133000749884E090E09093CE038093CD0308C02E
:101340008EE494E062E140E050E00E94F72A06C09B
:10135000CF01B9010E940D64892B91F3FF91EF91A8
:10136000BF91AF919F918F917F916F915F914F91BD
:101370003F912F910F900BBE0F900FBE0F901F90BB
:1013800018950F931F93CF93DF9301EC19E0CAECEC
:10139000DEE1FE0120E030E080819181892BC9F4FB
:1013A000F901EE0FFF1FE20FF31FEE0FFF1F9F016A
:1013B0002453314E40EA50E060E070E0D9014D9393
:1013C0005D936D937C931397E653F14E11830083E5
:1013D00006C02F5F3F4F36962A303105E9F620E0F0
:1013E00030E088819981892BF1F4F901EE0FFF1F1C
:1013F000E20FF31FEE0FFF1FDF01A453B14E40EACF
:1014000050E060E070E04D935D936D937C93139793
:10141000E653F14E118300838091D4059091D50558
:1014200087FF32C007C02F5F3F4F26962A30310515
:10143000C1F62AC08091DC059091DD05A091DE0502
:10144000B091DF05CDB7DEB72A970FB6F894DEBFAF
:101450000FBECDBFEDB7FEB7319620E032E03A8344
:10146000298382839383A483B583468357836087CC
:1014700071870E94AA672DB73EB7265F3F4F0FB610
:10148000F8943EBF0FBE2DBFDF91CF911F910F91FA
:1014900008950F931F93CF93DF93CAECDEE103E22D
:1014A00012E0288139812115310529F18DB79EB7C8
:1014B00008970FB6F8949EBF0FBE8DBFEDB7FEB76D
:1014C0003196ADB7BEB712961C930E9311978A81D1
:1014D0009B81AC81BD8182839383A483B583378351
:1014E00026830E94AA678DB79EB708960FB6F89418
:1014F0009EBF0FBE8DBF26969FE1C630D90789F6E5
:10150000DF91CF911F910F910895EEE7F8E280816E
:10151000918182549244B9F000D000D081E295E0EC
:10152000ADB7BEB712969C938E931197EE57F842C3
:101530001496FC93EE9313970E94BC670F900F9044
:101540000F900F9008953A96B1E4E53FFB07F8F24B
:1015500008954F925F926F927F928F929F92AF9277
:10156000BF92CF92DF92EF92FF920F931F93609101
:101570006D1A70916E1A80916F1A9091701AE090A6
:101580006D1AF0906E1A00916F1A1091701A809077
:101590006D1A90906E1AA0906F1AB090701A4090C9
:1015A0006D1A50906E1A60906F1A7090701A2DB765
:1015B0003EB72A5030400FB6F8943EBF0FBE2DBF45
:1015C000CDB6DEB60894C11CD11C2FE335E0EDB7D3
:1015D000FEB73283218320E831E541E050E00E94EC
:1015E0003464F60133832283C801B70120E831E572
:1015F00041E050E00E94346420E13EE040E050E0F1
:101600000E943464332727FD3095F6013583248307
:10161000C501B40120E13EE040E050E00E943464A6
:101620002CE330E040E050E00E943464332727FD93
:101630003095F60137832683C301B2012CE330E0F5
:1016400040E050E00E943464772767FD7095F60112
:10165000718760870E94BC672DB73EB7265F3F4FFA
:101660000FB6F8943EBF0FBE2DBF1F910F91FF9094
:10167000EF90DF90CF90BF90AF909F908F907F9032
:101680006F905F904F90089500D08CEE98E0EDB78A
:10169000FEB7928381830E94BC6784EC98E0EDB72B
:1016A000FEB7928381830E94BC678DE998E0EDB715
:1016B000FEB7928381830E94BC6783E798E0EDB711
:1016C000FEB7928381830E94BC6789E498E0EDB7FE
:1016D000FEB7928381830E94BC6783E298E0EDB7F6
:1016E000FEB7928381830E94BC6783EF97E0EDB7DA
:1016F000FEB7928381830E94BC678AEB97E0EDB7C7
:10170000FEB7928381830E94BC678EE897E0EDB7B5
:10171000FEB7928381830E94BC6785E697E0EDB7B0
:10172000FEB7928381830E94BC6786E397E0EDB7A2
:10173000FEB7928381830E94BC6784E097E0EDB797
:10174000FEB7928381830E94BC6783ED96E0EDB77C
:10175000FEB7928381830E94BC678FE996E0EDB764
:10176000FEB7928381830E94BC678FE696E0EDB757
:10177000FEB7928381830E94BC6783E496E0EDB755
:10178000FEB7928381830E94BC6784E196E0EDB747
:10179000FEB7928381830E94BC678BEE95E0EDB724
:1017A000FEB7928381830E94BC678CEB95E0EDB716
:1017B000FEB7928381830E94BC6785E995E0EDB70F
:1017C000FEB7928381830E94BC678FE595E0EDB7F9
:1017D000FEB7928381830E94BC670F900F9008959B
:1017E00000D084E199E0ADB7BEB712969C938E937A
:1017F00011970E94BC672091DB030F900F9022236A
:10180000A9F000D000D0EDB7FEB7319681E199E0A4
:10181000ADB7BEB712969C938E9311972283138215
:101820000E94BC670F900F900F900F90089500D00A
:101830008BE499E0EDB7FEB7928381830E94BC6789
:101840000F900F900895CF92DF92EF92FF920F9337
:101850001F930E94DA0700D000D000D02AE135E0C3
:10186000EDB7FEB7328321836383748385839683C8
:101870000E94BC672DB73EB72A5F3F4F0FB6F89462
:101880003EBF0FBE2DBF81E00E9489072091D30388
:101890003091D4034091D5035091D6030E948B63BD
:1018A0007B018C0182E00E948907EDB7FEB73A9771
:1018B0000FB6F894FEBF0FBEEDBFCDB6DEB60894EE
:1018C000C11CD11C2EE035E0328321839701A80191
:1018D000F60122833383448355832091D7033091CB
:1018E000D8034091D9035091DA030E948B63F6012B
:1018F00066837783808791870E94BC672DB73EB748
:10190000285F3F4F0FB6F8943EBF0FBE2DBF8BE44C
:1019100099E0EDB7FEB7928381830E94BC670F9078
:101920000F901F910F91FF90EF90DF90CF9008954F
:101930008F929F92AF92BF92CF92DF92EF92FF92DF
:101940000F931F93CF93DF934B018091D405909118
:10195000D50581FD74980E94B8305C0181EE95E058
:101960000E94132C0AC0C6010296B4010E94A3284B
:10197000892BE9F4C6010E94302D6C01009799F77C
:10198000E0C0C6010296B4010E949B28D5018C914B
:101990008150888780E091E0A0E0B0E089879A8755
:1019A000AB87BC8781EE95E0B6010E942E2C84E0C7
:1019B0000E940731F6019583848383E00E940731FA
:1019C000D60117969C938E931697F501E080189692
:1019D0008C911897E81AFF2400E010E086E0EE0CE6
:1019E000FF1C001F111F8A95D1F719966D917D91EB
:1019F0008D919C911C9720EC30E040E050E00E94DB
:101A0000EE63672F782F892F9927E60EF71E081FA0
:101A1000191FD6011996ED92FD920D931C931C97F8
:101A2000F501808118968C938091D4059091D5050D
:101A300081FD08C08091F60380FD04C081FF79C05C
:101A40001D9B77C0D60119966D917D918D919C91CA
:101A50001C97EDB7FEB772970FB6F894FEBF0FBE96
:101A6000EDBF0DB71EB70F5F1F4F25E432E0328385
:101A700021830894A11CB11CD8011396BC92AE928C
:101A80001297F401208114962C93149715961C92AA
:101A90001597218116962C93169717961C92D501AF
:101AA0002E91F80120871186D60114962D913C9134
:101AB00015973387228716962D913C911797358776
:101AC0002487272F382F492F55273787268724E645
:101AD00030E040E050E00E94EE63672F782F892FBE
:101AE00099270E943464F801718B608B0E94AA6769
:101AF0002091DB038DB79EB742960FB6F8949EBF38
:101B00000FBE8DBF2223A9F000D000D0EDB7FEB7E5
:101B1000319683E291E0ADB7BEB712969C938E9357
:101B20001197228313820E94BC670F900F900F9031
:101B30000F908091D4059091D50581FF0CC0749AC7
:101B40000AC080E894E00E946D2BEC016C010097C4
:101B500009F017CFEECFDF91CF911F910F91FF903A
:101B6000EF90DF90CF90BF90AF909F908F900895AF
:101B7000CF93DF93EC01109207061092060688813E
:101B80009981009729F0845D924009F0D1C00BC083
:101B90009091FC1180917D1A981749F484ED92E0A0
:101BA0009983888302C0613111F081E0C4C0F89448
:101BB00078949091FC1180917D1A981719F42FEF69
:101BC0003FEF0FC0E0917D1AF0E0EF71F070E75B3E
:101BD000FD4E8081282F30E080917D1A8F5F8093A9
:101BE0007D1AC90190709093E4058093E3058D30D0
:101BF00009F47AC08F3F61F28231910569F18F3724
:101C0000910521F08830910509F052C08091E705D7
:101C10009091E805181619060CF05FC060917828BD
:101C20007091792888E090E00E947E676091782822
:101C30007091792880E290E00E947E676091782818
:101C40007091792888E090E00E947E678091E70596
:101C50009091E80501973DC06091782870917928AE
:101C60008DE090E00E947E671092E6051092E505F7
:101C700013C0E258F54E80816091782870917928E0
:101C800090E00E947E678091E5059091E6050196BF
:101C90009093E6058093E505E091E505F091E60572
:101CA0008091E7059091E805E817F90714F315C04E
:101CB00060917828709179280E947E678091E7056D
:101CC0009091E8052091E305FC01E258F54E208350
:101CD00001969093E8058093E7058091E705909140
:101CE000E805CF9709F054CF10927D1A80917D1AA4
:101CF0008093FC118091E7059091E805FC01E25882
:101D0000F54E108290930706809306061092E80520
:101D10001092E7058091141F9091151F009709F408
:101D200037CF6091F90540E050E00E94F72A30CFAC
:101D30001982188283E0DF91CF910895CF93DF93CA
:101D4000EC0188819981009721F083549740B9F480
:101D50000BC089EE95E060E870E00E94A12E83E45C
:101D600097E09983888306C089EE95E00E943A2D1A
:101D7000892B11F481E006C00E948206EACF198205
:101D8000188283E0DF91CF9108950F931F93CF9333
:101D9000DF93882389F08BE09FE16FEF70E049E0EB
:101DA00050E00E9429678BE09FE164E170E049E028
:101DB00050E00E940C691CC0CBE0DFE109E015E0B7
:101DC00000D000D0EDB7FEB73196ADB7BEB71296D2
:101DD0001C930E9311978991828313820E94BC6792
:101DE0000F900F900F900F90BFE1C331DB0741F7C9
:101DF00000D08BE499E0EDB7FEB7928381830E9417
:101E0000BC670F900F90DF91CF911F910F910895B4
:101E1000EF92FF920F931F936091E0037091E103A3
:101E200080E090E00E941B6761E872E00E943067EA
:101E3000009709F077C08FE892E09093F3038093C6
:101E4000F20382EF93E06EE070E042E050E00E9427
:101E50000C698CE390E09093F5038093F40384EF96
:101E600093E060E170E042E050E00E940C6982E0A3
:101E700090E09093F7038093F60386EF93E062E19E
:101E800070E042E050E00E940C691092D50510927B
:101E9000D40584ED95E060E070E042E050E00E94FF
:101EA0000C690F2EF2E2EF2EFFEFFF2EFCEC0F2F4E
:101EB000FBE31F2FF02DE092D303F092D4030093A5
:101EC000D5031093D60383ED93E066E070E044E021
:101ED00050E00E940C69E092D703F092D80300937F
:101EE000D9031093DA0387ED93E06AE070E044E0F1
:101EF00050E00E940C698DEE97E4AAE8BCE3809361
:101F0000CF039093D003A093D103B093D2038FEC6F
:101F100093E062E070E044E050E00E940C6981E0F0
:101F20000E94C50E1F910F91FF90EF900895729837
:101F3000729A8EE40E94554280EA0E94AE4280E08E
:101F40000E94AE4280E00E94AE428FE40E94554261
:101F50000E94C042282F2295269526952370213075
:101F6000A1F48091751A9091761AA091771AB09188
:101F7000781A0196A11DB11D8093751A9093761A57
:101F8000A093771AB093781A15C0223098F08091F8
:101F9000791A90917A1AA0917B1AB0917C1A0196C5
:101FA000A11DB11D8093791A90937A1AA0937B1A80
:101FB000B0937C1A00D000D0EDB7FEB7319688E818
:101FC00092E0ADB7BEB712969C938E931197228381
:101FD00013820E94AA670F900F900F900F908EE4CB
:101FE0000E94554280E80E94AE4280E00E94AE42CC
:101FF00080E00E94AE420E94A64280E090E00895F8
:10200000EF92FF920F931F93729A8091F60383FDD4
:102010000EC080E090E027EE33E0F901E115F10514
:1020200011F03197F1F7019680359105B1F78EE403
:102030000E9455428823B1F08091711A9091721AD2
:10204000A091731AB091741A0196A11DB11D8093CD
:10205000711A9093721AA093731AB093741A21E0B4
:1020600030E08BC080E090E027EE33E0F901E1152D
:10207000F10511F03197F1F7019680359105B1F72F
:102080008FE40E9455420E94C042082F8295869597
:10209000869583708130A1F48091751A9091761A9B
:1020A000A091771AB091781A0196A11DB11D809365
:1020B000751A9093761AA093771AB093781A15C070
:1020C000823098F08091791A90917A1AA0917B1AB7
:1020D000B0917C1A0196A11DB11D8093791A90933D
:1020E0007A1AA0937B1AB0937C1A0E94C042182FD0
:1020F0000E94C042E82E0E94CA42F82E0E94A642C8
:102100008091F60383FF7298702F7F7360E0610FF8
:10211000711D80E090E00E94D96220E134E048EC3B
:102120005BE30E948B636093691270936A128093E1
:102130006B1290936C127E2D60E06F0D711D769581
:1021400067957695679580E090E00E94D96224EAD1
:102150003CEF44E25CE30E948B6320E030E040E22D
:1021600052E40E9408626093171F7093181F8093B7
:10217000191F90931A1F20E030E0C9011F910F91A1
:10218000FF90EF9008950E9412088091F2039091C1
:10219000F30390FF02C00E9400108091F20390911F
:1021A000F30391FF0AC00E94DA076093061F709341
:1021B000071F8093081F9093091F0895DF93CF9303
:1021C00000D0CDB7DEB780910C1F89838091121F9C
:1021D0008A83CE0101960E94B7280F900F90CF916D
:1021E000DF910895DF93CF9300D000D000D0CDB71A
:1021F000DEB7CE0101966EE070E042E050E00E9452
:10220000EE6889819A812FEF8F3F920749F482EF20
:1022100093E06EE070E042E050E00E940C6904C080
:102220009093F3038093F203CE01019660E170E096
:1022300042E050E00E94EE6889819A812FEF8F3F43
:10224000920779F48CE390E09093F5038093F40384
:1022500084EF93E060E170E042E050E00E940C699E
:1022600004C09093F5038093F403CE01019662E1DC
:1022700070E042E050E00E94EE6889819A812FEF81
:102280008F3F920779F482E090E09093F703809378
:10229000F60386EF93E062E170E042E050E00E94D6
:1022A0000C6904C09093F7038093F603CE01019666
:1022B00060E070E042E050E00E94EE6889819A811F
:1022C0002FEF8F3F920769F41092D5051092D40535
:1022D00084ED95E060E070E042E050E00E940C691F
:1022E00004C09093D5058093D4058BE09FE164E111
:1022F00070E049E050E00E94EE680E94DE10CE01DE
:10230000039666E070E044E050E00E94EE688B8146
:102310009C81AD81BE818F5F9F4FAF4FBF4F49F40E
:1023200083ED93E066E070E044E050E00E940C69C9
:1023300008C083ED93E066E070E044E050E00E9466
:10234000EE68CE0103966AE070E044E050E00E943F
:10235000EE688B819C81AD81BE818F5F9F4FAF4FB7
:10236000BF4F49F487ED93E06AE070E044E050E04D
:102370000E940C6908C087ED93E06AE070E044E0D9
:1023800050E00E94EE68CE01039662E070E044E007
:1023900050E00E94EE688B819C81AD81BE818F5F91
:1023A0009F4FAF4FBF4F49F48FEC93E062E070E076
:1023B00044E050E00E940C6908C08FEC93E062E0BA
:1023C00070E044E050E00E94EE6826960FB6F89464
:1023D000DEBF0FBECDBFCF91DF9108954F925F92C8
:1023E0006F927F928F929F92AF92BF92DF92EF9205
:1023F000FF920F931F93DF93CF93CDB7DEB729974B
:102400000FB6F894DEBF0FBECDBF4C011092DB05B6
:102410008FEF898365E0E62E62E1F62E00E010E0A2
:1024200052E0A52EB12CAC0EBD1E2E010894411C0D
:10243000511C4AE0642E712C6C0E7D1E4AC008307F
:10244000110519F438E0D32E49C0C201B5010E942C
:10245000A73589818F3F11F08E3F19F48093DB05FA
:102460003DC081149104D1F4C5010E94923580933E
:10247000131F20E030E0AE014E5F5F4FF901E55FD2
:10248000F04EDA01A20FB31F8C9180832F5F3F4F74
:102490002830310599F7DD24D39420C0C5010E946E
:1024A0009235F7018083D501F80123E0EE0FFF1F7D
:1024B0002A95E1F7E00FF11FE350FE4E8D918193D5
:1024C000A615B705D9F70F5F1F4F89E090E0E80E1A
:1024D000F91ED02E8981882309F0B1CF8D2D299640
:1024E0000FB6F894DEBF0FBECDBFCF91DF911F9125
:1024F0000F91FF90EF90DF90BF90AF909F908F90E3
:102500007F906F905F904F9008956F927F928F921F
:102510009F92AF92BF92CF92DF92EF92FF920F9372
:102520001F93DF93CF93CDB7DEB7C556D0400FB61C
:10253000F894DEBF0FBECDBF3C01162F633821F4E7
:102540008BEF95E00E94D928D3018D919C91009743
:1025500029F08459964009F0AFC40EC08BEF95E086
:1025600061E870E04CE754E00E94DC2884E996E0E2
:10257000F3019183808302C0123111F081E0A0C485
:102580000E94C3108091F20380FD03C0AA24BB24E3
:102590005BC0B2E0CB2ED12CCC0EDD1E00D000D023
:1025A00000D0EDB7FEB73196ADB7BEB71296DC924C
:1025B000CE92119784E690E09383828388E992E03B
:1025C000958384830E941B685C010BE01FE1EDB7DB
:1025D000FEB736960FB6F894FEBF0FBEEDBFA4E669
:1025E000EA2EF12CFCE98F2EF2E09F2E2DB73EB79C
:1025F000285030400FB6F8943EBF0FBE2DBFEDB748
:10260000FEB73196C6018A0D9B1DADB7BEB71296B7
:102610009C938E931197F382E28295828482D801F3
:102620008D918D01868317820E941B68A80EB91EAA
:10263000EDB7FEB738960FB6F894FEBF0FBEEDBFEC
:10264000FFE103311F0791F68091F2039091F303AC
:10265000892B81F12DB73EB7285030400FB6F89442
:102660003EBF0FBE2DBFEDB7FEB73196CE0102962D
:102670008A0D9B1DADB7BEB712969C938E93119792
:1026800084E690E09383828381EA92E09583848359
:102690008091D7059091D805978386830E941B6807
:1026A000A80EB91EEDB7FEB738960FB6F894FEBF68
:1026B0000FBEEDBF8091F20381FF4FC089E290E031
:1026C0006BE270E04AE250E027E00E94D0328BE0FB
:1026D0009FE10E9422352DB73EB72A5030400FB6F9
:1026E000F8943EBF0FBE2DBF0DB71EB70F5F1F4F33
:1026F0009E012E5F3F4F2A0D3B1DADB7BEB7129610
:102700003C932E93119724E630E0F8013383228323
:1027100028EA32E035832483AA2797FDA095BA2FB3
:10272000BC01CD010E94DB6220E030E048EC52E4C5
:102730000E947162D80116966D937D938D939C9340
:1027400019970E941B68A80EB91EEDB7FEB73A96FE
:102750000FB6F894FEBF0FBEEDBF8091F2039091CB
:10276000F30394FF55C089E290E06BE270E04AE227
:1027700050E026E00E94D03281E090E00E94EE110D
:102780008093DA058DEF91E10E9422352DB73EB797
:102790002A5030400FB6F8943EBF0FBE2DBF0DB784
:1027A0001EB70F5F1F4F9E012E5F3F4F2A0D3B1D2F
:1027B000ADB7BEB712963C932E93119724E630E046
:1027C000F8013383228322EB32E035832483AA2766
:1027D00097FDA095BA2FBC01CD010E94DB6220E0DD
:1027E00030E048EC52E40E947162D80116966D9375
:1027F0007D938D939C9319970E941B68A80EB91E18
:10280000EDB7FEB73A960FB6F894FEBF0FBEEDBF18
:102810008091F20382FF36C02DB73EB72A50304078
:102820000FB6F8943EBF0FBE2DBFEDB7FEB7319681
:10283000CE0102968A0D9B1DADB7BEB712969C9332
:102840008E93119784E690E0938382838DEB92E0E0
:10285000958384838091F0119091F111A091F211F0
:10286000B091F31186839783A087B1870E941B687C
:10287000A80EB91EEDB7FEB73A960FB6F894FEBF94
:102880000FBEEDBF8091F20383FF31C00E94EE07BF
:102890002DB73EB72A5030400FB6F8943EBF0FBE5A
:1028A0002DBFEDB7FEB731969E012E5F3F4F2A0D2B
:1028B0003B1DADB7BEB712963C932E93119724E6FD
:1028C00030E0338322832BEC32E03583248366832C
:1028D0007783808791870E941B68A80EB91EEDB789
:1028E000FEB73A960FB6F894FEBF0FBEEDBF8091CB
:1028F000F20384FF35C02091BE1A3091BF1A409177
:10290000C01A5091C11A8DB79EB70A970FB6F894A6
:102910009EBF0FBE8DBFEDB7FEB73196CE010296BA
:102920008A0D9B1DADB7BEB712969C938E931197DF
:1029300084E690E09383828389ED92E0958384839B
:1029400026833783408751870E941B68A80EB91ED3
:10295000EDB7FEB73A960FB6F894FEBF0FBEEDBFC7
:102960008090F4039090F5038091F2039091F3032B
:102970008821992185FF68C06091BE1A7091BF1AA5
:102980008091C01A9091C11AE090F411F090F51165
:102990000091F6111091F7112DB73EB72A50304033
:1029A0000FB6F8943EBF0FBE2DBFCDB6DEB608946D
:1029B000C11CD11C9E012E5F3F4F2A0D3B1DADB7A0
:1029C000BEB712963C932E93119724E630E0F601A1
:1029D0003383228322EE32E0358324836E197F090C
:1029E000800B910B0E94D9627B018C01B40180E0C5
:1029F00090E00E94D9629B01AC01C801B7010E941E
:102A00007162D60116966D937D938D939C93199761
:102A10000E941B68A80EB91E8091BE1A9091BF1A21
:102A2000A091C01AB091C11A8093F4119093F5113E
:102A3000A093F611B093F711EDB7FEB73A960FB623
:102A4000F894FEBF0FBEEDBF8091F20386FF35C044
:102A50002091C21A3091C31A4091C41A5091C51ADC
:102A60008DB79EB70A970FB6F8949EBF0FBE8DBF65
:102A7000EDB7FEB73196CE0102968A0D9B1DADB71C
:102A8000BEB712969C938E93119784E690E0938341
:102A9000828389ED92E09583848326833783408700
:102AA00051870E941B68A80EB91EEDB7FEB73A9673
:102AB0000FB6F894FEBF0FBEEDBF8091F20387FF03
:102AC00035C020916D1A30916E1A40916F1A509155
:102AD000701A8DB79EB70A970FB6F8949EBF0FBEB7
:102AE0008DBFEDB7FEB73196CE0102968A0D9B1DC4
:102AF000ADB7BEB712969C938E93119784E690E083
:102B0000938382838FEE92E0958384832683378339
:102B1000408751870E941B68A80EB91EEDB7FEB70B
:102B20003A960FB6F894FEBF0FBEEDBF8091F20348
:102B30009091F30390FF36C02DB73EB72A50304036
:102B40000FB6F8943EBF0FBE2DBFEDB7FEB731965E
:102B5000CE0102968A0D9B1DADB7BEB712969C930F
:102B60008E93119784E690E09383828388EF92E0BE
:102B7000958384838091691290916A12A0916B125F
:102B8000B0916C1286839783A087B1870E941B68DF
:102B9000A80EB91EEDB7FEB73A960FB6F894FEBF71
:102BA0000FBEEDBF8091F2039091F30391FF36C009
:102BB0002DB73EB72A5030400FB6F8943EBF0FBE37
:102BC0002DBFEDB7FEB73196CE0102968A0D9B1D43
:102BD000ADB7BEB712969C938E93119784E690E0A2
:102BE0009383828383E093E0958384838091061F9F
:102BF0009091071FA091081FB091091F86839783AA
:102C0000A087B1870E941B68A80EB91EEDB7FEB75A
:102C10003A960FB6F894FEBF0FBEEDBF8091F20357
:102C20009091F30392FF41C081E00E9489072DB784
:102C30003EB72A5030400FB6F8943EBF0FBE2DBFAE
:102C40000DB71EB70F5F1F4F9E012E5F3F4F2A0D1E
:102C50003B1DADB7BEB712963C932E93119724E659
:102C600030E0F8013383228320E133E0358324838D
:102C70002091D3033091D4034091D5035091D603D2
:102C80000E948B63D80116966D937D938D939C93D0
:102C900019970E941B68A80EB91EEDB7FEB73A96A9
:102CA0000FB6F894FEBF0FBEEDBF8091F203909176
:102CB000F30393FF41C082E00E9489072DB73EB71E
:102CC0002A5030400FB6F8943EBF0FBE2DBF0DB74F
:102CD0001EB70F5F1F4F9E012E5F3F4F2A0D3B1DFA
:102CE000ADB7BEB712963C932E93119724E630E011
:102CF000F801338322832DE133E03583248320914F
:102D0000D7033091D8034091D9035091DA030E9440
:102D10008B63D80116966D937D938D939C93199731
:102D20000E941B68A80EB91EEDB7FEB73A960FB603
:102D3000F894FEBF0FBEEDBF779A8091D4059091B5
:102D4000D50593FD749A8091D4059091D50582FDA7
:102D500008C08091F60380FD04C081FF31C01D9B37
:102D60002FC000D000D08AE293E0ADB7BEB7129674
:102D70009C938E931197CE01029614969C938E93FA
:102D800013970E94AA672091DB030F900F900F907A
:102D90000F902223A9F000D000D0EDB7FEB73196F6
:102DA00080E291E0ADB7BEB712969C938E931197D7
:102DB000228313820E94BC670F900F900F900F9098
:102DC0008091E0058983FE01EA0DFB1D12828501D9
:102DD0000E5F1F4F5E010894A11CB11CC501B80114
:102DE0000E9434328091F60382FF45C082EE93E068
:102DF000B501A80126EC3AE10E94D4428091D405A5
:102E00009091D50592FF37C0E6ECAE2EEAE1BE2EDA
:102E100071E3872E73E0972E00D000D0EDB7FEB798
:102E20003196ADB7BEB712969C928E921197D5018E
:102E30008D915D01828313820E94AA670F900F908B
:102E40000F900F90B6EDAB16BAE1BB0629F78AE0FA
:102E500090E00E94DF6700D000D086E393E0EDB7FA
:102E6000FEB792838183148303830E94AA670F9025
:102E70000F900F900F908091D4059091D50582FD11
:102E800073980E944A3C8BEF95E00E94CB2880917A
:102E9000D7059091D805892B11F00E944A3D809169
:102EA000E0058F5F8093E0058091D4059091D50572
:102EB00082FF5CCB739A5ACBD3011D921C9283E0A4
:102EC000CB59DF4F0FB6F894DEBF0FBECDBFCF9109
:102ED000DF911F910F91FF90EF90DF90CF90BF9007
:102EE000AF909F908F907F906F900895CF93DF93D6
:102EF000EC0180910B1F8F3FB1F580910C1F8F3F2C
:102F000091F580910D1F8F3F71F580910E1F8F3FBE
:102F100051F580910F1F8F3F31F58091101F8F3F2A
:102F200011F58091111F8F3FF1F48091121F8F3F97
:102F3000D1F489E290E06BE270E04AE250E027E0F1
:102F40000E94D03280E090E00E94EE11C752DA4F2A
:102F500088838BE09FE164E170E049E050E00E94EB
:102F60000C690E94DE10DF91CF9108956C9A6B9AE4
:102F70006A9A6F9A729A749A739A779A809880B3C1
:102F8000897F80BB87E080937E00549AF89461E249
:102F9000E0E0F0E0609357008491E2E0F0E06093BD
:102FA00057002491E4E0F0E060935700649190E0D2
:102FB000A0E0B0E0DC019927882730E040E050E055
:102FC000542F432F322F2227820F931FA41FB51F88
:102FD000860F911DA11DB11D80934512909346123D
:102FE000A0934712B093481278940E94F2106D9803
:102FF0007598ED9AEAE6F0E0808188608083E8E6E3
:10300000F0E080818160808380E090E00E9476170C
:103010000E944F4208952F923F924F925F926F927B
:103020007F928F929F92AF92BF92CF92DF92EF9258
:10303000FF920F931F93CF93DF93EC01009741F41E
:1030400089E290E06BE270E04AE250E027E00AC0DB
:103050008130910549F489E290E06BE270E04AE248
:1030600050E026E00E94D032CE010E94EE11FE0117
:10307000E752FA4F8083CD2BA1F00DEFC02E01E176
:10308000D02EEE24FF244F0115E2212E19E0312E1F
:10309000B1E24B2EB9E05B2EABE46A2EA9E07A2EAA
:1030A000ECC08BE09FE10E9422357C01CBE0DFE1A8
:1030B00006E419E000D000D0EDB7FEB73196ADB709
:1030C000BEB712961C930E93119789918283138237
:1030D0000E94BC670F900F900F900F90BFE1C3311B
:1030E000DB0741F700D000D000D00DB71EB70F5F4F
:1030F0001F4F86E399E0EDB7FEB792838183B70156
:10310000882777FD8095982F0E94DB6220E030E0D1
:1031100048EC52E40E947162D80112966D937D933F
:103120008D939C9315970E94BC67EDB7FEB73696BA
:103130000FB6F894FEBF0FBEEDBF8881882319F447
:103140002EE333E002C02FE333E000D000D082E36F
:1031500099E0ADB7BEB712969C938E9311971496D3
:103160003C932E9313970E94BC670F900F908BE4B3
:1031700099E0EDB7FEB7928381830E94BC670F9000
:103180000F9082C0C6010E9422355C01E701F3E086
:10319000CC0FDD1FFA95E1F7CE0DDF1DC350DE4EDB
:1031A00000E010E000D000D0EDB7FEB731968DE220
:1031B00099E0ADB7BEB712969C938E931197899103
:1031C000828313820E94BC670F5F1F4F0F900F9086
:1031D0000F900F900830110529F700D000D000D0D3
:1031E0000DB71EB70F5F1F4FADB7BEB712963C921B
:1031F0002E921197B501882777FD8095982F0E9410
:10320000DB6220E030E048EC52E40E947162F80199
:1032100062837383848395830E94BC678DB79EB756
:1032200006960FB6F8949EBF0FBE8DBFD6011896B6
:103230008C91882319F48EE393E002C08FE393E02E
:1032400000D000D0EDB7FEB75282418294838383D1
:103250000E94BC670F900F90ADB7BEB712967C92DC
:103260006E9211970E94BC670894E11CF11CE9E082
:10327000F0E0CE0EDF1E0F900F90D4018C9190E005
:10328000E816F9060CF47ECFDF91CF911F910F91D4
:10329000FF90EF90DF90CF90BF90AF909F908F9076
:1032A0007F906F905F904F903F902F90089588E4AB
:1032B00093E00E94E66708952F923F924F925F92AB
:1032C0006F927F928F929F92AF92BF92CF92DF9236
:1032D000EF92FF920F931F93DF93CF93CDB7DEB79B
:1032E00028970FB6F894DEBF0FBECDBF9D838C83A9
:1032F000DC018D919C91892B11F00C94EA2760914F
:10330000E0037091E1038EE79AE10E941B678EE76C
:103310009AE160E470E00E943967009759F4609187
:103320007828709179288AE090E00E947E6781E099
:103330000C94EF278130910551F480917E1A282E4C
:10334000332444245524662477244301D4C1823095
:103350009105A1F420917E1A30917F1A922F80E07E
:10336000830F911D9C01330F220B322F1C01422E23
:10337000522E622E722E822E922EBDC18330910566
:1033800009F0A6C020917E1A80907F1AB091801A11
:10339000BB8330E040E050E060E070E080E090E02F
:1033A00000E10E94845D122F732E642E552E462E4E
:1033B000372E282E9E83282D30E040E050E060E03C
:1033C00070E080E090E008E00E94845D210FE1E081
:1033D000211708F0E0E0370DF1E0371508F0F0E0D4
:1033E000BE2FB30FE1E0B31708F0E0E0FE2B460D6F
:1033F000E1E0461508F0E0E0AF2FA40F31E0A4179C
:1034000008F030E0E32B550D41E0551508F040E0A1
:10341000FE2EF50E31E0F51608F030E0432B640D7A
:1034200051E0641508F050E0E42EE60E31E0E616B7
:1034300008F030E0532B730D41E0731508F040E0C5
:10344000652F670F31E0671708F030E0432B820DDE
:1034500031E0821508F030E0542F580F41E0581742
:1034600008F040E0342BEE819E0F930F0B81020F8A
:1034700081E0021708F080E0182F1B0F81E01B1776
:1034800008F080E0B82FBA0F81E0BA1708F080E0AA
:10349000782F7F0D81E07F1508F080E0482F4E0DDA
:1034A00081E04E1508F080E0382F360F81E03617A6
:1034B00008F080E0850F21E0851708F020E0180172
:1034C0004B2E572E642E732E882E922E990E13C1DA
:1034D0008430910551F08AE0282E33244424552469
:1034E000662477248824992406C120917E1A80902E
:1034F0007F1AF091801AFA833091811A398330E073
:1035000040E050E060E070E080E090E008E10E9480
:10351000845D122F732E642E552E462E372E282EA4
:103520009F83282D30E040E050E060E070E080E0D4
:1035300090E000E10E94845D210FE1E0211708F096
:10354000E0E0370DF1E0371508F0F0E0BE2FB30FE3
:10355000E1E0B31708F0E0E0FE2B460DE1E0461590
:1035600008F0E0E0AF2FA40F31E0A41708F030E03E
:10357000E32B550D41E0551508F040E00E2F050FE7
:1035800031E0051708F030E0432B640D51E064157D
:1035900008F050E0B42EB60E31E0B61608F030E078
:1035A000532B730D41E0731508F040E0652F670F52
:1035B00031E0671708F030E0432B820D31E08215CF
:1035C00008F030E0542F580F41E0581708F040E061
:1035D000342B4F81490F430FF980F20E81E0F21630
:1035E00008F080E0182F1B0F81E01B1708F080E027
:1035F000E82EEA0E81E0EA1608F080E0D82ED00E20
:1036000081E0D01608F080E0C82ECB0C81E0CB140E
:1036100008F080E0B82EB60E81E0B61608F080E023
:10362000A82EA50E91E0A51608F090E0940F9887BB
:10363000AA812A2F30E040E050E060E070E080E0B6
:1036400090E008E00E94845D2F0DE1E02F1508F066
:10365000E0E0310FF1E0311708F0F0E0BE2FB30FDA
:10366000E1E0B31708F0E0E0FE2B4E0DE1E04E156F
:1036700008F0E0E0AF2FA40F31E0A41708F030E02D
:10368000E32B5D0D41E05D1508F040E01E2F150FA6
:1036900031E0151708F030E0432B6C0D51E06C154C
:1036A00008F050E0042F060F31E0061708F030E074
:1036B000532B7B0D41E07B1508F040E0652F670F31
:1036C00031E0671708F030E0432B8A0D51E08A158E
:1036D00008F050E0480F31E0481708F030E0532B75
:1036E000E885E90F222E3B2E4A2E512E602E762E93
:1036F000842E9E2E950E00D08BE499E0ADB7BEB718
:1037000012969C938E9311970E94BC670F900F9016
:10371000B2E62B1689F4E5E63E1671F4F4E64F1690
:1037200059F4552049F4662039F4772029F488208B
:1037300019F4992009F40DC59101A201B301C40146
:1037400002E6A02E15E6B12EB4E6CB2EDD24EE2443
:10375000FF2400E010E00E94035E823008F099C16F
:1037600027E7221681F43FE6331669F4442059F422
:10377000552049F4662039F4772029F4882019F47B
:10378000992009F4DBC79101A201B301C401A7E7A5
:10379000AA2EFFE6BF2ECC24DD24EE24FF2400E079
:1037A00010E00E94035E823008F0B6C084E628165E
:1037B00089F491E6391671F4442061F4552051F4EE
:1037C000662041F4772031F4882021F4992011F407
:1037D0000C9448279101A201B301C401E4E6AE2E86
:1037E00001E6B02ECC24DD24EE24FF2400E010E01E
:1037F0000E94035E823008F046C0A5E72A1679F4DD
:10380000332069F4442059F4552049F4662039F4F2
:10381000772029F4882019F4992009F4CAC5B6E75D
:103820002B1679F4332069F4442059F4552049F4D7
:10383000662039F4772029F4882019F4992009F4B6
:10384000C7C5E8E62E1611F00C94E827332011F0D6
:103850000C94E827442011F00C94E827552011F02F
:103860000C94E827662011F00C94E827772011F0DB
:103870000C94E827882011F00C94E827992011F087
:103880000C94E82765C5F4E62F1681F429E6321674
:1038900069F4442059F4552049F4662039F477201E
:1038A00029F4882019F4992009F455C535E6231622
:1038B00081F48EE6381669F4442059F4552049F411
:1038C000662039F4772029F4882019F4992009F426
:1038D00099C795E6291611F00C94E827A4E63A1644
:1038E00011F00C94E827442011F00C94E82755209F
:1038F00011F00C94E827662011F00C94E82777204B
:1039000011F00C94E827882011F00C94E8279920F6
:1039100011F00C94E8271DC4B3E72B1689F4E2E7F5
:103920003E1671F4442061F4552051F4662041F4B0
:10393000772031F4882021F4992011F40C94D325B8
:103940009101A201B301C40113E7A12EB2E7BB2E7E
:10395000CC24DD24EE24FF2400E010E00E94035E6E
:10396000823008F04AC0F5E62F1679F43B1469F46A
:10397000442059F4552049F4662039F4772029F47D
:10398000882019F4992009F4A7C729E6221689F49A
:1039900032E7331671F4442061F4552051F4662067
:1039A00041F4772031F4882021F4992011F40C940B
:1039B000802583E3281611F00C94E82791E7391647
:1039C00011F00C94E827442011F00C94E8275520BE
:1039D00011F00C94E827662011F00C94E82777206A
:1039E00011F00C94E827882011F00C94E827992016
:1039F00011F00C94E8270C944827A3E62A1691F4BA
:103A0000B4E63B1679F4E1E64E1661F4552051F424
:103A1000662041F4772031F4882021F4992011F4B4
:103A20000C944827F3E72F1689F425E6321671F433
:103A300031E6431659F4552049F4662039F47720CD
:103A400029F4882019F4992009F4D3C483E72816AF
:103A500011F00C94E827381611F00C94E827442054
:103A600011F00C94E827552011F00C94E8276620FB
:103A700011F00C94E827772011F00C94E8278820A7
:103A800011F00C94E827992011F00C94E8270C947D
:103A9000E22594E7291689F4AFE63A1671F44A163E
:103AA00061F4B2E65B1649F4662039F4772029F414
:103AB000882019F4992009F4CBC49101A201B30123
:103AC000C401A4E7AA2EFFE6BF2EEFE6CE2E02E643
:103AD000D02EEE24FF2400E010E00E94035E82302E
:103AE00008F0A4C0E5E72E1689F4F3E63F1671F45A
:103AF0002DE6421659F4552049F4662039F4772012
:103B000029F4882019F4992009F493C59101A201A0
:103B1000B301C40115E7A12EB3E6BB2EADE6CA2E54
:103B2000DD24EE24FF2400E010E00E94035E8230DA
:103B300090F52C1489F43A1479F438E6431661F4BC
:103B4000552051F4662041F4772031F4882021F487
:103B5000992011F40C94572787E6281689F49FE6DC
:103B6000391671F4ACE64A1659F4552049F466202A
:103B700039F4772029F4882019F4992009F49CC499
:103B8000B2E72B1611F00C94E8273B1611F00C94B9
:103B9000E827E5E632C0F1E32F1681F43F1671F411
:103BA00021E7421659F4552049F4662039F477206C
:103BB00029F4882019F4992009F43BC530E723162D
:103BC00089F485E6381671F492E7491659F45520C0
:103BD00049F4662039F4772029F4882019F49920D3
:103BE00009F47AC6A0E32A1611F00C94E827B1E391
:103BF0003B1611F00C94E827E1E74E1611F00C94F7
:103C0000E827552011F00C94E827662011F00C9459
:103C1000E827772011F00C94E827882011F00C9405
:103C2000E827992011F00C94E827ABC4F0E72F1691
:103C300091F42DE6321679F435E7431661F488E6FF
:103C4000581649F4662039F4772029F4882019F4AD
:103C5000992009F4A2C59101A201B301C401F0E7C2
:103C6000AF2EEDE6BE2E05E7C02E18E6D12EEE24CF
:103C7000FF2400E010E00E94035E823008F04DC097
:103C80002A1489F49CE6391671F4A5E64A1659F40B
:103C90005D1449F4662039F4772029F4882019F45A
:103CA000992009F455C3B1E62B1691F4EDE63E16C2
:103CB00079F4F5E74F1661F428E6521649F46620C8
:103CC00039F4772029F4882019F4992009F44BC598
:103CD00039E6231611F00C94E8278CE6381611F01B
:103CE0000C94E82791E6491611F00C94E827A3E616
:103CF0005A1611F00C94E827662011F00C94E8276E
:103D0000772011F00C94E827882011F00C94E82714
:103D1000992011F00C94E827B0C0B4E72B1691F469
:103D2000E3E73E1679F4F5E64F1661F422E7521602
:103D300049F4662039F4772029F4882019F4992071
:103D400009F4C7C59101A201B301C401B4E7AB2EC8
:103D5000A3E7BA2EF5E6CF2EE2E7DE2EEE24FF240F
:103D600000E010E00E94035E823020F531E323166C
:103D700011F00C94E8273D1411F00C94E82787E724
:103D8000481611F00C94E82790E7591611F00C949E
:103D9000E827662011F00C94E827772011F00C94A6
:103DA000E827882011F00C94E827992011F00C9452
:103DB000E8273BC0A2E72A1691F4B7E63B1679F450
:103DC000E0E74E1661F4F5E75F1649F4662039F432
:103DD000772029F4882019F4992009F43CC32CE6B3
:103DE000221611F00C94E82731E6331611F00C94EA
:103DF000E82784E7481611F00C94E82798E759164D
:103E000011F00C94E827662011F00C94E827772035
:103E100011F00C94E827882011F00C94E8279920E1
:103E200011F00C94E8270C94A5276091E0037091A1
:103E3000E10380E090E00E941B678C0169E673E07B
:103E40000E943067009719F477980C94EA27C8010C
:103E50006CE673E00E943067009719F4779A0C942F
:103E6000EA27779B03C02CE633E002C029E633E063
:103E700000D000D08EEA94E079C36091E0037091A5
:103E8000E10380E090E00E941B678C0160E773E033
:103E90000E943067009709F047C06091E00370917D
:103EA000E10380E090E00E941B678C01009711F411
:103EB0000C94EA2763E773E00E943067009769F487
:103EC00082E29FEFACECBBE38093D3039093D403E7
:103ED000A093D503B093D6031EC0C8010E940E66FE
:103EE0007B018C0120E030E040E050E00E946D62F8
:103EF0008823B1F081E00E9489079B01AC01C801D1
:103F0000B7010E9471626093D3037093D4038093CE
:103F1000D5039093D60383ED93E066E070E0A6C0EE
:103F200000D08FED94E0A8C0C80169E773E00E945B
:103F30003067009709F048C06091E0037091E10399
:103F400080E090E00E941B678C01009711F40C94B4
:103F5000EA2763E773E00E943067009769F482E222
:103F60009FEFACECBBE38093D7039093D803A0936F
:103F7000D903B093DA031EC0C8010E940E667B010C
:103F80008C0120E030E040E050E00E946D62882328
:103F9000B1F082E00E9489079B01AC01C801B70122
:103FA0000E9471626093D7037093D8038093D90302
:103FB0009093DA0387ED93E06AE070E057C000D099
:103FC00082ED94E00C94DD27C8016CE773E00E9459
:103FD0003067009709F053C06091E0037091E103EE
:103FE00080E090E00E941B678C01009711F40C9414
:103FF000EA2763E773E00E943067009769F48DEE6B
:1040000097E4AAE8BCE38093CF039093D003A093F6
:10401000D103B093D20326C0C8010E940E665B0193
:104020006C0120E030E040E050E00E946D628823A7
:1040300001F180E00E9489077B018C01C601B50176
:1040400021EE3AE744E95EE30E940862A801970185
:104050000E9471626093CF037093D0038093D10369
:104060009093D2038FEC93E062E070E044E050E084
:1040700062C400D085EC94E0EDB7FEB767C00E9443
:10408000DA0700D000D000D02EEB34E0ADB7BEB7D9
:1040900012963C932E931197EDB7FEB7638374830A
:1040A000858396830E94BC672DB73EB72A5F3F4F3A
:1040B0000FB6F8943EBF0FBE2DBF81E00E94890766
:1040C0002091D3033091D4034091D5035091D6036E
:1040D0000E948B637B018C0182E00E948907ADB74F
:1040E000BEB71A970FB6F894BEBF0FBEADBFCDB620
:1040F000DEB60894C11CD11C22EB34E012963C932E
:104100002E9311979701A801F601228333834483EC
:1041100055832091D7033091D8034091D903509112
:10412000DA030E948B63D60116966D937D938D936F
:104130009C9319970E94BC67EDB7FEB738960FB6EF
:10414000F894FEBF0FBEEDBF8BE499E092838183AC
:104150003AC76091E0037091E10380E090E00E9433
:104160001B67009771F160E070E040E150E00E9451
:10417000F8649B01AC018091D4059091D50582171C
:10418000930799F13093D5052093D40584ED95E0FC
:1041900060E070E042E050E00E940C692091D4059C
:1041A0003091D50500D000D08EE994E0ADB7BEB710
:1041B00012969C938E93119714963C932E9313977B
:1041C0000EC02091D4053091D50500D000D08AE8EA
:1041D00094E0EDB7FEB792838183348323830E94FA
:1041E000BC670F900F900F900F9000D08BE499E078
:1041F000ADB7BEB712969C938E9311970E94BC6781
:1042000000D08DE794E0EDB7FEB79283818381E023
:1042100090E0948383830E94BC6782E794E0ADB70B
:10422000BEB712969C938E93119782E090E01496FD
:104230009C938E9313970E94BC6787E694E0EDB73A
:10424000FEB79283818384E090E0948383830E940D
:10425000BC678BE594E0ADB7BEB712969C938E9386
:10426000119788E090E014969C938E9313970E9488
:10427000BC6780E594E0EDB7FEB79283818380E16F
:1042800090E0948383830E94BC6784E494E0ADB79C
:10429000BEB712969C938E93119780E290E014968D
:1042A0009C938E9313970E94BC6786E394E0EDB7CE
:1042B000FEB79283818380E490E0948383830E949D
:1042C000BC6788E294E0ADB7BEB712969C938E931C
:1042D000119780E890E014969C938E9313970E9418
:1042E000BC6789E194E0EDB7FEB79283818380E0FB
:1042F00091E0948383830E94BC678AE094E0ADB729
:10430000BEB712969C938E93119780E092E014961C
:104310009C938E9313970E94BC678EEF93E0EDB74A
:10432000FEB79283818380E094E0948383830E942C
:10433000BC6780EF93E0ADB7BEB712969C938E93A7
:10434000119780E098E014969C938E9313972AC05F
:104350000E94440B3FC66091E0037091E10380E04E
:1043600090E00E941B6763E773E00E94306700974C
:1043700011F481E001C080E00E94C50E2091DB03B2
:10438000222309F427C600D000D0EDB7FEB731963E
:104390008DEE93E0ADB7BEB712969C938E931197B6
:1043A000228313820E94BC670F900F900F900F9092
:1043B00011C60E94A90A2091DB03222309F40AC630
:1043C00000D000D0EDB7FEB731968AEE93E0E2CF91
:1043D00088E493E00E94E6672091DB03222309F43E
:1043E000F9C500D000D0EDB7FEB7319687EE93E067
:1043F000D1CF6091E0037091E10380E090E00E94F2
:104400001B678C0169E673E00E943067009731F406
:104410008091F6039091F703846085C0C8016CE633
:1044200073E00E9430679C018091F6039091F7033E
:10443000232B11F48B7F77C082FD03C02CE633E081
:1044400002C029E633E000D000D08CEE94E0D3C166
:104450000C940000BFC500D083EE93E0ADB7BEB7AB
:1044600012969C938E9311970E94BC672091DB0358
:104470000F900F902223A9F000D000D0EDB7FEB727
:10448000319680EE93E0ADB7BEB712969C938E93B3
:104490001197228313820E94BC670F900F900F9098
:1044A0000F9088E10FB6F89480936000109260003E
:1044B0000FBE0C94007C8EC56091E0037091E10307
:1044C00080E090E00E941B677C0169E673E00E9437
:1044D0003067009749F40E944A3C8091F60390911E
:1044E000F70381608D7F1FC0C7016CE673E00E94F7
:1044F0003067009741F40E944A3D8091F603909105
:10450000F7038C7F10C001E813E0C701B8010E94D7
:104510003067009789F40E944A3D8091F60390919C
:10452000F7038E7F82609093F7038093F60386EF04
:1045300093E062E170E0FDC18091F60381FF0BC062
:1045400000D000D084EF94E0EDB7FEB79283818372
:104550001483038327CF80FD03C02CE633E002C021
:1045600029E633E000D000D080EF94E0ADB7BEB7CD
:1045700012969C938E93119714963C932E931397B7
:1045800011CF00D081EC93E0EDB7FEB79283818329
:104590000E94BC672DB73EB72C5030400FB6F89440
:1045A0003EBF0FBE2DBFEDB7FEB731968AEA93E04E
:1045B000ADB7BEB712969C938E9311978091711AE6
:1045C0009091721AA091731AB091741A8283938396
:1045D000A483B5838091751A9091761AA091771A69
:1045E000B091781A86839783A087B1878091791AD2
:1045F00090917A1AA0917B1AB0917C1A8287938746
:10460000A487B5870E94BC672091DB03EDB7FEB796
:104610003E960FB6F894FEBF0FBEEDBF222309F4FD
:10462000D9C400D000D0EDB7FEB7319687EA93E049
:10463000B1CEF89429E081E090E0FC01209357008E
:10464000C895E02C80E090E0FC0120935700C895CD
:10465000F02C7894F89483E090E0FC0120935700CC
:10466000C895002D82E090E0FC0120935700C8958A
:10467000102D789400D000D000D08DE993E0EDB7F4
:10468000FEB7928381838091451290914612A0914A
:104690004712B091481283839483A583B6830E9406
:1046A000BC6700D000D0EDB7FEB7319686E793E047
:1046B000ADB7BEB712969C938E9311971283138257
:1046C00004831582F6821782E08611860E94BC67F9
:1046D000EDB7FEB73A960FB6F894FEBF0FBEEDBF2A
:1046E0000E94850A2091660000D000D0EDB7FEB789
:1046F00031968AE693E0ADB7BEB712969C938E933F
:104700001197228313820E94BC670F900F908BE455
:1047100099E0EDB7FEB7928381830E94BC67209138
:10472000DB030F900F90222309F454C400D000D073
:10473000EDB7FEB7319687E693E02CCE80E090E0AF
:104740000E940B1881E090E00E940B182091DB037F
:10475000222309F43FC400D000D0EDB7FEB7319654
:1047600084E693E017CE0E94970F00D08BE499E087
:10477000EDB7FEB7928381830E94BC672091DB0373
:104780000F900F90222309F425C400D000D0EDB77C
:10479000FEB7319681E693E0FDCD6091E003709124
:1047A000E10380E090E00E941B678C0169E673E002
:1047B0000E943067009731F48091F6039091F703DF
:1047C0008860B1CEC8016CE673E00E9430679C013E
:1047D0008091F6039091F703232B11F4877FA3CEEA
:1047E00083FD03C02CE633E002C029E633E000D0AD
:1047F00000D088EF94E0EDB7FEB7928381833483D5
:104800002383D0CD6091E0037091E10380E090E0DC
:104810000E941B6766E873E00E943067009729F4E6
:104820001092E2051092E10547C081EE95E00E94EA
:10483000132C7C010CE813E03CC02DB73EB72C5084
:1048400030400FB6F8943EBF0FBE2DBFEDB7FEB798
:104850003196ADB7BEB712961C930E931197D70140
:1048600012968C9112978283138213968C911397D0
:104870008483158218968C911897868317821496D4
:104880008D919C9115979187808716968D919C911B
:104890001797938782870E94AA67EDB7FEB73C9669
:1048A0000FB6F894FEBF0FBEEDBFC7010E94302DBA
:1048B0007C01E114F10409F62091DB03222309F4C1
:1048C00089C300D000D0EDB7FEB731968EE593E0F6
:1048D00061CD0E94080F7EC36091E0037091E103F7
:1048E00080E090E00E941B67009741F160E070E07B
:1048F00040E150E00E94F8647093F3036093F20388
:1049000000D000D0EDB7FEB731962DE433E0ADB75F
:10491000BEB712963C932E931197738362830E94C5
:10492000BC670F900F900F900F9082EF93E06EE0B6
:1049300070E042E050E00E940C694CC300D000D00F
:104940008AE393E0EDB7FEB7928381838091F2030F
:104950009091F303948383830E94BC670F900F9020
:104960008BE499E0ADB7BEB712969C938E931197E6
:104970000E94BC6700D08DE293E0EDB7FEB7928352
:10498000818381E090E0948383830E94BC6781E20D
:1049900093E0ADB7BEB712969C938E93119782E0C9
:1049A00090E014969C938E9313970E94BC6782E1CB
:1049B00093E0EDB7FEB79283818384E090E0948327
:1049C00083830E94BC6783E093E0ADB7BEB71296C5
:1049D0009C938E93119788E090E014969C938E930D
:1049E00013970E94BC6786EF92E0EDB7FEB7928303
:1049F000818380E190E0948383830E94BC6787EE8B
:104A000092E0ADB7BEB712969C938E93119780E259
:104A100090E014969C938E9313970E94BC678AED46
:104A200092E0EDB7FEB79283818380E490E09483B7
:104A300083830E94BC678AEC92E0ADB7BEB7129642
:104A40009C938E93119780E890E014969C938E939C
:104A500013970E94BC678DEB92E0EDB7FEB792838F
:104A6000818380E091E0948383830E94BC678EEA17
:104A700092E0ADB7BEB712969C938E93119780E0EB
:104A800092E014969C938E9313970E94BC6781EAE0
:104A900092E0EDB7FEB79283818380E094E0948347
:104AA00083830E94BC6784E992E0ADB7BEB71296DB
:104AB0009C938E93119780E098E014969C938E932C
:104AC00013970E94BC6787E892E0EDB7FEB7928328
:104AD000818380E090E1948383830E94BC6720916E
:104AE000DB030F900F900F900F90222309F472C2F6
:104AF00000D000D0EDB7FEB7319684E892E04ACC02
:104B00006091E0037091E10380E090E00E941B67F8
:104B1000009741F160E070E04AE050E00E94F864E4
:104B20007093F5036093F40300D000D0EDB7FEB7A7
:104B3000319627E632E0ADB7BEB712963C932E937E
:104B40001197738362830E94BC670F900F900F9040
:104B50000F9084EF93E060E170E042E050E00E944B
:104B60000C6914C000D000D086E492E0EDB7FEB727
:104B7000928381838091F4039091F50394838383DE
:104B80000E94BC670F900F900F900F902091DB0355
:104B9000222309F41FC200D000D0EDB7FEB7319632
:104BA00083E492E0F7CB0E94AC2E2091DB0322231A
:104BB00009F410C200D000D0EDB7FEB7319680E402
:104BC00092E0E8CB00D08DE292E0EDB7FEB79283A1
:104BD00081830E94BC670F900F9080E00E94C50EF9
:104BE0000E94A90A00D000D085E192E0ADB7BEB71F
:104BF00012969C938E93119780E490E014969C9368
:104C00008E9313970E94BC6700D0EDB7FEB7319624
:104C100082E092E0ADB7BEB712969C938E93119747
:104C200080911B1F8283138280911C1F84831582B5
:104C30000E94BC670F900F9087EE91E0EDB7FEB732
:104C4000928381838091F4039091F503948383830D
:104C50000E94BC678EEC91E0ADB7BEB712969C93F4
:104C60008E9311978091F2039091F30314969C9385
:104C70008E9313970E94BC670F900F900F900F9028
:104C80000E94DA0700D000D000D021EC31E0EDB76F
:104C9000FEB732832183ADB7BEB713966D937D9374
:104CA0008D939C9316970E94BC67EDB7FEB736961E
:104CB0000FB6F894FEBF0FBEEDBF0E9412080E940F
:104CC000EE0700D000D000D023EB31E0ADB7BEB787
:104CD00012963C932E931197EDB7FEB763837483BE
:104CE000858396830E94BC672DB73EB72A5F3F4FEE
:104CF0000FB6F8943EBF0FBE2DBF1D9903C02CE622
:104D000033E002C023EB33E000D000D087EA91E02B
:104D1000ADB7BEB712969C938E93119714963C93A1
:104D20002E9313970E94BC672091BE1A3091BF1A30
:104D30004091C01A5091C11AE090C21AF090C31A63
:104D40000091C41A1091C51A00D000D000D0EDB760
:104D5000FEB731968AE891E0ADB7BEB712969C9344
:104D60008E9311972283338344835583E682F7829F
:104D7000008711870E94BC67EDB7FEB738960FB663
:104D8000F894FEBF0FBEEDBF8DE791E09283818363
:104D90000E94BC678091F6030F900F9081FF0EC0B8
:104DA00000D087E791E0ADB7BEB712969C938E9383
:104DB00011970E94BC670F900F9017C080FD03C031
:104DC0002CE633E002C029E633E000D000D083E7D0
:104DD00091E0EDB7FEB792838183348323830E94F1
:104DE000BC670F900F900F900F908091F60383FD9A
:104DF00003C02CE633E002C029E633E000D000D047
:104E000080E691E0ADB7BEB712969C938E93119752
:104E100014963C932E9313970E94BC672091D4055F
:104E20003091D50583E591E0EDB7FEB7928381839C
:104E3000348323830E94BC670F900F900F900F90D4
:104E4000779B03C02CE633E002C029E633E000D0B4
:104E500000D087E491E0ADB7BEB712969C938E93D5
:104E6000119714963C932E9313970E94BC67209140
:104E7000DB030F900F900F900F90222309F4AAC02C
:104E800000D000D0EDB7FEB7319684E491E082CA3D
:104E90000E94230C2091DB03222309F49BC000D045
:104EA00000D0EDB7FEB7319681E491E073CA0E945D
:104EB000001000D000D000D086E391E0EDB7FEB73F
:104EC000928381838091691290916A12A0916B12F2
:104ED000B0916C1283839483A583B6830E94BC67D0
:104EE00089E291E0ADB7BEB712969C938E9311976D
:104EF0008091171F9091181FA091191FB0911A1F30
:104F0000EDB7FEB783839483A583B6830E94BC6705
:104F10000F900F900F900F908BE499E0ADB7BEB754
:104F200012969C938E9311970E94BC672091DB038D
:104F30000F900F90222309F44DC000D000D0EDB7A0
:104F4000FEB7319686E291E025CA6091E003709148
:104F5000E10380E090E00E941B6766EB73E00E9433
:104F600030670097A9F46091E0037091E10380E05D
:104F700090E00E941B67009769F10E941266982FCB
:104F8000803140F580915201892B8093520122C0DB
:104F90008091520100D000D02CEF34E0EDB7FEB785
:104FA0003283218390E08F709070948383830E947A
:104FB000BC670F900F908BE499E0ADB7BEB7129627
:104FC0009C938E9311970E94BC670F900F9002C024
:104FD0000E94F00BEC81FD811182108283E0289603
:104FE0000FB6F894DEBF0FBECDBFCF91DF911F91FA
:104FF0000F91FF90EF90DF90CF90BF90AF909F9078
:105000008F907F906F905F904F903F902F9008957A
:10501000CF93DF93EC0188819981009729F0845325
:10502000974009F082C076C00E94B6178091F603BF
:1050300080FD02C00E944A3D809170008C7F809369
:1050400070008091B60080628093B6001092B2002A
:1050500082E08093B1008091B60090E087709070FC
:10506000892BC9F780917000816080937000EAEC11
:10507000FEE11182108236968FE1E630F807C9F71B
:105080000E94C10980E090E06DEE78E00E94703AE5
:1050900088E493E00E94E66780E00E94C50E0E94CB
:1050A0009E3B8093F1050E941C3B8093F20500D04B
:1050B00000D000D0EDB7FEB731962BEB33E0ADB7A3
:1050C000BEB712963C932E931197828313828091E0
:1050D000F105848315820E94AA6710920906109236
:1050E00008068DB79EB706960FB6F8949EBF0FBE02
:1050F0008DBF84E094E09093151F8093141F83E28A
:1051000090E09093FA058093F90584E397E0998302
:10511000888302C0633211F081E00AC088E096E023
:1051200060E070E00E945C19E4CF1982188283E08D
:10513000DF91CF910895DC01FB0180818C93818107
:1051400011968C930895FC01DB0190818C91981746
:1051500019F020E030E009C020E0918111968C9197
:10516000981321E081E0282730E0C9010895FC016F
:10517000808180931B1F818180931C1F0895DC0117
:105180001996ED91FC911A970280F381E02D3097EA
:1051900009F0099508950F931F938C0188E16BE145
:1051A0007FE10E941831C8010E9435291F910F919B
:1051B00008950E9438290895CF92DF92EF92FF92CE
:1051C0000F931F938C017B016A014CE854E00E940D
:1051D0003B29F801D286C186C70160E974E00E94CC
:1051E0007B291F910F91FF90EF90DF90CF90089552
:1051F000EF92FF920F931F93DF93CF9300D0CDB721
:10520000DEB78C0188E10E941031BC017E01089458
:10521000E11CF11CC7010E949B28D8011996ED9151
:10522000FC911A970190F081E02DC801B701099512
:105230000F900F90CF91DF911F910F91FF90EF9002
:105240000895FC01A781B0852D913C91F901099544
:105250000895DC011796ED91FC9118970280F38177
:10526000E02D309709F0099508950E94894308952B
:105270000E946C290895CF92DF92EF92FF920F93D4
:105280001F938C017B016A010E947229F801D0866C
:10529000C782C70164E974E00E947B291F910F91C6
:1052A000FF90EF90DF90CF900895CF93DF93EC01C4
:1052B0008AE899E00E94132C08C0828193818C17A0
:1052C0009D0731F0CF010E94302DFC010097A9F716
:1052D000CF01DF91CF910895BC018AE899E00E9447
:1052E000C72C0895FC01738362838AE899E0BF01AB
:1052F0000E942E2C08950F931F93CF93DF938B0161
:105300000E945529EC01009731F01D830C83C801E0
:105310000E94E5458E83DF91CF911F910F910895F3
:105320008AE899E00E940F2C0895809198098F5F78
:1053300080939809815008951F93CF93DF93EC01D8
:10534000162F888580FF1EC08C819D81892BD1F00E
:10535000D0938F09C0938E0982E08887EC81FD810C
:10536000CE0106960995992787FD90950297029799
:1053700010F0133829F4CE01BE010E94C62902C0E4
:1053800081E08887DF91CF911F910895CF92DF92BE
:10539000EF92FF920F931F93CF93DF93EC017B016A
:1053A000C0908E09D0908F09E0918C09F0918D0901
:1053B00003C00190F081E02DEC17FD0719F0309744
:1053C000C1F74CC0209709F449C08885882339F17A
:1053D000188600918C0910918D090BC0C017D10758
:1053E00029F0C80167E8AE010E949C29F8010081FC
:1053F00011810115110591F78C819D81892B79F01F
:10540000CE15DF0561F0D0938F09C0938E09EC8132
:10541000FD81CE01069663E840E050E00995E091F9
:105420008C09F0918D09CE17DF0791F4888199815D
:1054300090938D0980938C090DC0808191818C1788
:105440009D0729F4888199819183808303C0FC01A1
:10545000309799F7D0928F09C0928E09DF91CF9142
:105460001F910F91FF90EF90DF90CF900895609182
:105470008E0970918F090E94C62908958AE8809349
:1054800098091092BE1F10921D1F10928D09109244
:105490008C0910928F0910928E0908951F93CF9353
:1054A000DF93809199098823C1F010929909C091E6
:1054B0008C09D0918D0911E00EC08985882341F0B7
:1054C00018871986CE0162E840E050E00E949C29CE
:1054D0000990D881C02D209781F720911D1F22238C
:1054E00009F470C08091BE1F90E0FC01EE0FFF1F19
:1054F000EE0FFF1FE80FF91FE25EF04E6081609330
:1055000097094181528150939609409395090380F0
:10551000F481E02DF0939409E093930901968F7143
:1055200090708093BE1F215020931D1F309709F06B
:1055300042C080918C0990918D099093920980933B
:10554000910911E031C0809199098823B9F0109236
:105550009909C0918C09D0918D090EC08985882345
:1055600041F018871986CE0162E840E050E00E94C1
:105570009C290990D881C02D209781F740919509E9
:1055800050919609809191099091920960919709A3
:105590000E949C29E0919109F0919209808191816A
:1055A0009093920980939109809191099091920929
:1055B000892B49F607C0613811F481E08087CF015B
:1055C0000E949C298091990920911D1F30E0280F8D
:1055D000311DC901DF91CF911F91089580919909E3
:1055E00020911D1F30E0280F311DC9010895DC01F5
:1055F00020911D1F203219F421E030E01AC0809163
:10560000BE1F820F8F718093900990E0FC01EE0F16
:10561000FF1FEE0FFF1FE80FF91FE25EF04E6083E1
:1056200052834183B483A3832F5F20931D1F20E007
:1056300030E0C90108950F931F9300918E091091D6
:105640008F090E949C2910938F0900938E091F9146
:105650000F910895CF93DF93DC01EB0160918C09EA
:1056600040918D09862F942F9C01F90103C0019070
:10567000F081E02DEA17FB07B9F03097C1F76C9382
:1056800011964C931197B0938D09A0938C0981E0EA
:1056900018968C93189717961C921E921697CD0108
:1056A00061E8AE010E941B2BDF91CF910895FC01B0
:1056B000009741F080858150823020F481E081871D
:1056C00080939909089520E030E0FC0180858823CB
:1056D00011F021E030E0C9010895DC0112964D91EE
:1056E0005C91139720E030E01FC01496ED91FC917F
:1056F0001597E20FF31F80818823A1F481E0808356
:105700008D919C911197AC01249FC001259F900D14
:10571000349F900D112416962D913C911797280FC8
:10572000391F07C02F5F3F4F24173507F0F220E0E5
:1057300030E0C9010895DC0116962D913C91179730
:105740001296ED91FC91139740E050E01DC0261792
:10575000370799F41496ED91FC911597E40FF51F16
:105760008081181614F4815080831496ED91FC9179
:105770001597E40FF51F808108958D919C911197E5
:10578000280F391F4F5F5F4F4E175F0700F38FEFF2
:105790000895FC01AB01668177814617570718F41D
:1057A00020E030E017C0A0E0808191812281338128
:1057B000FC01E29FC001E39F900DF29F900D112428
:1057C000680F791F4617570708F0A1E081E0A82766
:1057D0002A2F30E0C90108950F931F938C01FC011B
:1057E000428153818481958160E070E00E94296745
:1057F000F8012281338180819181A901489F900124
:10580000499F300D589F300D11248681978160E0AB
:1058100070E0A9010E9429671F910F910895FC0172
:10582000118210820895FC01808191810895FC010C
:10583000DB018D919C91918380830895FC010190FF
:10584000F081E02D309731F080819181009721F037
:10585000FC01FACFE0E0F0E0CF010895CF93DF93B1
:10586000EC01AB012881398121153105D1F0F90115
:10587000A0E0B0E014C0E417F50761F480819181E5
:10588000109719F49983888302C08D939C93118299
:10589000108207C0DF01808191819C01F90130975E
:1058A00051F7FA011182108288819981009739F0AD
:1058B000FC01808191810097D9F7309719F45983C1
:1058C000488302C051834083DF91CF910895CF93E5
:1058D000DF93EC01AB012881398121153105D1F02D
:1058E000F901A0E0B0E014C0E417F50761F480818D
:1058F0009181109719F49983888302C08D939C93AA
:105900001182108207C0DF01808191819C01F90121
:10591000309751F788819981FA0191838083598367
:105920004883DF91CF910895CF93DF93EC01E88115
:10593000F981309719F420E030E019C0DF0180814F
:105940009181892B21F4198218829F0110C02C911A
:1059500011963C911197AD01C901DC018D919C918B
:105960001197892BA1F7FA01118210829D01C901BB
:10597000DF91CF910895DC01ED91FC911197309763
:1059800021F0808191818D939C93CF010895CF93D5
:10599000DF93EC012881398121153105D1F0F9011E
:1059A000A0E0B0E014C0E617F70761F480819181B0
:1059B000109719F49983888302C08D939C93118268
:1059C000108207C0DF01808191819C01F90130972D
:1059D00051F7DF91CF910895FC010190F081E02D06
:1059E00020E030E005C02F5F3F4F0190F081E02DB7
:1059F0003097C9F7C90108950F931F93CF93DF9391
:105A00008C01FB01EA0161157105F9F4DC012D91AE
:105A10003C9121153105C1F0F901A0E0B0E012C0C0
:105A2000EC17FD0751F480819181109709F4D8019A
:105A30008D939C931182108207C0DF018081918138
:105A40009C01F901309761F7F80180819181998378
:105A50008883D183C083DF91CF911F910F910895E7
:105A6000FC01009719F420E030E002C02081318170
:105A7000C901089520E030E0FC0186819781892BDF
:105A800011F421E030E0C9010895FC012281338145
:105A900080819181280F391FC9010895FC018081FF
:105AA0009181089520919A0930919B092115310522
:105AB00011F021E030E0C901089580919A09909198
:105AC0009B09892B19F420E030E004C020919C0947
:105AD00030919D09C901089580919A0990919B097F
:105AE000892B29F410929D0910929C0908950E9417
:105AF000A538BC01E0919A09F0919B09428153813C
:105B000080819181480F591F461B570B0CC0228181
:105B1000338180819181280F391F261B370B241771
:105B2000350708F4A9010480F581E02D309779F755
:105B3000460F571F50939D0940939C090895CF939A
:105B4000DF93EC01E0919A09F0919B098E179F0772
:105B500041F48C819D8190939B0980939A0914C094
:105B6000FC01309731F0848195818C179D07C1F736
:105B700007C01D821C821F821E82DF91CF91089573
:105B80008C819D81958384830E946C2DF2CFFC01D2
:105B900080819181860F971F918380830E946C2D55
:105BA000089582EA94E00E94572B0895EF92FF92A5
:105BB0000F931F93CF93DF937C01FC018081918130
:105BC000009729F08A35910509F06DC00BC010923D
:105BD0009B0910929A098AE590E0F70191838083EE
:105BE00081E065C0673849F59A01E0919A09F09122
:105BF0009B0903C00480F581E02D309741F3868135
:105C0000978182179307B1F3E0939A09F0939B0968
:105C10000FC016968D919C9117978217930711F0DC
:105C2000FD0106C014968D919C91159795838483F0
:105C3000A481B581109769F7CECF623861F6C09123
:105C40009A09D0919B0900E010E02AC0CE010E9481
:105C5000624A892B01F18E819F8168E8AE010E9422
:105C6000F72A892BA1F41F821E828C819D81011548
:105C7000110521F0F8019583848304C090939B095A
:105C800080939A091D821C820E946C2DD8CF82EAD3
:105C900094E00E94572B8E018C819D819C01E9012B
:105CA0002097A1F698CFF7011182108283E0DF914F
:105CB000CF911F910F91FF90EF900895CF93DF93B5
:105CC000EC0182EA94E00E94572B8E819F81892B00
:105CD00069F0E0919A09F0919B0906C0EC17FD0765
:105CE000A9F00480F581E02D3097C1F780918E09ED
:105CF00090918F099F838E8380919A0990919B093F
:105D00009D838C83D0939B09C0939A090E946C2D2C
:105D1000DF91CF9108950F931F938C010E947A4ACF
:105D2000C8010E945E2E1F910F9108950F931F933B
:105D30008C010E94434AC8010E945E2E1F910F9160
:105D400008950F931F938C010E94854AC8010E94F9
:105D50005E2E1F910F9108950F931F9310911B1F9B
:105D600000911C1F0E94DB382DB73EB722553040F2
:105D70000FB6F8943EBF0FBE2DBFEDB7FEB73196FC
:105D80002CEB39E0ADB7BEB712963C932E9311972A
:105D900012831382048315826683778380879187B9
:105DA0008091B0219091B121A091B221B091B32105
:105DB00082879387A487B5878091B4219091B5217C
:105DC000A091B621B091B72186879787A08BB18B20
:105DD0008091B8219091B921A091BA21B091BB21B5
:105DE000828B938BA48BB58B8091BC219091BD212C
:105DF000A091BE21B091BF21868B978BA08FB18FD0
:105E00008091C0219091C121A091C221B091C32164
:105E1000828F938FA48FB58F8091C4219091C521DB
:105E2000A091C621B091C721868F978FA0A3B1A35F
:105E30008091C8219091C921A091CA21B091CB2114
:105E400082A393A3A4A3B5A38091CC219091CD214B
:105E5000A091CE21B091CF2186A397A3A0A7B1A7EF
:105E60008091D0219091D121A091D221B091D321C4
:105E700082A793A7A4A7B5A78091D4219091D521FB
:105E8000A091D621B091D72186A797A7A0ABB1AB9F
:105E90008091D8219091D921A091DA21B091DB2174
:105EA00082AB93ABA4ABB5AB8091DC219091DD21AB
:105EB000A091DE21B091DF2186AB97ABA0AFB1AF4F
:105EC0008091E0219091E121A091E221B091E32124
:105ED00082AF93AFA4AFB5AFEDB7FEB7FF96809199
:105EE000E4219091E521A091E621B091E721808302
:105EF0009183A283B383EDB7FEB7ED5BFF4F809133
:105F0000E8219091E921A091EA21B091EB218083D1
:105F10009183A283B383EDB7FEB7E95BFF4F809116
:105F2000EC219091ED21A091EE21B091EF218083A1
:105F30009183A283B383EDB7FEB7E55BFF4F8091FA
:105F4000F0219091F121A091F221B091F321808371
:105F50009183A283B383EDB7FEB7E15BFF4F8091DE
:105F6000F4219091F521A091F621B091F721808341
:105F70009183A283B3830E94BC6710911B1F009181
:105F80001C1F2DB73EB72E5A3F4F0FB6F8943EBF99
:105F90000FBE2DBF0E94DB38ADB7BEB7D2970FB68C
:105FA000F894BEBF0FBEADBFEDB7FEB731962DE47E
:105FB00039E012963C932E93119712831382048337
:105FC000158266837783808791878091F8219091ED
:105FD000F921A091FA21B091FB2182879387A487B0
:105FE000B5878091FC219091FD21A091FE21B09177
:105FF000FF2186879787A08BB18B8091002290919B
:106000000122A0910222B0910322828B938BA48B58
:10601000B58B8091042290910522A0910622B09127
:106020000722868B978BA08FB18F80910822909149
:106030000922A0910A22B0910B22828F938FA48F04
:10604000B58F80910C2290910D22A0910E22B091DB
:106050000F22868F978FA0A3B1A3809110229091D9
:106060001122A0911222B091132282A393A3A4A380
:10607000B5A38091142290911522A0911622B0917F
:10608000172286A397A3A0A7B1A780912022909161
:106090002122A0912222B091232282A793A7A4A714
:1060A000B5A78091242290912522A0912622B0911B
:1060B000272286A797A7A0ABB1AB0E94BC672DB7DC
:1060C0003EB72E5C3F4F0FB6F8943EBF0FBE2DBFBC
:1060D0001F910F91089580E38093A2090895AC0168
:1060E0003091A209832F90E0841795079CF020E35C
:1060F000231B80919E0990919F09820F911D840F0F
:10610000951F8138910530F4341B3093A20921E0AA
:1061100030E002C020E030E0C90108959091A2096A
:10612000980F9093A209089540919E0950919F095C
:106130009C014817590718F420E030E012C0809104
:10614000A0099091A109820F931F9093A1098093B8
:10615000A009421B530B50939F0940939E0921E0D5
:1061600030E0C901089590939F0980939E09089596
:106170008091A0099091A109C0962091AC04309122
:10618000AD04280F391FC90108958091A2092091FB
:10619000AC043091AD04280F311DC901089540E0D1
:1061A00050E08091AC049091AD04C0962091A30979
:1061B0003091A4092817390711F041E050E0CA01D5
:1061C00008958091A3099091A409089580919E0952
:1061D00090919F0908959091A20980E3891B0895E9
:1061E00080E39091A209891B20919E0930919F091B
:1061F000280F311DC9010895E82FF0E0EE0FFF1FB1
:10620000E953F04E7183608381E090E00895E82FB8
:10621000F0E0EE0FFF1FE953F04E80819181089569
:10622000282F30E0220F331F2157304EC901089527
:1062300090E0880F991F8157904E0E949B2881E023
:1062400090E00895E7ECFFE1119211928FE1E73FB2
:10625000F807D1F78FEB9FE16AE874E00E949B2872
:1062600081EC9FE16AE874E00E949B2883EC9FE147
:106270006AE874E00E949B2885EC9FE16AE874E07C
:106280000E949B2808951092A1091092A0091092D3
:106290009F0910929E0980E38093A2098091AC042B
:1062A0009091AD04C0969093A4098093A3090E9495
:1062B00022310895EF92FF920F931F938C017B017F
:1062C0000E9443311093A4090093A309F0929F09FF
:1062D000E0929E091F910F91FF90EF900895A7EC17
:1062E000BFE1FC0180E301900D928150E1F7AFEB3B
:1062F000BFE1FB0188E001900D928150E1F7089524
:10630000DC01E7ECFFE180E301900D928150E1F7C1
:10631000DB01EFEBFFE188E001900D928150E1F7A6
:1063200008950F931F93CF93DF93EC018091A209FF
:10633000482F50E080919E0990919F09C096841B40
:10634000950B8138910518F020E030E032C000E371
:1063500010E0F801E41BF50B2091AC043091AD0482
:10636000240F351FCE01B901AF010E942067809133
:10637000A209081B11090C0F1D1F2091A3093091C0
:10638000A4098091A0099091A109280F391F40917B
:106390009E0950919F09C801B9010E942067209170
:1063A0009E0930919F09205D3F4F8091A209281BD3
:1063B0003109C901DF91CF911F910F9108950F937A
:1063C0001F934091A20950E000E310E0F801E41BA4
:1063D000F50B2091AC043091AD04240F351FB901A9
:1063E000AF010E9420678091A209081B1109C80112
:1063F0001F910F910895E091A309F091A409609174
:10640000AC047091AD049B01205D3F4FE217F30790
:1064100049F040919E0950919F09C901BF010E9416
:10642000206708958091A0099091A1090097D9F063
:1064300040919E0950919F09405D5F4FDC01D096CD
:10644000A60FB71F20E330E007C0FB01E20FF31FE8
:106450008D9180832F5F3F4F24173507B4F310923F
:10646000A1091092A0090895EF92FF920F931F9334
:10647000F82EE92E162F072F0E944331212F302F9F
:10648000C9018C018138910510F000E810E080917D
:10649000A3099091A4096F2D7E2DA8010E94206769
:1064A00010939F0900939E09C8011F910F91FF90BF
:1064B000EF900895E091FA1FF091FB1F8081909179
:1064C000F91F89230895E091F71FF091F81F80814B
:1064D0009091F91F892B8083E091FC1FF091FD1FA3
:1064E00080819091F91F892B80830895E091F71F97
:1064F000F091F81F90818091F91F80958923808306
:10650000E091FC1FF091FD1F90818091F91F809513
:10651000892380830895E091F71FF091F81F9081FF
:106520008091F91F809589238083E091FC1FF09171
:10653000FD1F80819091F91F892B80838FEB93E061
:106540008115910511F00197F1F72FB7F894E091BB
:10655000FC1FF091FD1F90818091F91F8095892388
:10656000808383E890E08115910511F00197F1F7A0
:10657000E091FA1FF091FB1F40813091F91F2FBF6E
:1065800078948BE393E08115910511F00197F1F771
:106590008081832311F481E00895842F832308955B
:1065A0005093FD1F4093FC1F7093F81F6093F71FDB
:1065B0009093FB1F8093FA1F81E090E002C0880F48
:1065C000991F2A95E2F78093F91F0E948B32089554
:1065D000382F4FB7F894E091FC1FF091FD1F808198
:1065E0009091F91F892B808383E090E081159105BC
:1065F00011F00197F1F7332351F0E091FC1FF09176
:10660000FD1F90818091F91F80958923808387E108
:1066100090E08115910511F00197F1F7E091FA1FD3
:10662000F091FB1F80812091F91F822309F430E053
:1066300089E590E08115910511F00197F1F7E0915E
:10664000FC1FF091FD1F80812095282320834FBFE0
:106650008BE390E08115910511F00197F1F7832FFD
:1066600008950F931F93182F08E0812F81700E94C7
:10667000E8321695811110680150B9F7812F1F91EA
:106680000F9108958FEF0E9431330895DF92EF92BA
:10669000FF920F931F93CF93DF93E82EEB010E949D
:1066A0008B328823A1F580EF0E94313380E4FF24F0
:1066B000182F98EFD92ED80E81E00E94E832082FCB
:1066C00081E00E94E832882329F0002371F08EEFE8
:1066D000F82E1FC0002349F41E1528F0888180FF82
:1066E00004C0E11611F0F12E01E0802F0E94E83283
:1066F000888186958883002311F0806888831150F3
:106700001D15D1F6112329F02196812FD1CFFF2419
:10671000FA948F2DDF91CF911F910F91FF90EF9001
:10672000DF9008950F931F93CF93DF93082FEB0112
:106730000E948B32209751F085E50E94313318E09A
:1067400089910E9431331150D9F703C08CEC0E941B
:106750003133802F0E943133DF91CF911F910F9100
:106760000895FF920F931F93CF93DF93F82EFB01B1
:10677000DA01E9018081482F50E0918180E0482BC7
:10678000592B80E1F81671F4CA018E7F33E0880F2F
:10679000991F3A95E1F726814CE050E0421B5109E0
:1067A000480F591F57FF06C081E08C9350954195C3
:1067B0005F4F01C01C9288E2F81691F48481682F23
:1067C00070E0CB01807690708036910549F066FFCD
:1067D00002C04E7F05C065FF02C04C7F01C0487FEC
:1067E000CA0124E0969587952A95E1F78883842F3E
:1067F0008F70F801808380E0DF91CF911F910F911E
:10680000FF900895FF920F931F93DF93CF93CDB71F
:10681000DEB728970FB6F894DEBF0FBECDBFF82EB7
:10682000362FDE011196E6EBF4E028E001900D92A0
:106830002150E1F7042F112707FD109581E792E021
:10684000AC01049FC001059F900D149F900D112471
:1068500064E670E00E942164CB0124E6329FB0011F
:106860001124680F791FFE0131969E01275F3F4F6B
:10687000808190E00817190719F46F5F7F4F04C0FB
:106880003196E217F307A1F7FF2019F07095619593
:106890007F4FCB0128960FB6F894DEBF0FBECDBF59
:1068A000CF91DF911F910F91FF9008957F928F926A
:1068B0009F92AF92BF92CF92DF92EF92FF920F938F
:1068C0001F93DF93CF93CDB7DEB729970FB6F89418
:1068D000DEBF0FBECDBF782E6B015A0149018EEB92
:1068E00060E070E00E9492338E010F5F1F4F4AE01C
:1068F000E42EF12CEC0EFD1E0E944233F801819330
:106900008F01EE15FF05C1F77E010894E11CF11C13
:10691000C70169E070E00E945750882311F083E0BE
:1069200008C0872DB701A601950184010E94B133EB
:1069300080E029960FB6F894DEBF0FBECDBFCF9191
:10694000DF911F910F91FF90EF90DF90CF90BF905C
:10695000AF909F908F907F9008956F927F928F92CB
:106960009F92AF92BF92CF92DF92EF92FF920F93DE
:106970001F93DF93CF93CDB7DEB729970FB6F89467
:10698000DEBF0FBECDBF6C015B014A0139010E9421
:106990008B328EEBB6010E9492338E010F5F1F4F38
:1069A0005AE0E52EF12CEC0EFD1E0E944233F80158
:1069B00081938F01EE15FF05C1F77E010894E11C5C
:1069C000F11CC70169E070E00E945750882311F064
:1069D00083E009C0F6018081B701A501940183011C
:1069E0000E94B13380E029960FB6F894DEBF0FBE47
:1069F000CDBFCF91DF911F910F91FF90EF90DF906E
:106A0000CF90BF90AF909F908F907F906F900895A0
:106A10001F93CF93DF93182FEB010E948B320E94BC
:106A20005A32882311F482E009C084E4BE010E9436
:106A30009233113011F00E94633280E0DF91CF91E8
:106A40001F9108950F931F93DF93CF93CDB7DEB7B8
:106A50002B970FB6F894DEBF0FBECDBF182F092FAE
:106A6000885F612F792F0E940835882309F04CC078
:106A700066E471E48FE090E00E94C135812F902F91
:106A8000BE016F5F7F4FAE014E5F5F4F9E012D5F76
:106A90003F4F0E94AD348823B9F5DE011496EEEA2B
:106AA000F4E088E001900D928150E1F71B81212FE5
:106AB00030E081E792E0AC01249FC001259F900D5A
:106AC000349F900D112464E670E00E9421643A81A5
:106AD00024E6329F90011124260F371FFE013496C1
:106AE000AE01445F5F4F8081181719F42F5F3F4F4D
:106AF00004C03196E417F507B1F78981882331F096
:106B0000309521953F4F02C024E331E2C9012B9615
:106B10000FB6F894DEBF0FBECDBFCF91DF911F91AE
:106B20000F9108950F931F938C010E948B3284EB79
:106B3000B8010E94923381E00E94E832182F0E942F
:106B40008B32111111E0812F1F910F9108950F9336
:106B50001F93CF93DF938C01EB01F8018081BE017D
:106B60000E944633F801808381508D3F28F488814C
:106B7000883211F0803189F7DF91CF911F910F9109
:106B80000895DC01CB0181159105A105B10529F01E
:106B900081509040A040B040D9F70895E6E4F1E07C
:106BA0008081908120813081829586958695837041
:106BB00092959F70892B832B22952F70822B08959D
:106BC00000D000D000D0EDB7FEB7319628E93AE00A
:106BD000ADB7BEB712963C932E93119793838283E1
:106BE000758364830E94BC678DB79EB706960FB607
:106BF000F8949EBF0FBE8DBF0895DF92EF92FF9273
:106C00000F931F93DF93CF9300D0CDB7DEB780E013
:106C10006CE046E00E94E43989E18093C400109260
:106C2000C50082E08093C00080E00E94C43A0E94C8
:106C3000953884B784B784B784B784B7EEE7F8E2B1
:106C400022E432E4318320833A968DB79EB70A97C7
:106C5000E817F907B8F300D000D089E09BE0ADB7A2
:106C6000BEB712969C938E9311978EEB94E0149678
:106C70009C938E9313970E94BC670F900F900F9078
:106C80000F900E94AF4C0E943E2A82EA94E060E09E
:106C900070E00E942A2B0E94C14BE0910905F091FF
:106CA0000A0509958091460190914601209146017F
:106CB00030914601829586958695837092959F7056
:106CC000892B832B22952F70822B90E00E94B54C4C
:106CD000CE0101960E94A037882359F000D089EE9A
:106CE0009AE0EDB7FEB7928381830E94BC670F9054
:106CF0000F907E010894E11CF11CC7010E94B72887
:106D00000E949B378C010E949637BC01C801A701E5
:106D10000E941F3B0E94AA370E94513F0E94913758
:106D20000E943D3F00D08CED9AE0ADB7BEB7129601
:106D30009C938E9311970E94BC6700D0EDB7FEB76D
:106D4000319608ED1AE0ADB7BEB712961C930E93BC
:106D500011978A81828313820E94BC67EDB7FEB7C8
:106D60003196ADB7BEB712961C930E9311978981D9
:106D7000828313820E94BC670F900F9086ED9AE089
:106D8000EDB7FEB7928381830E94BC670F900F908E
:106D90000E94854DE0917B05F0917C050995E0917D
:106DA0006205F09163050995E0912405F0912505B0
:106DB00009950091600510916105E0907905F090CA
:106DC0007A050E941C3BD82E0E949E3B2DB73EB7F1
:106DD0002A5030400FB6F8943EBF0FBE2DBFEDB71E
:106DE000FEB731962BEB3AE0ADB7BEB712963C93A7
:106DF0002E93119713830283F582E482D682178241
:106E0000808711860E94BC67E0918505F091860518
:106E10002DB73EB7265F3F4F0FB6F8943EBF0FBE6B
:106E20002DBF3097F1F00995BC0180E890E00E94F9
:106E30000D648FEF6F3F7807A1F000D000D088EA93
:106E40009AE0ADB7BEB712969C938E9311971496A5
:106E50007C936E9313970E94BC670F900F900F90D6
:106E60000F9000D086EA9AE0EDB7FEB79283818357
:106E70000E94BC670F900F908DEB95E060E070E092
:106E80000E942A2B80E794E00E94344A00D08EE9C9
:106E90009AE0ADB7BEB712969C938E9311970E945D
:106EA000BC670F900F900F900F90CF91DF911F91C3
:106EB0000F91FF90EF90DF900895EF92FF920F9364
:106EC0001F9380E880936100109261000E94FD355D
:106ED0000E944E2A0E94003B8091FE1F9091FF1F4E
:106EE000009729F001979093FF1F8093FE1FE09079
:106EF0000020F090012000910220109103200E94B8
:106F0000DB38E616F7060807190711F30E94DB388D
:106F100060930020709301208093022090930320BF
:106F2000D7CF85E490E00E94FE68089583E490E066
:106F30000E940669089581E490E00E940669089520
:106F4000F8946DE170E042E050E00E94EE687894C1
:106F500080E008950F931F93DF93CF93CDB7DEB7F3
:106F6000A2970FB6F894DEBF0FBECDBF8FE390E0BF
:106F70000E94066989839A83982F8B50803108F08C
:106F80009A838A818095981709F476C000D084E4AA
:106F90009BE0EDB7FEB7928381830E94BC6780E0DF
:106FA00090E00F900F909E012D5F3F4FFC01EC5D34
:106FB000F44FE491D901A80FB91FEC9301968830E2
:106FC0009105A1F7F8948E010D5F1F4FC8016DE187
:106FD00070E048E050E00E940C6920E030E0C80119
:106FE000F901E45DF44FE491DC01A20FB31FEC93CF
:106FF0002F5F3F4F2E30310599F765E270E04EE08C
:1070000050E00E940C6920E030E0CE010396F901C7
:10701000E65CF44FE491DC01A20FB31FEC932F5F09
:107020003F4F2A30310599F763E370E04AE050E0C2
:107030000E940C6981E490E06DEC7BEA0E94246977
:1070400083E490E060E070E00E94246985E490E0D1
:1070500060E00E9416698DE390E060E070E00E94BD
:1070600024698AE1898385EE8A8369817A818FE345
:1070700090E00E94246978948981A2960FB6F894D2
:10708000DEBF0FBECDBFCF91DF911F910F9108954D
:10709000EF92FF920F931F9320910C2030910D20BF
:1070A00040910E2050910F20E82EFF2400E010E0C8
:1070B0002E0D3F1D401F511F20930C2030930D209B
:1070C00040930E2050930F2080910820909109202A
:1070D000A0910A20B0910B208E0D9F1DA01FB11F03
:1070E0008093082090930920A0930A20B0930B204E
:1070F0008091AC218823A1F08091042090910520FB
:10710000A0910620B0910720E80EF91E0A1F1B1F50
:10711000E0920420F09205200093062010930720AF
:107120001F910F91FF90EF900895F8941092B60080
:1071300016BC83EF87BD92E094BD84E085BD85B326
:1071400085BB90936E00789408952091570A3091F2
:10715000580A8091570A9091580A28173907A9F7B9
:10716000C901089507C022E330E0000021503040FB
:10717000E1F701970097B9F70895BC014091570ACC
:107180005091580A8091570A9091580A4817590708
:10719000A9F72091570A3091580A8091570A909187
:1071A000580A28173907A9F7241B350B2617370764
:1071B00080F30895089520910C2030910D20409186
:1071C0000E2050910F2080910C2090910D20A091C5
:1071D0000E20B0910F20281739074A075B0759F78F
:1071E000B901CA0108951F920F920FB60F920BB604
:1071F0000F9211242F933F934F935F936F937F933D
:107200008F939F93AF93BF93EF93FF938091570A10
:107210009091580A01969093580A8093570A80914A
:10722000590A8F5F8093590A8091590A8038A9F4CE
:107230001092590A80910C2090910D20A0910E205F
:10724000B0910F200196A11DB11D80930C20909349
:107250000D20A0930E20B0930F208091AC218823A5
:10726000F1F080915A0A8F5F80935A0A80915A0AEE
:107270008038A9F410925A0A809104209091052038
:10728000A0910620B09107200196A11DB11D809309
:10729000042090930520A0930620B09307200E941D
:1072A000522D892B11F00E94D12DFF91EF91BF91AA
:1072B000AF919F918F917F916F915F914F913F918E
:1072C0002F910F900BBE0F900FBE0F901F9018952F
:1072D0001F920F920FB60F9211241092E2040F909A
:1072E0000FBE0F901F9018951F920F920FB60F921E
:1072F0000BB60F9211242F933F934F935F936F938D
:107300007F938F939F93AF93BF93EF93FF93E091FE
:10731000D804F091D9048081E091E304F091E40471
:10732000309709F00995FF91EF91BF91AF919F912F
:107330008F917F916F915F914F913F912F910F901E
:107340000BBE0F900FBE0F901F9018951F920F92BB
:107350000FB60F9211241092EF040F900FBE0F90F2
:107360001F9018951F920F920FB60F920BB60F92A7
:1073700011242F933F934F935F936F937F938F933A
:107380009F93AF93BF93EF93FF93E091E504F09148
:10739000E6048081E091F004F091F104309709F067
:1073A0000995FF91EF91BF91AF919F918F917F913F
:1073B0006F915F914F913F912F910F900BBE0F9066
:1073C0000FBE0F901F90189590E02DE030E0829F47
:1073D000F001839FF00D929FF00D1124E852FB4FB6
:1073E000A281B3811C92A481B5816C93A681B781DF
:1073F00088ED8C93A085B1854C93128614861386F4
:107400000895CF93DF93AB0190E02DE030E0829FB1
:10741000D001839FB00D929FB00D1124A852BB4F95
:10742000ED012A9691E00AC09883ED91FC911197A5
:10743000808388818823E9F74F5F5F4FFA01849149
:10744000882391F7DF91CF910895CF93DF93262F73
:10745000372FA90190E02DE030E0829FD001839F7B
:10746000B00D929FB00D1124A852BB4FED012A968A
:1074700091E02DE018C08A3041F49883ED91FC91A1
:107480001197208388818823E9F7FA0180818D3064
:1074900041F09883ED91FC91119780838881882336
:1074A000E9F74F5F5F4FFA018081882321F7DF9171
:1074B000CF91089590E02DE030E0829FF001839F0E
:1074C000F00D929FF00D1124E852FB4F81E082876E
:1074D000A081B1816C933A9680818823E9F7089561
:1074E00090E02DE030E0829FF001839FF00D929FAD
:1074F000F00D1124E852FB4F74876387089591E0E3
:107500009093E204E091D804F091D90480838091B3
:10751000E2048823E1F70895482F8A30C9F4809166
:107520005B0A90E02DE030E0829FF001839FF00D38
:10753000929FF00D1124E852FB4F81E08287A081D9
:10754000B1818DE08C933A9680818823E9F702C05F
:107550008D30B9F080915B0A90E02DE030E0829FA1
:10756000F001839FF00D929FF00D1124E852FB4F24
:1075700081E08287A081B1814C933A9680818823F3
:10758000E9F780E090E0089580935B0A8AEC94E04C
:10759000909379288093782808950F931F93DF9311
:1075A000CF93CDB7DEB7FE013A960CE51AE0C801DD
:1075B00060E470E0488559859F010E9459688F8179
:1075C000B8010E94253ACF91DF911F910F91089544
:1075D00084B7877F84BF88E10FB6F89480936000FA
:1075E000109260000FBE08952FE088E190E00FB682
:1075F000F894A895809360000FBE209360000895D2
:10760000A895089588E10FB6F894809360001092D1
:1076100060000FBE0895F89428E088E190E00FB66E
:10762000F894A895809360000FBE20936000FFCF70
:1076300080939C0A0895089580919D0A0895DA0127
:107640008093620190936301609360017093610184
:107650004115510521F1FA01819180936B01119639
:107660008C9180936A01DF01119681818093690179
:10767000FD01319611968C9180936801DF0111967E
:10768000818180936701FD01319611968C918093E1
:1076900066018181809365018281809364010895F0
:1076A000809117208091172090E0089580913901F2
:1076B00081FF03C020E030E013C081E491E06FE17E
:1076C00040E00E944441282F813019F421E030E04D
:1076D00007C080E090E0213111F481E090E09C014E
:1076E000C90108958091390181FF02C091E016C05F
:1076F00081E491E06FE140E00E944441282F8151F4
:10770000823058F02F3149F0213039F090E02230AA
:1077100009F491E081E0982701C090E0892F089555
:1077200081E491E06FE140E00E944441823021F029
:10773000823111F081E0089580E00895809139014F
:1077400081FF02C080E1089585E491E06FE040E0B0
:107750000E94444108950F931F93182F883059F0C9
:10776000863049F0893039F0863129F0893119F0B5
:1077700022E430E060C08091390181FF03C024E43D
:1077800030E059C00E94723B8823E1F381E491E02C
:107790006FE140E00E944441082F181709F449C0E6
:1077A000183099F480913901809139018D7F80934F
:1077B00039018DE090E00197F1F782E491E06FE10B
:1077C00040E023E00E944E4125C0193141F486314A
:1077D000A9F482E491E06FE140E029E009C01631AC
:1077E00069F4893159F482E491E06FE140E026E0E8
:1077F0000E944E4183E090E00197F1F782E491E02E
:107800006FE140E0212F0E944E41083019F489E6D3
:1078100091E002C083E090E00197F1F781E491E00C
:107820006FE140E00E944441811719F023E430E009
:1078300002C020E430E0C9011F910F9108958091AA
:10784000940090919500909345228093442221E0EA
:10785000209331228091390181FF15C02093AB2103
:1078600080919400909195009093412280934022C2
:1078700020932F22809139018D7F8093390180914F
:10788000AB218823E1F786E10E94AB3B81E0809346
:10789000AC2108958091AC21882351F480919E0AF7
:1078A000882321F081E080939F0A02C00E941F3C40
:1078B00081E090E008950E94723B8823E1F31092EA
:1078C000AC2180913901809139018D7F80933901FC
:1078D0008DE090E00197F1F782E491E06FE140E004
:1078E00023E00E944E4183E090E00197F1F7809100
:1078F000390182608093390180912F228823E9F138
:1079000080919400909195002091402230914122E5
:1079100082179307A0F480910C2290910D22A091E0
:107920000E22B0910F228C57914EAF4FBF4F8093D4
:107930000C2290930D22A0930E22B0930F228091DF
:10794000940090919500821B930BA0E0B0E02091F1
:107950000C2230910D2240910E2250910F22820F65
:10796000931FA41FB51F80930C2290930D22A09308
:107970000E22B0930F2210922F2280913122882361
:10798000E9F18091940090919500209144223091EA
:10799000452282179307A0F480911422909115221A
:1079A000A0911622B09117228C57914EAF4FBF4F26
:1079B0008093142290931522A0931622B09317223D
:1079C0008091940090919500821B930BA0E0B0E011
:1079D00020911422309115224091162250911722A5
:1079E000820F931FA41FB51F80931422909315221A
:1079F000A0931622B09317221092312208958091FD
:107A00009F0A882321F00E941F3C10929F0A8091B8
:107A1000A00A882321F00E945B3C1092A00A1092D9
:107A20009E0A0895CF93DF93FC01AB0181E0809320
:107A30009E0A8091F0219091F121A091F221B091C4
:107A4000F3210196A11DB11D8093F0219093F121A6
:107A5000A093F221B093F321862F8E5F87FF0CC095
:107A60008091A9219091AA2101969093AA218093B7
:107A7000A921CFEFDFEF08C021EA3AE0C901BF0139
:107A80000E942067C0E0D0E00E94FF3CCE01DF9161
:107A9000CF9108958091AC21882381F080919E0A36
:107AA000882321F40E94723B882331F481E0809383
:107AB000A00A21E030E004C00E945B3C20E030E0FE
:107AC000C90108951F93DF93CF930F92CDB7DEB70F
:107AD0008FB7898380919E0A882331F5F89480912D
:107AE000AC21882351F08091390181FD1BC00E9497
:107AF000723B8823B9F090E003C00E944A3C91E0B9
:107B0000809147018E3010F41FEF01C010E09923DF
:107B100011F00E944A3D16FF05C089818FBF21E008
:107B200030E004C089818FBF20E030E0C9010F90B0
:107B3000CF91DF911F9108950F931F938091AC21F6
:107B4000882311F000E003C00E944A3C01E081E478
:107B500091E06FE140E00E944441863111F08131B3
:107B600019F4109147010AC086E491E06FE140E00A
:107B70000E94444193E0899F102D1124002311F0AD
:107B80000E944A3D812F1F910F9108950F931F93DB
:107B9000CF93DF93182F21E020939E0A0091AC2110
:107BA0008091390181FF16C08091940090919500D9
:107BB000909341228093402220932F222093AB2147
:107BC000809139018D7F809339018091AB21882389
:107BD000E1F700E00E94723B8823E1F38091AC2141
:107BE000882309F441C0809131228823E9F18091F2
:107BF0009400909195002091442230914522821763
:107C00009307A0F48091142290911522A09116223E
:107C1000B09117228C57914EAF4FBF4F80931422D3
:107C200090931522A0931622B0931722809194006E
:107C300090919500821B930BA0E0B0E0209114225C
:107C4000309115224091162250911722820F931FD6
:107C5000A41FB51F8093142290931522A09316227F
:107C6000B09317221092312289E10E94AB3B86E04B
:107C70000E940731892B19F4C0E0D0E015C00E94A2
:107C80009E3BC82F86E00E940731282F8091390142
:107C900081FD0AC02150203108F02FE085E491E0F9
:107CA0006FE040E00E944E418091940090919500D9
:107CB000909343228093422281E080933022F89473
:107CC00080913901826080933901809139018D7FE3
:107CD000809339011E5F81EA9AE0612F0E947C4106
:107CE00078948091A6219091A72101969093A72145
:107CF0008093A6210E94723B8823E1F382E491E005
:107D000060EE45E00E944441182F86E00E94073152
:107D1000892B71F08091390181FD0AC02C2FC0316F
:107D200008F02FE085E491E06FE040E00E944E41D2
:107D3000002319F00E941F3C02C00E945B3C80910E
:107D400030228823E9F18091940090919500209150
:107D500042223091432282179307A0F4809110228F
:107D600090911122A0911222B09113228C57914E22
:107D7000AF4FBF4F8093102290931122A0931222F5
:107D8000B09313228091940090919500821B930BE5
:107D9000A0E0B0E0209110223091112240911222F7
:107DA00050911322820F931FA41FB51F809310229E
:107DB00090931122A0931222B0931322109230229A
:107DC0008091AC21882361F080919400909195007E
:107DD000909345228093442281E08093312207C012
:107DE00082E491E06FE140E023E00E944E410E9476
:107DF000FF3C113011F410E01EC01330A9F4809143
:107E0000E8219091E921A091EA21B091EB2101961E
:107E1000A11DB11D8093E8219093E921A093EA214F
:107E2000B093EB2112E007C0153011F413E003C04A
:107E3000173009F411E0812F90E0DF91CF911F916D
:107E40000F910895CF93DF93EB010E94123D9C01A7
:107E5000009731F4CE010E94C63D9C01009749F085
:107E60008091A9219091AA2101969093AA218093B3
:107E7000A921C901DF91CF910895282F81E0809336
:107E80009E0A8091390181FD09C0203108F02FE060
:107E900085E491E06FE040E00E944E410E94FF3C8B
:107EA00008951F93182F0E94723B8823E1F31093CB
:107EB0009D0A88E491E06FE140E0212F0E944E414D
:107EC0001F9108950E94513F86E00E94AB3B0895A8
:107ED0008FEF80934E018CE691E060EF44E022E06A
:107EE0000E944E418CE290E06EE041E025E00E946D
:107EF0004E4180E880936F018091460180936D012F
:107F000084E491E060E245E021E00E944E41089562
:107F10008FEF94E00E94572B81E08093172080918F
:107F20001820909119200196909319208093182081
:107F300081E090E00895CF93DF93582FA92F2091EF
:107F40001F20822F90E0FC01F695FE2FEE27F7957B
:107F5000E795880F991FE80FF91FE05EFF4D4081FC
:107F6000442309F409C18091390181FD05C1809143
:107F7000AC21882309F400C147FF23C0822F90E081
:107F8000FC01F695FE2FEE27F795E795880F991FD0
:107F9000E80FF91FE05EFF4D10828091E021909183
:107FA000E121A091E221B091E3210196A11DB11D33
:107FB0008093E0219093E121A093E221B093E3210B
:107FC000DBC0433018F5822F90E0FC01F695FE2FC0
:107FD000EE27F795E795880F991FE80FF91FE05EE8
:107FE000FF4D10828091DC219091DD21A091DE2156
:107FF000B091DF210196A11DB11D8093DC219093EA
:10800000DD21A093DE21B093DF21B6C0C42FD0E0E4
:1080100022976C177D0718F5822F90E0FC01F695EA
:10802000FE2FEE27F795E795880F991FE80FF91FA8
:10803000E05EFF4D10828091D8219091D921A091CE
:10804000DA21B091DB210196A11DB11D8093D821C9
:108050009093D921A093DA21B093DB218DC0822F98
:1080600090E09C013695322F222737952795880F6F
:10807000991F280F391F2F5D3F4D852F9A2FB9016A
:1080800050E00E94206720911F20822F90E0FC0189
:10809000F695FE2FEE27F795E795880F991FE80FC5
:1080A000F91FE056FF4D808180931020822F90E0D1
:1080B000FC01F695FE2FEE27F795E795880F991F9F
:1080C000E80FF91FE05EFF4D10822F5F20931F2005
:1080D000233010F010921F2080911F2090E0FC01AF
:1080E000F695FE2FEE27F795E795880F991FE80F75
:1080F000F91FE05EFF4D8081882311F00E94883FC8
:10810000609147016093112080911620882311F01F
:10811000681710F46093162080911F2090E0FC01F6
:10812000F695FE2FEE27F795E795880F991FE80F34
:10813000F91FE056FF4D80818093102084E070E0AD
:108140000E94FC306091102083E070E00E94FC30BF
:108150008091F4219091F521A091F621B091F72121
:108160000196A11DB11D8093F4219093F521A09358
:10817000F621B093F72102C0C0E0D0E0CE01DF913C
:10818000CF910895CF93DF93EC0188819981009777
:1081900021F08E5F944049F505C08EEF94E09983FD
:1081A000888302C0623811F081E022C0109217204B
:1081B0000E9443310E94B83060E870E00E949B3F0B
:1081C0001816190644F40E94B330E0917F05F0912F
:1081D00080050995E2CF8091142090911520019699
:1081E0009093152080931420D8CF1982188283E0B1
:1081F000DF91CF9108950F931F930DEF13E0C80106
:108200000197F1F70E943A41109220201092A2208B
:108210001092242110921F2010921E20E9E3F1E019
:1082200080818E7F808380818D7F80838DE090E050
:108230000197F1F780818160808382E491E06FE1B2
:1082400040E023E00E944E41C8010197F1F7809180
:108250005D0180915E010E94683F8FEF94E060E0D5
:1082600070E00E942A2B0E941F3C81E090E01F9149
:108270000F9108951092230B1092220BEFE6F0E07D
:108280008081806280830895FC018081862390E054
:1082900002C0959587954A95E2F70895F894FC01F8
:1082A0009081862F8095892330E002C0220F331FF2
:1082B0004A95E2F76223862B808378940895CF93C2
:1082C000DF93FC01EC01219680917B018083A0E883
:1082D000B1E08150282F30E02F573E4F8D91899388
:1082E000A217B307D9F7E058FF4F8C91819381E033
:1082F0008083DF91CF910895DC0160938001E1E8F4
:10830000F1E0635070E06E577E4F8D918193E617D8
:10831000F707D9F708951F920F920FB60F92112405
:108320000F900FBE0F901F9018951F920F920FB6CF
:108330000F9211240F900FBE0F901F9018951F924F
:108340000F920FB60F9211240F900FBE0F901F9037
:1083500018951F920F920FB60F9211241092AB2115
:108360000F900FBE0F901F9018951F920F920FB68F
:108370000F9211241092AB210F900FBE0F901F90FF
:1083800018951F920F920FB60F9211248F9381E0D0
:10839000809317208F910F900FBE0F901F9018950C
:1083A0001F920F920FB60F9211241092AB210F90D3
:1083B0000FBE0F901F9018951F920F920FB60F923D
:1083C00011248F939F938091220B9091230B019600
:1083D0009093230B8093220B9F918F910F900FBE50
:1083E0000F901F9018951F920F920FB60F920BB619
:1083F0000F9211242F933F934F935F936F937F932B
:108400008F939F93AF93BF93CF93DF93EF93FF939C
:10841000809147018093112090911E2082E8989FBF
:10842000E0011124C05EDF4DFE01319680917B0199
:108430008883A0E8B1E08150282F30E02F573E4FCD
:108440008D918193A217B307D9F7FE01E058FF4F32
:108450008C918083FE01EF57FF4F81E080838091F4
:108460001E208F5F80931E20833010F010921E20FC
:108470000E94883FFF91EF91DF91CF91BF91AF9123
:108480009F918F917F916F915F914F913F912F912C
:108490000F900BBE0F900FBE0F901F90189510926B
:1084A000B90080E28093B8000895982F84EA809301
:1084B000BC008091BC0087FFFCCF8091B900887F11
:1084C000883021F0803111F081E008959093BB0055
:1084D00084E88093BC008091BC0087FFFCCF909122
:1084E000B900987F983111F480E0089580E09034CD
:1084F00009F081E00895982F44EA34E824E9409394
:10850000BC008091BC0087FFFCCF8091B900887FC0
:10851000883011F0803199F79093BB003093BC0004
:108520008091BC0087FFFCCF8091B900887F8032AA
:1085300011F0883539F42093BC008091BC0084FD93
:10854000FCCFDDCF08950E945542089584E98093C1
:10855000BC008091BC0084FDFCCF08958093BB00DB
:1085600084E88093BC008091BC0087FFFCCF8091A1
:10857000B90090E0887F883209F091E0892F089552
:1085800084EC8093BC008091BC0087FFFCCF80917D
:10859000BB00089584E88093BC008091BC0087FFF5
:1085A000FCCF8091BB000895CF93DF93EC01A0E056
:1085B000B0E0FE01EA0FFB1F808180933F0111961E
:1085C000A031B105B1F780913C018F7D80933C01D2
:1085D00080913C01877F80933C01A0E0B0E0FB01EB
:1085E000EA0FFB1F808180933E011196A031B105F7
:1085F000B1F780913C01806880933C0180913D01FE
:1086000080FFFCCF4051504080913C0180628093BC
:108610003C0180913C01877F80933C0117C0A0E022
:10862000B0E0FB01EA0FFB1F808180933E011196B1
:10863000A031B105B1F780913C01806880933C0185
:1086400080913D0180FFFCCF40515040141615062B
:1086500034F340E050E080913E01F901E40FF51F52
:1086600080834F5F5F4F40315105A9F781E090E073
:10867000DF91CF9108950F931F93CF93DF93809154
:10868000B4219091B521A091B621B091B721019666
:10869000A11DB11D8093B4219093B521A093B62163
:1086A000B093B7210E940B468C0184E29BE00E94AC
:1086B000132C08C0EA81FB81309709F00995CE019F
:1086C0000E94302DEC010097A9F70115110519F052
:1086D000C8010E942129DF91CF911F910F91089528
:1086E0000E94854D0E9443310E94954480E695E0AA
:1086F0009093AF218093AE210E941E4682E090E0CD
:1087000060E074E040E05EE12FEF31E00E94B244AF
:108710000895CF93DF93EC018091B0219091B12126
:10872000A091B221B091B3210196A11DB11D8093FA
:10873000B0219093B121A093B221B093B321CE0187
:108740000E94EB45892B19F420E030E00CC00E9418
:10875000FB31E0916405F091650587EB93E4BE0180
:10876000099521E030E0C901DF91CF910895CF92C2
:10877000DF92EF92FF920F931F93CF93DF937C01D1
:108780008B016A0184E29BE00E94132C09C0EC81FA
:10879000FD81309711F0C8010995CE010E94302D5E
:1087A000EC010097A1F7C701B801A6010E94292991
:1087B000DF91CF911F910F91FF90EF90DF90CF90BD
:1087C0000895BC0184E29BE00E94C72C0895BC017F
:1087D00084E29BE00E942E2C08950F93FC011086EA
:1087E000A0912A0BB0912B0B109751F082819381AD
:1087F00060E040E050E020E030E000E0FD0109955D
:108800000F9108950F93FC01AB012481358181E024
:10881000808775836483A0912A0BB0912B0B1097EE
:1088200031F08281938161E000E0FD0109950F91B3
:1088300008950F93FC01A0912A0BB0912B0B109778
:1088400049F024813581828193816085A90101E00D
:10885000FD0109950F910895E091280BF091290BE6
:10886000309709F0099508959093290B8093280B70
:10887000089590932B0B80932A0B089586E29BE03A
:108880000E94132C0895EF92FF920F931F93CF93A2
:10889000DF938C01EB017A0186E29BE00E94132CAE
:1088A00013C0828193818C179D0759F4A681B781EB
:1088B000109769F0CF01B801AE019701FD0109954C
:1088C00006C0CF010E94302DFC01009751F7DF91C7
:1088D000CF911F910F91FF90EF900895BC0186E218
:1088E0009BE00E94C72C08950F93CF93DF93EC0178
:1088F0007B836A8318865F834E8386E29BE0BE019A
:108900000E942E2CE0912A0BF0912B0B309749F00E
:108910004C815D818A819B81688520E030E001E0A7
:108920000995DF91CF910F91089586E29BE00E9417
:108930000F2C0895089580915D0B90915E0B089522
:108940000F931F9307E41BE0C8010E941E4BC80150
:1089500040970E941E4BC8014B970E94D9281F9137
:108960000F910895CF92DF92EF92FF920F931F9392
:10897000FC018B017A0169018CE29BE0BF0145E4B7
:1089800055E00E94DC281093580B0093570BF0928F
:108990005A0BE092590BD0925C0BC0925B0B84E7B0
:1089A00095E40E9439441F910F91FF90EF90DF9062
:1089B000CF900895AF92BF92CF92DF92EF92FF9245
:1089C0000F931F93DF93CF9300D000D000D0CDB78B
:1089D000DEB77B010E94B830FC010190F081E02DF0
:1089E000FA83E983EC30F10568F400E010E053E02D
:1089F000A52EB12CAC0EBD1E45E0C42ED12CCC0E44
:108A0000DD1E39C000D000D088E295E0ADB7BEB71A
:108A100012969C938E9311971496FC93EE93139752
:108A20000E94AA670F900F900F900F9029C00E948C
:108A3000B830F801EE0FFF1FEE0FFF1FE80FF91F10
:108A400082819381F501918380830E94B8300F5F0A
:108A50001F4FF801EE0FFF1FEE0FFF1FE80FF91F6A
:108A600040815181D6014C9311965C936B817C813E
:108A7000C7010E94434489819A8108171907B8F2F7
:108A800026960FB6F894DEBF0FBECDBFCF91DF9113
:108A90001F910F91FF90EF90DF90CF90BF90AF901C
:108AA00008950F931F9307E41BE060915D0B709195
:108AB0005E0BC80143E855E420E030E00E94604BC3
:108AC0000E94B24C60915D0B70915E0B0E940D6430
:108AD000BC01C801409748E955E420E030E00E941D
:108AE000604B1F910F9108950F93013051F48091C5
:108AF000570B9091580B90935E0B80935D0B0E94E7
:108B000051450F91089580915D0B90915E0B2091DE
:108B10005B0B30915C0B880F991F2817390708F4FD
:108B2000C90190935E0B80935D0B0E94514508959F
:108B3000CF93DF930E9443310E94B830EC01198239
:108B400018820E943E4425C0E881F981EE0FFF1F84
:108B5000EE0FFF1FEC0FFD1F12968D919C91139746
:108B600093838283E881F9813196EE0FFF1FEE0F28
:108B7000FF1FEC0FFD1F14968D919C91159791830B
:108B8000808388819981019699838883CD010E9491
:108B9000302DDC01009729F018968C9118978823C6
:108BA00099F688819981880F991F880F991F0296DD
:108BB0000E94B33088819981892B21F08CE29BE05F
:108BC0000E94CB28DF91CF910895E0914D05F0915F
:108BD0004E0509950895EF92FF920F931F938C0114
:108BE000E0914B05F0914C050995F82EE92EF8011E
:108BF0006281738181E00E94FC302F2D3E2DC901DE
:108C00009C01009711F021E030E0C9011F910F9104
:108C1000FF90EF900895CF93DF93E0914905F09195
:108C20004A050995EC01009729F06A817B8181E072
:108C30000E94FC30CE01DF91CF9108950E949029CF
:108C40000895FC01818190E0308120E0822B932BFC
:108C500002C0880F991F6A95E2F7892F9927FA01B8
:108C6000E15BFA4F208130E08223932328E030E05B
:108C7000241B350B02C0969587952A95E2F7089537
:108C8000CF92DF92EF92FF920F931F93CF93DF93D8
:108C90007C018A01A901283031050CF5FB012181F5
:108CA00030E0908180E0282B392B02C0220F331F47
:108CB0000A95E2F7232F3327FA01E15BFA4F80810F
:108CC00090E02823392388E090E0841B950B02C0B4
:108CD000369527958A95E2F7F701208375C06901DB
:108CE000E3E0D594C794EA95E1F70115110521F069
:108CF000DB01C0E0D0E029C0C0E0D0E0F701EC0F1C
:108D0000FD1FDB01AC0FBD1F8C9180832196CC151C
:108D1000DD05A4F3477050704115510509F454C0A6
:108D20006C0F7D1FCE0DDF1DFB01308120E0232F56
:108D30003327FA01E15BFA4F808190E02823392341
:108D400088E090E0841B950B39C0F701EC0FFD1F04
:108D50003C9120E011968C91119790E0822B932BFF
:108D6000002E02C0880F991F0A94E2F79083219683
:108D70001196CC15DD054CF3DA01A770B070109791
:108D800019F1FB01EC0FFD1FCE0DDF1D218130E03D
:108D9000908180E0282B392B02C0220F331F0A95C7
:108DA000E2F7232F3327FD01E15BFA4F808190E04A
:108DB0002823392388E090E08A1B9B0B02C036955C
:108DC00027958A95E2F72883DF91CF911F910F9124
:108DD000FF90EF90DF90CF900895FC0120E030E00D
:108DE00004C08181280F311D329680818823C9F704
:108DF000C9010895FC0150E080E190E0861B970BCB
:108E0000821B930B02C0440F551F8A95E2F78081A5
:108E1000852B80838181842B81830895AF92BF92BB
:108E2000CF92DF92EF92FF920F931F93CF93DF9336
:108E30008C016A0179012830310584F4FA0120811E
:108E400030E080E190E0861B970B8E199F0902C0ED
:108E5000220F331F8A95E2F7F8016FC05901A3E092
:108E6000B594A794AA95E1F76115710551F0E80151
:108E7000A0E0B0E044275527461B570B485F5F4FE3
:108E800026C0C0E0D0E0F801EC0FFD1FD601AC0F0A
:108E9000BD1F8C9180832196CA15DB05A4F3A70121
:108EA000477050704115510509F44DC0F801EC0FA1
:108EB000FD1FCC0DDD1D288130E088E090E0841B93
:108EC000950B02C0359527958A95E2F72CC0F601DF
:108ED000EA0FFB1F808190E0042E02C0880F991FCB
:108EE0000A94E2F72881292B28832981282B2983BA
:108EF00011962196AA15BB0554F3A701477050702F
:108F00004115510501F1F801EA0FFB1FAC0DBD1D24
:108F10002C9130E0685F7F4F641B750B02C0359564
:108F200027956A95E2F730E080E190E0841B950B8D
:108F300002C0220F331F8A95E2F78081832B808342
:108F40008181822B8183DF91CF911F910F91FF90BF
:108F5000EF90DF90CF90BF90AF9008954F925F92C7
:108F60006F927F928F929F92AF92BF92CF92DF9239
:108F7000EF92FF920F931F93DF93CF9300D0CDB763
:108F8000DEB77C01DC0116962C9140E050E0822F88
:108F900090E087709070892B11F041E050E02695A9
:108FA000269526958A01020F111DC80102960E947E
:108FB0006F30892B19F420E030E054C00E94C53096
:108FC000FC01D70112968C911297808313968C9195
:108FD00081830E94C53022E0622E712C680E791EBA
:108FE000C30160E070E0A8010E942967F701A48036
:108FF000B580CC24DD242E010894411C511C2CC0CA
:10900000D50111968C91E82EFF24860183E01595F9
:1090100007958A95E1F7060D171DB7E08B2E912C69
:109020008C209D20983138F0892F0E941031AC019E
:10903000C801B40108C0892F0E9407319A8389832F
:10904000C801B401A20197010E940E47CE0CDF1C9B
:10905000E2E0F0E0AE0EBF1ED5019C91992381F6AF
:1090600021E030E0C9010F900F90CF91DF911F9167
:109070000F91FF90EF90DF90CF90BF90AF909F90B7
:109080008F907F906F905F904F9008954F925F9276
:109090006F927F928F929F92AF92BF92CF92DF9208
:1090A000EF92FF920F931F93DF93CF9300D000D0E6
:1090B000CDB7DEB70E94B830182F092F82E090E0BC
:1090C0000E949430892B09F466C0E12FF02F918122
:1090D00080E02081820F911D0E9455294C0100974C
:1090E00009F45BC00E94B8305C01F401268140E0C5
:1090F00050E0822F90E087709070892B11F041E052
:1091000050E0269526952695CA01820F911D0E9452
:109110009430892B09F43FC0F40104811581CC24DB
:10912000DD2443E0442E512C4C0E5D1E3E0108947C
:10913000611C711C2BC0F8018181E82EFF24B6014F
:1091400033E0759567953A95E1F76A0D7B1DA601A9
:1091500047705070983150F0C30197010E9440460B
:10916000F8018081B3010E9418310CC01C821B825F
:10917000C20197010E9440466B817C81F801808189
:109180000E94FC30CE0CDF1C0E5F1F4FF801908157
:10919000992389F602C088249924C4010F900F9066
:1091A0000F900F90CF91DF911F910F91FF90EF9053
:1091B000DF90CF90BF90AF909F908F907F906F90F7
:1091C0005F904F900895E0917D05F0917E0509959F
:1091D0000895E0912605F091270509950895E091FD
:1091E0008105F091820509950895E0918305F0913C
:1091F00084050995089580E090E008950895E09130
:109200001905F0911A0509950895892B31F0E0911F
:109210001905F0911A0509950895E0911B05F09143
:109220001C050995089580E090E008950F931F9321
:10923000DF93CF93CDB7DEB7E0970FB6F894DEBFDC
:109240000FBECDBF0E94E6308C010E94B830602F67
:10925000AE014F5F5F4F0E941A51882309F443C04B
:1092600088A99801281B3109C9010E949430892BD3
:10927000D1F12E81222361F18A859B853BEA8D3CC9
:10928000930719F08F5F9F4F71F5223071F028E03E
:1092900030E0BE01645F7F4F21503040FB01E20FA0
:1092A000F31F80818F3F21F007C022E030E0F1CF33
:1092B000121613068CF30CC089E10E94183189E163
:1092C0000E9410316BE17FE10E94A328892B59F0A5
:1092D00088E1BE016A5E7F4F0E941831E091660509
:1092E000F09167050995E0960FB6F894DEBF0FBEC2
:1092F000CDBFCF91DF911F910F910895AF92BF9293
:10930000CF92DF92EF92FF920F931F93DF93CF9351
:10931000CDB7DEB7E0970FB6F894DEBF0FBECDBF76
:109320006C015B01FE01319680E3DF011D928A959D
:10933000E9F781E089831A821B828CE00E94073161
:109340008C831D821F828091610B89878F5F809340
:10935000610B03E008878DEC9BEA9B878A8789E194
:109360000E9410316AE874E00E94A328892B31F032
:1093700082E08E838FEF8C878D8709C089E10E9400
:109380001031BC01CE010C960E949B280E838DECFF
:109390009BEA9D8B8C8BCE0146966BE17FE10E9410
:1093A0009B280E94B8309FA78EA70E94E63088AB0A
:1093B0007E010894E11CF11CC7010E943153082F63
:1093C00090E00E946F30892B39F10E94C530BC01BA
:1093D000C701402F0E945B52E0900F05F0901005EE
:1093E0000E94C5308C010E94F030BC01C801F70119
:1093F0000995C114D10481F0009719F0019761F427
:1094000004C0C50160E070E003C0C50164E070E025
:1094100041E050E0F6010995E0960FB6F894DEBF02
:109420000FBECDBFCF91DF911F910F91FF90EF90B5
:10943000DF90CF90BF90AF9008950E94B24C809380
:10944000610BE0911905F0911A0509950895CF93E4
:10945000DF93EC0102C00E94372A8991999100970D
:10946000D1F7DF91CF910895CF93DF93EC0104C042
:1094700060E070E00E942A2B899199910097C1F7D2
:10948000DF91CF910895FC01808191812281338108
:10949000820F931F918380830895EF92FF920F9321
:1094A0001F93FC01E080F180028113810E94A538A6
:1094B0000E0D1F1D081B190BC8011F910F91FF9066
:1094C000EF9008950F931F938C010E94A53840E000
:1094D00050E0F80120813181821B930B019622819B
:1094E00033812817390710F441E050E0CA011F9179
:1094F0000F9108950F931F938C010E94A538F801D6
:10950000918380831F910F9108950F931F938C0176
:10951000FC01738362830E94A538F80191838083E4
:109520001F910F910895EF92FF920F931F93CF9386
:10953000DF937C018A01FC0180819181009729F0F1
:109540008B34910509F04BC01AC082E69BE00E9463
:10955000132CEC0109C06C817D81CE0102960E9422
:10956000A12E0990D881C02D2097A9F781E0809382
:10957000640B8BE490E0F7019183808302C068382C
:1095800011F081E030C082E69BE00E94132CEC01D8
:1095900023C0CE01029608171907D9F482E69BE092
:1095A000BE010E94C72C00918E0910918F098A85F7
:1095B0009B8590938F0980938E09EC85FD8530976C
:1095C00019F08E859F85099510938F0900938E0958
:1095D000D0CF0990D881C02D2097D9F6CACFF701F6
:1095E0001182108283E0DF91CF911F910F91FF9044
:1095F000EF900895CF93DF93EC018091640B882363
:1096000031F0CE0102960E943A2D9C0113C082E6F1
:109610009BE00E94132CFC0109C0EC17FD0719F414
:1096200020E030E007C00190F081E02D3097A9F7ED
:1096300021E030E0C901DF91CF910895CF93DF930E
:10964000EC018091640B882329F0CE0102960E94E0
:109650009F2D04C01F821E821986188682E69BE019
:10966000BE010E94C72CDF91CF9108950F931F93E5
:10967000CF93DF93EC018091640B882391F00091EC
:109680008E0910918F0986E995E090938F09809358
:109690008E09CE0102960E948B2E10938F090093A3
:1096A0008E0982E69BE0BE010E94C72C82E69BE009
:1096B000BE010E942E2CDF91CF911F910F91089532
:1096C0000F931F93CF93DF93EC0180918E099091BC
:1096D0008F099B878A875D874C873F872E8780917C
:1096E000640B882399F000918E0910918F0986E907
:1096F00095E090938F0980938E09CE0102960E9487
:10970000A12E10938F0900938E0902C07D836C8374
:1097100082E69BE0BE010E94C72C82E69BE0BE0170
:109720000E942E2CDF91CF911F910F9108950F93DE
:109730001F93CF93DF93EC018091640B882391F00A
:1097400000918E0910918F0986E995E090938F0919
:1097500080938E09CE0102960E94962E10938F0957
:1097600000938E0982E69BE0BE010E94C72C82E630
:109770009BE0BE010E942E2CDF91CF911F910F9193
:1097800008951092640B82E69BE00E940F2C86E9FC
:1097900095E060E070E00E942A2B0895CF93DF935C
:1097A000E6E3F2E2C8EFD1E2AAE2B2E2119211924C
:1097B00019921992199219921D9282E2EE34F807C9
:1097C000A9F7DF91CF910895CF92DF92EF92FF92A8
:1097D0000F931F93CF93DF93EC01FC01E65DFD4DEA
:1097E0008081882349F10091940010919500BE0179
:1097F000660F771F660F771F68507E4DFE01EE0FD4
:10980000FF1FEA5CFD4D808191819801281B390B77
:109810006901EE24FF24DB012D913D914D915C9176
:109820001397C20ED31EE41EF51ECD92DD92ED926B
:10983000FC92139711830083FE01EE0FFF1FEE0FC2
:10984000FF1FE850FE4D6081718182819381DF911D
:10985000CF911F910F91FF90EF90DF90CF900895DF
:1098600060E070E080E090E00895FC01EE0FFF1FE3
:10987000EE0FFF1FE850FE4D4083518362837383D8
:1098800008950F931F93CF93DF930AE212E2C8EF7C
:10989000D1E2E6E3F2E2D8018C918823C9F060912D
:1098A000940070919500808191819B01281B390B58
:1098B00040E050E088819981AA81BB81820F931F8B
:1098C000A41FB51F88839983AA83BB837183608398
:1098D0000F5F1F4F24963296B2E206331B07D9F66C
:1098E000DF91CF911F910F910895A091650BB091D9
:1098F000660B1097C1F01092660B1092650B1496D0
:109900006D917C9115971296ED91FC911397CD0175
:109910000995E091650BF091660B309721F08081FD
:1099200091810E94915008950F931F93FC018091A3
:10993000650B9091660B33832283158304837183B7
:109940006083F093660BE093650B892B19F4CB01D0
:109950000E94915080E090E01F910F9108950E9425
:10996000775008950E94E86408950E94ED64089578
:10997000FC0180819181089570E06F5B7F4F660FDD
:10998000771F680F791FCB010895E62FF0E0EF5B9A
:10999000FF4FEE0FFF1FE80FF91F8081918108959F
:1099A0000895CF93DF93EC0180EA95E0BE010E9419
:1099B000C92B892B21F0BE016E5F7F4F0CC088EA56
:1099C00095E0BE010E94C92B892B19F460E070E07C
:1099D00002C06A817B81CB01DF91CF910895CF9343
:1099E000DF93EC0180EA95E0BE010E94C92B892B30
:1099F00079F068817981CE0102960E943432CE01DD
:109A00008E579F4FCE54DF4FBE010E946F311DC055
:109A100088EA95E0BE010E94C92B892BB1F00E9413
:109A20004331688179818A819B810E9434328CA97B
:109A300090E00E946F300E94C5304CA99E012C5FBF
:109A40003F4FB90150E00E942067DF91CF91089508
:109A5000CF93DF93EC0180EA95E0BE010E94C92B11
:109A6000892B19F080EA95E009C088EA95E0BE01EB
:109A70000E94C92B892B29F088EA95E0BE010E943B
:109A80009B2BDF91CF910895BC018E579F4F6E5451
:109A90007F4F0E94803108950F931F93CF93DF93E0
:109AA0000E94CF30892BB1F088EA95E00E946D2B9F
:109AB000EC01009769F00E94E630998388830E9448
:109AC000E1309B838A83CE0104960E94DF318CAB08
:109AD0008E0115C080EA95E00E946D2BEC018C018F
:109AE000009769F002960E94913199838883BE01A4
:109AF0006E547F4FCE018E579F4F0E948031C80118
:109B0000DF91CF911F910F91089580EA95E00E9417
:109B1000EC2B88EA95E00E94EC2B0895E091CA11A5
:109B2000F091CB11309711F480E0089509950895D4
:109B30009093CB118093CA110895FC0180918E09F6
:109B400090918F09958F848F778F668F0895FC0190
:109B500080918E0990918F0992878187748763879E
:109B60000895AC011092AF1160918E0970918F0928
:109B7000E8EBF1E120E014C0808191818417950722
:109B800069F4828193818617970741F42093AF117E
:109B900011821082CA010E94EF54089534962F5FFB
:109BA000243050F32093AF11089580EB91E10E948F
:109BB0003A2D892B21F080EB91E10E948B2E0895A4
:109BC000EF92FF920F931F93CF93DF937C018A0153
:109BD000FC0180819181009729F08C50934009F01D
:109BE00002C12CC080E00BC0E82FF0E0EE0FFF1F99
:109BF000EE0FFF1FE854FE4E118210828F5F8430FB
:109C000098F38093AB1180918E0990918F09909376
:109C1000C9118093C8110E94952980934E2280EB30
:109C200091E160E470E00E94A12E0E942B548CE030
:109C300093E0F7019183808381E0D9C0623009F419
:109C4000B4C0633030F4662309F484C0613079F71E
:109C500097C0673819F0683851F73CC01092AC11C2
:109C6000C8EBD1E113C08A819B818017910741F431
:109C7000888199810E94EF54198218821B821A826E
:109C800024968091AC118F5F8093AC118091AC11C0
:109C9000843048F3EEE5F7E209C0848D958D801796
:109CA000910719F4158E148E118EB09627E2EE3DB1
:109CB000F20799F7E4EFF7E208C0818592858017F3
:109CC000910711F4158214823D9688E2E637F80771
:109CD000A1F7ADCFE1E1403B5E0709F0A8CFCA0193
:109CE0000E943A2D892B09F4A2CF1092AC112DC0FD
:109CF000F0E035E0EE0FFF1F3A95E1F7E25AF84D3C
:109D0000818D8823E9F080EB91E10E948B2E809178
:109D1000AC1190E025E0880F991F2A95E1F7825A4F
:109D2000984D90935D2780935C2782E00E948B552D
:109D300080914F2290915022892B11F00E948E4DDC
:109D40008091AC118F5F8093AC11E091AC11E43045
:109D500078F26DCF4115510509F469CF50935D2715
:109D600040935C2783E00E948B5580914F22909115
:109D70005022892B11F00E948E4D0E94D54D57CF55
:109D80004115510509F453CF509359274093582753
:109D900085E00E948B5580914F2290915022892B13
:109DA00009F445CF0E948E4D42CF80914F22909171
:109DB0005022892B09F43BCF80916022863031F408
:109DC0008091782281FF02C00E94D54D81E00E94DF
:109DD0008B5580914F2290915022892B09F427CFE7
:109DE0000E94D24F24CFF7011182108283E0DF91CD
:109DF000CF911F910F91FF90EF900895CF93DF9334
:109E0000A0915C27B0915D27109719F0ED016C9639
:109E100005C0C0915827D09159272996809157277E
:109E200086FF22C01092AD11E8EBF1E140E016C0D0
:109E30002081318114968D919C91159728173907AF
:109E400059F482819381009739F04093AD11998341
:109E500088831B821A8206C034964F5F443040F3D9
:109E60004093AD110E94D54D88819981009731F0C2
:109E70004A815B8160914E220E941B2BDF91CF9122
:109E800008958DEB95E062E040E050E00E941B2BCE
:109E90001092502210924F220895AC018DEB95E064
:109EA00060E00E94F72A0895AC018DEB95E061E037
:109EB0000E94F72A0895CF93DF93EA010E94105D74
:109EC000FC01009741F080918E0990918F09928753
:109ED0008187D487C387CF01DF91CF9108950F93F6
:109EE0001F93DF93CF9300D000D0CDB7DEB78C01A6
:109EF000AB018FEF89838A838B838C83CE0101969C
:109F0000B8010E945B4FFC01009711F01583048398
:109F1000CF010F900F900F900F90CF91DF911F9175
:109F20000F910895AC011092AE11E8EBF1E120E041
:109F300016C0322F3F5F80819181892B71F420936D
:109F4000AE115183408380918E0990918F09938344
:109F50008283CA010E940C5508953496232F243021
:109F600040F32093AE1108950F931F93CF93DF9387
:109F70008A010E946454EC01009771F080918E096F
:109F800090918F099D8F8C8F1F8F0E8F8DEB95E099
:109F900060E0AE010E94F72ACE01DF91CF911F91C0
:109FA0000F910895EF92FF920F931F93809160227B
:109FB000863009F075C080914F22909150228050D8
:109FC000954009F06DC004E912E01093502200930F
:109FD0004F2292E0E92EE092592284E9F82EF09285
:109FE0005A2210927C2210927B220E942354809548
:109FF000909590937C2280937B2210926222109203
:10A0000061220E94B4538095909590936222809330
:10A0100061220E948E4D1093502200934F22E092B5
:10A020005922F0925A2220915A2730915B27C90178
:10A03000FC01DC01A459BD4F8CE692E00D90019229
:10A040000197E1F78FE692E26CE672E00E945453CA
:10A050008091532280936F228091542280937022AA
:10A060008091552280937122809156228093722292
:10A0700010927C2210927B220E942354809590950E
:10A0800090937C2280937B22109262221092612214
:10A090000E94B453809590959093622280936122A0
:10A0A0000E948E4D1F910F91FF90EF900895DC015B
:10A0B00020E040E050E098E115C0FD01E40FF51FFD
:10A0C000E08138E08E2F8227F82FF17080FD29275C
:10A0D0002695F13009F42068315011F0E695F2CF61
:10A0E0004F5F5F4F4617570741F7822F08959FB77D
:10A0F000F894E1E7F0E08081807D808388B38F620F
:10A1000088BB10929000E1E9F0E01082109292007A
:10A1100010929500109294008081856080839FBF8B
:10A1200008952FB7F894909399008093980088B37E
:10A130008F6288BBE1E7F0E08081826080832FBF7F
:10A1400008951F920F920FB60F920BB60F92112423
:10A150002F933F934F935F936F937F938F939F932F
:10A16000AF93BF93EF93FF938091940090919500EC
:10A1700090933B2280933A2281E080932C2280911D
:10A180007100807D809371000E94754C80912C221B
:10A190008823E9F1809194009091950020913A22D2
:10A1A00030913B2282179307A0F480910022909176
:10A1B0000122A0910222B09103228C57914EAF4F01
:10A1C000BF4F8093002290930122A0930222B0936C
:10A1D00003228091940090919500821B930BA0E044
:10A1E000B0E0209100223091012240910222509152
:10A1F0000322820F931FA41FB51F80930022909308
:10A200000122A0930222B093032210922C22FF91EC
:10A21000EF91BF91AF919F918F917F916F915F91DE
:10A220004F913F912F910F900BBE0F900FBE0F904B
:10A230001F901895BF92CF92DF92EF92FF920F93EB
:10A240001F93DF93CF93CDB7DEB728970FB6F8945F
:10A25000DEBF0FBECDBF6C01B62E7A0182E086173D
:10A2600008F0C4C0F6019081892F87708983892FF7
:10A2700086958695869581708A83892F82958F70C1
:10A2800081708B83929596959770892F81708C83BE
:10A29000969591709D839181892F8695869583707F
:10A2A0008E8392959F70892F83708F839695969554
:10A2B0009887DA01FE01319688E001900D92815075
:10A2C000E1F7F6018281F701808786010D5F1F4F5C
:10A2D0003E813323A1F1F801918180E0F6012381D1
:10A2E000820F911DF7019287818786010B5F1F4FB7
:10A2F000323091F4C7010B966AE874E00E949B2803
:10A30000F8018181F7018387F6018581F701848750
:10A310008601095F1F4F1CC03330D1F4F601D7010D
:10A3200096012850304084851B968C931B9731975B
:10A330001196E217F307B9F7085F1F4F09C0C7016D
:10A340000B966AE874E00E949B28F701128611863A
:10A3500038853323C1F18D81882361F4F80191811F
:10A3600080E02081820F911DF701948B838B0E5F1B
:10A370001F4F05C0F70181859285948B838B323006
:10A3800089F4C70145966AE874E00E949B28F801A9
:10A390008181F701858BF8018081F701868B0E5F43
:10A3A0001F4F1AC03330C1F4D801F70190E017965F
:10A3B0008C911797858B9F5F119731969830B9F7DD
:10A3C000085F1F4F09C0C70145966AE874E00E9404
:10A3D0009B28F701148A138A902F9C198B2D891BB7
:10A3E000F70187A716A705A7B91608F490E0892FEB
:10A3F00028960FB6F894DEBF0FBECDBFCF91DF9188
:10A400001F910F91FF90EF90DF90CF90BF90089534
:10A41000CF93DF93FC01DB0185E0EB0119928A9574
:10A42000E9F7858190E083709070892B11F082E0CC
:10A430008C93878190E083709070892B21F082E06B
:10A4400012968C931297858190E083709070892B7F
:10A4500099F0878190E083709070892B69F023894F
:10A460003489818592852817390731F481E0848306
:10A4700012961C92129701C01482858183708230DB
:10A4800021F0833021F488E003C082E001C080E045
:10A4900011968C93119787818370823021F08330DD
:10A4A00021F488E003C082E001C080E013968C9321
:10A4B000DF91CF910895CF92DF92EF92FF920F93A9
:10A4C0001F93DF93CF9300D000D00F92CDB7DEB7AC
:10A4D0007C016B01042FBE016F5F7F4F0E94085209
:10A4E00049818A8190E0840F911D03962B81820F10
:10A4F000911D2C81820F911D2D81820F911D10E0E5
:10A500000817190714F480E09EC0D70111962C910A
:10A51000119730E021703070F3E0220F331FFA956D
:10A52000E1F712968C91129790E081709070E4E0C0
:10A53000880F991FEA95E1F7282B8C918770282BBB
:10A5400013968C91139790E08170907075E0880F4E
:10A55000991F7A95E1F7282B14968C91149790E027
:10A560008170907066E0880F991F6A95E1F7282B3B
:10A57000F601208315962C91159730E023703070EA
:10A58000220F331F220F331F16968C91169790E0DF
:10A590008370907034E0880F991F3A95E1F7282B6B
:10A5A00017968C9117978295880F880F807C822B45
:10A5B000818318968C918283423011F043E00AC067
:10A5C000D70119968C911997F60183831A968C916D
:10A5D000848345E03A81A32FB0E01A96AE0DBF1DEB
:10A5E00020E007C0F601E90FF11D8C9180832F5FF9
:10A5F0001197922F940F2317A9F78B81823081F442
:10A60000F601E90FF11DD70153968C915397808382
:10A610009F5FF601E90FF11D54968C9180839F5F37
:10A620003C81A32FB0E05496AE0DBF1D20E007C0C3
:10A63000F601E80FF11D8C9180832F5F1197822F17
:10A64000890F2317A9F70F900F900F900F900F907D
:10A65000CF91DF911F910F91FF90EF90DF90CF90FE
:10A660000895DF93CF9300D000D00F92CDB7DEB71F
:10A67000BE016F5F7F4F0E94085289819A81890FC6
:10A680008D5F9B81890F9C81890F9D81890F0F9020
:10A690000F900F900F900F90CF91DF9108959093AE
:10A6A000D3118093D2110895FC015381560F50931A
:10A6B0005622272F33274281420F40935522A181F2
:10A6C000A0935422E081E0935322842F90E08217DC
:10A6D000930748F48A2F8F5F80935422882319F4BC
:10A6E000EF5FE0935322852F90E0707086179707F5
:10A6F00090F4842F8F5F80935522882361F480919A
:10A7000054228F5F80935422882329F4809153220E
:10A710008F5F809353220895FC0161507040680F51
:10A72000791F20E030E00EC0508140E08181DA01E5
:10A73000A80FB11D2A0F3B1F2A173B0710F42F5FEC
:10A740003F4F3296E617F70778F3E617F70749F415
:10A75000908180E0280F391F2817390710F42F5FE8
:10A760003F4F832F922F0895E7E5F2E240E050E05B
:10A77000308120E08181B901680F711D460F571F9C
:10A780004617570710F44F5F5F4F329672E2EB3671
:10A79000F70771F74115510519F42FEF3FEF02C08C
:10A7A000342F252FC901089590915A22692F70E006
:10A7B000645170403091592220E0620F731FAB0149
:10A7C000480F511DE3E6F2E2308120E08181D9019A
:10A7D000A80FB11D4A0F5B1F4A175B0710F44F5FAC
:10A7E0005F4F3296B2E2EB36FB0771F76150704073
:10A7F0006E0F7F1F0EC0308120E08181D901A80F2C
:10A80000B11D4A0F5B1F4A175B0710F44F5F5F4F84
:10A810003296E617F70778F3E617F70751F49081B9
:10A8200080E0480F591F4817590718F44F5F5F4FD2
:10A8300006C04115510519F42FEF3FEF02C0342F28
:10A84000252FC901089586E00E94D453089581E11F
:10A850000E94D453089580E009C0E82FF0E0EE0F85
:10A86000FF1FE252F84D118210828F5F8430A8F3EF
:10A8700080E00BC0E82FF0E095E0EE0FFF1F9A9507
:10A88000E1F7E25AF84D118E8F5F843098F380E043
:10A8900094E09093D9118093D81120E04DE050E0DE
:10A8A0000EC0822F90E0849FF001859FF00D949F51
:10A8B000F00D1124EC50F84D158214822F5F2A30D0
:10A8C00080F32093DA1108950F931F93CF93DF93B2
:10A8D0008C01EB014091D8115091D9114F5F5F4F1E
:10A8E0008DE74030580710F040E050E1342F252F1D
:10A8F00060E012C0E62FF0E075E0EE0FFF1F7A95E2
:10A90000E1F7E25AF84D818D882329F08481958101
:10A910008217930719F36F5F643061F74093D81182
:10A920005093D9111092DA11E0E0F0E020E01EC05F
:10A93000A22FB0E035E0AA0FBB1F3A95E1F7A25A6B
:10A94000B84D59968C915997882321F42093DA11A8
:10A95000FD0110C0873049F4309731F05A969C9130
:10A960005A97828D891708F4FD012F5F243000F378
:10A970002093DA11309769F182E0818F8091D411B0
:10A9800084878091D51185878091D61186878091A3
:10A99000D711878788ED94E0938B828B958B848B7E
:10A9A00081E090E0918B808B138E81E0828F83E039
:10A9B000808F168A80E1878B54834583D783C68333
:10A9C000E80188819981AA81BB8180839183A283D8
:10A9D000B383CF01DF91CF911F910F910895AC0107
:10A9E0001092DA1120E013C0E22FF0E0322F3F5F27
:10A9F000EE0FFF1FE252F84D808191818417950779
:10AA000029F42093DA11118210820895232F243023
:10AA100058F32093DA110895AC011092DA1120E076
:10AA200012C0E22FF0E0322F3F5FEE0FFF1FE25225
:10AA3000F84D80819181892B29F42093DA1151837B
:10AA400040830895232F243060F32093DA11089572
:10AA5000BC0180915C2790915D2708960E94545319
:10AA6000E0915C27F0915D27809153228087E091EF
:10AA70005C27F0915D27809154228187E0915C27CB
:10AA8000F0915D27809155228287E0915C27F091BB
:10AA90005D278091562283870895282F892F922F32
:10AAA0000895EF92FF920F931F939C01442755271F
:10AAB000F22EE32E00E010E0362F272F40E050E08A
:10AAC000A90133272227E22AF32A042B152BB701E9
:10AAD000C8011F910F91FF90EF900895FC014091E4
:10AAE00051225091522227E537E2241B350B621781
:10AAF00073070CF49B011216130664F42093F227DB
:10AB00003093F327E417F50729F0CA01BF01A90123
:10AB10000E94206708950F931F93CF93DF93C091F6
:10AB20005C27D0915D27843009F402C22FE732E21E
:10AB300030935B2720935A2730935222209351223F
:10AB4000833091F4898D282F30E02F7030702330BE
:10AB5000310529F488899989892B09F48EC022301E
:10AB6000310509F052C77CC0823009F08AC080915B
:10AB7000D7118F5F8093D711882399F48091D611D4
:10AB80008F5F8093D611882361F48091D5118F5FF8
:10AB90008093D511882329F48091D4118F5F8093FD
:10ABA000D4111092502210924F221092F32710923B
:10ABB000F227298D273011F0253041F48A8D8F5FDF
:10ABC0008A8F843109F021C7198E1FC7222309F407
:10ABD0001CC788899989892B09F44BC08A8D8150BB
:10ABE0008A8F8F5F09F011C73B8D383029F02150D3
:10ABF000223048F4353039F4198E80E88093572795
:10AC00000E94FE4EB8C5353010F080E307C083E0E7
:10AC100090E002C0880F991F3A95E2F78A8F8B8DDA
:10AC20008F5F8B8F898D90E08F709070833091054E
:10AC3000D1F08430910544F48130910509F46EC35C
:10AC4000029709F0E2C60CC08630910509F426C5CA
:10AC50008830910509F422C5049709F0D6C61EC5AF
:10AC6000109278225EC384E0809357270E94FE4EA4
:10AC7000B7C52F70233009F0C8C688E080935727E6
:10AC80006EC5853019F5E0915827F09159278481D8
:10AC90009581892B09F4B9C610925D2710925C2723
:10ACA000C9010C9790935B2780935A279093522267
:10ACB000809351221092F3271092F2271092502283
:10ACC00010924F2288E08093572730C189010852A3
:10ACD000104080915722853409F097C690915922EF
:10ACE00080E020915A22AC01420F511D80914F22E9
:10ACF000909150228417950708F487C650935022EC
:10AD000040934F2280915D2290E08F739070892B49
:10AD100009F07BC680915E22882309F076C64091B7
:10AD2000EE275091EF27C091CB05D091CC054C1761
:10AD30005D0759F42091F0273091F1278091CD05DE
:10AD40009091CE0528173907A1F080916722909144
:10AD500068228417950709F058C62091692230911E
:10AD60006A228091F0279091F1272817390709F07E
:10AD70004CC60E94B4538F5F9F4F09F046C6809126
:10AD80006022863009F43AC18131E9F1813009F05D
:10AD90003CC680916B22883009F037C610926B2236
:10ADA00080916D2290916E22EFEF873F9E0710F009
:10ADB000099601C0089690936E2280936D2280912F
:10ADC000632290916422A0916522B09166228093C3
:10ADD000672290936822A0936922B0936A2280919F
:10ADE000EE279091EF27A091F027B091F127809363
:10ADF000632290936422A0936522B093662280E43C
:10AE0000F8018087DFC580914F22909150224C97A6
:10AE10009093502280934F2283E792E290935B2796
:10AE200080935A278091712290917222892B31F060
:10AE30000E9427548F5F9F4F09F0E7C580916D22D4
:10AE400090916E22892B09F4E0C584EF97E29093EC
:10AE5000592780935827A091CD05B091CE056091D8
:10AE6000C7057091C8054091C9055091CA053FC0FA
:10AE70002481358121153105A9F180916D229091B0
:10AE80006E228217930771F52681378121153105CE
:10AE900039F080916B2290916C228217930711F503
:10AEA000208131812C173D0729F4828193818A17F3
:10AEB0009B0739F12617370729F48281938184177C
:10AEC0009507F9F08091632290916422821793078D
:10AED00049F420916522309166228281938128175E
:10AEE000390779F03D96F0935927E0935827E09180
:10AEF0005827F091592728E2E637F20708F4B8CF2F
:10AF000084C510925D2710925C2782E080935727BA
:10AF100083E792E290935B2780935A279093522283
:10AF2000809351221092F3271092F2270E94FE4E36
:10AF30002091F2273091F3272115310509F465C5D9
:10AF4000C9014C969093502280934F22909359229E
:10AF500080935A22E0915827F09159278085809359
:10AF60005F2281E180936022C901089690936F224D
:10AF700080937022109272221092712284819581A6
:10AF800090936C2280936B228681978190936E229E
:10AF900080936D228091EE279091EF27A091F0276A
:10AFA000B091F1278093632290936422A09365224D
:10AFB000B093662280819181A281B38180936722C0
:10AFC00090936822A0936922B0936A228FE792E25D
:10AFD00090935B2780935A270E94275480959095E1
:10AFE0009093722280937122892B09F0EBC48FEF2A
:10AFF0009FEF9093722280937122E4C40E942354A5
:10B000008F5F9F4F09F001C540916D2250916E22D4
:10B010004115510509F4F9C460916B2270916C22BD
:10B020006115710509F4F1C4CEE5D7E2898D882355
:10B03000E9F08C819D8148175907C1F48E819F8169
:10B040006817790799F420916322309164228881EE
:10B0500099812817390751F4209165223091662291
:10B060008A819B812817390709F473C1A09687E26A
:10B07000CE3BD807D9F2D0F2809178228F738230FC
:10B08000F1F45093DD114093DC111092DA1113C0EA
:10B09000E42FF0E0EE0FFF1FE252F84D2091DC119B
:10B0A0003091DD11808191812817390709F471C031
:10B0B0004F5F4093DA114091DA11443048F38091A8
:10B0C000782282FDA2C484E1F80181A388E290E0A5
:10B0D0009093502280934F2280E580A3909172221A
:10B0E00080917622838F3091712280917522828F98
:10B0F000368F4091702280917422818F458F2091EC
:10B100006F222093DA1180917322808F248F9F5FAA
:10B11000978F992361F4832F8F5F868F882339F46B
:10B12000842F8F5F858F882311F42F5F248F2091C8
:10B130006B2230916C223093DD112093DC118091D1
:10B140006D2290916E22F801958B848B378B268B24
:10B150008091632290916422A0916522B091662231
:10B160008093672290936822A0936922B0936A2209
:10B170008091EE279091EF27A091F027B091F127D1
:10B180008093632290936422A0936522B0936622F9
:10B19000FEC31092DA11C0E0D0E022C0E22FF0E04E
:10B1A000A5E0EE0FFF1FAA95E1F7E25AF84D818D59
:10B1B000882311F4EF0118C0873079F4209721F02B
:10B1C000928D8A8D891748F4C22FD0E075E0CC0F9C
:10B1D000DD1F7A95E1F7C25AD84D2F5F2093DA111F
:10B1E0002091DA112430D0F2209709F40EC4D093C4
:10B1F0005D27C0935C2783E08A8F888F1E8A84E056
:10B200008F8B1B8E80916D2290916E229D838C83FB
:10B2100080916B2290916C229F838E838091632218
:10B2200090916422A0916522B091662288839983CF
:10B23000AA83BB8381E0898F8091D4118C87809110
:10B24000D5118D878091D6118E878091D7118F87E8
:10B2500081E090E0998B888B809172228B8780911E
:10B2600071228A8780917022898780916F228887D6
:10B2700081E090E00E9428558091772290E0807FC5
:10B280009070813591050CF449C01092DA1134C0E8
:10B29000F901E95AFD4D80A58093DB118823F1F176
:10B2A000813021F44F5F4093DA1126C08230C1F41F
:10B2B00081A58430A9F432A520E083A590E0822BFB
:10B2C000932B9093DD118093DC11F4E0893D9F076F
:10B2D00010F088ED94E09B8B8A8B9D8B8C8B1EC02D
:10B2E0009091DA11E92FF0E0E95AFD4D81A588230C
:10B2F000A9F0890F8093DA114091DA11242F30E000
:10B300008091772282958F7090E00597880F991F22
:10B31000880F991F281739070CF4BACF80E1809362
:10B3200078228091782282608093782282E08093D4
:10B330007F2284E0809380228093812288ED809315
:10B3400082228CE290E09093502280934F2280E6FC
:10B35000CBC2D0935D27C0935C2710925727809172
:10B360007822282F30E082FF03C0198E80E265C268
:10B370008091772282958F70880F880F8093DA11E1
:10B3800040914F225091502244515040481B510946
:10B390005093502240934F22898D90E08F7090708F
:10B3A0008230910531F42F7330702231310541F430
:10B3B00028C0019729F42F7330702230310509F12C
:10B3C000452B39F48091782290E083709070892B1E
:10B3D000C1F090916F228885981709F07BC29091F7
:10B3E00070228985981709F075C2909171228A851B
:10B3F000981709F06FC2909172228B85981709F007
:10B4000069C28091782284FF51C068897989611569
:10B41000710509F44BC0CE010C960E945453209143
:10B42000732280915322281709F040C09091742212
:10B43000809154229817D1F59091752280915522D0
:10B440009817A1F59091762280915622981771F560
:10B450002C87809154228D87809155228E878091F0
:10B4600056228F878B8D8823D1F42E89988D8A8DD3
:10B47000981B822F869586958695981B392F320FBB
:10B480003E8B8F89282F26952695821B97FD9195B7
:10B49000890F8F8B369536953695830F888F81E08F
:10B4A00080935727888D8A8F198A188A898D282F2B
:10B4B00030E0C9018F7090708430910509F4C2C1E9
:10B4C000853091055CF482309105D9F18330910586
:10B4D0000CF0BAC0019709F098C210C086309105EF
:10B4E00009F4F0C1863091050CF4CCC18730910588
:10B4F00009F4F0C1089709F088C299C180915727D3
:10B5000080FF18C083E0898F80E480935727198AD1
:10B51000188A20914F22309150222115310509F4CB
:10B520001AC180915727826080935727C9010E94D2
:10B53000285511C1809178228F73823009F065C23D
:10B54000EDCE8091572780FF74C0809178228F7351
:10B55000823109F06EC08091772290E0807F9070F8
:10B56000813591050CF449C01092DA1134C0F9010B
:10B57000E95AFD4D80A58093DB118823F1F18130DC
:10B5800021F44F5F4093DA1126C08230C1F481A5C7
:10B590008430A9F432A520E083A590E0822B932B80
:10B5A0009093DD118093DC1124E0893D920710F027
:10B5B00088ED94E09B8B8A8B9D8B8C8B1EC0909129
:10B5C000DA11E92FF0E0E95AFD4D81A58823A9F0B1
:10B5D000890F8093DA114091DA11242F30E08091A5
:10B5E000772282958F7090E00597880F991F880FBA
:10B5F000991F281739070CF4BACF83E0898F8091FF
:10B600006F228887809170228987809171228A8732
:10B61000809172228B8781E090E00E94285582E41D
:10B6200080935727198A188A1092502210924F221D
:10B6300092C080E2809357270E94FE4EE0915C27E3
:10B64000F0915D27118E3BCD8091782280FF2AC03A
:10B6500024FD28C088899989892B09F0D6C1809159
:10B660004F229091502201960E94285520915727F1
:10B67000822F80618093572780914F229091502292
:10B68000892B19F02261209357270E94FE4E81E0FA
:10B6900090E0998B888B88E0898F1B8E81E1809365
:10B6A00078221BC185FF21C060917D22362F20E0CA
:10B6B00040917E2250E0242B352B80915A27909187
:10B6C0005B27820F931F90935B2780935A27962FB7
:10B6D00080E0842B952B20914F2230915022281B03
:10B6E000390B3093502220934F2220914F223091DA
:10B6F00050222115310559F0898D84FD08C08091B3
:10B700005727826080935727C9010E94285590913E
:10B71000792280E020917A22820F911D9093DD1191
:10B720008093DC112C893D892817390710F0892B6B
:10B7300021F43093DD112093DC118091DC11909184
:10B74000DD119B8B8A8B8091572790E083709070DE
:10B75000892B09F45AC11092F3271092F2270E9404
:10B76000FE4E80915727282F85FF07C01092F327A0
:10B770001092F227198E84E192CF84FF0AC01092B2
:10B78000F3271092F22781E090E0998B888B84E078
:10B7900083CF8091F2279091F327892B01F120FF2D
:10B7A00002C0198A188A888999890097A1F42A8980
:10B7B0003B898091F2279091F3272817390720F4CD
:10B7C0003093F3272093F2278091F2279091F3276B
:10B7D000998B888B04C09093F3278093F2271B8E5C
:10B7E000809151229091522290935B2780935A2707
:10B7F0008091F2279091F327892B59F088899989B4
:10B80000009739F088969093502280934F2288E1D8
:10B810000BC08091572781FFF8C088E290E0909399
:10B82000502280934F2280E1809378225CC08091E7
:10B83000572780FFEAC0198E80E1809357270E9426
:10B84000FE4EE3C080914F2290915022009711F05C
:10B850000E942855809178229091572780FF0BC035
:10B8600090FF06C087E0898F1A8E198A188A19C03E
:10B8700086E0898F16C090FF1EC085E0898F198AE7
:10B88000188AC3C080914F2290915022009711F0E6
:10B890000E9428558091782280FF0DC087E0898F13
:10B8A0001A8E81E090E00E94285580E1809357270E
:10B8B0000E94FE4E0FC080914F2290915022892B02
:10B8C00049F4A3C08091572780FF9FC087E0898FEC
:10B8D0001A8E9BC080E1F80181A388E290E09093EA
:10B8E000502280934F2280E5809377228885809331
:10B8F00073228985809374228A85809375228B8533
:10B90000809376228C8580936F228D858093702220
:10B910008E85809371228F858093722286E080933A
:10B9200060228C819D8190936C2280936B228E810A
:10B930009F8190936E2280936D228091EE2790914B
:10B94000EF27A091F027B091F12780936322909385
:10B950006422A0936522B093662288819981AA818E
:10B96000BB818093672290936822A0936922B09351
:10B970006A22898D84FF05C010927A221092792262
:10B9800006C084E08093792288ED80937A2280E457
:10B9900080935F22809150228093592280914F2280
:10B9A00080935A2210927E2210927D2210927C2245
:10B9B00010927B220E9423548095909590937C2234
:10B9C00080937B2285E48093572210925822109214
:10B9D0005E2210925D228091D2119091D311019636
:10B9E0009093D3118093D21190935B2280935C2229
:10B9F00010926222109261220E94B4538095909519
:10BA0000909362228093612204C01092502210927F
:10BA10004F2210925727DF91CF911F910F910895D8
:10BA20000F931F93CF93DF93DC018B012091D811EB
:10BA30003091D911CDE0D0E02F5F3F4F8DE720301E
:10BA4000380710F020E030E1522F432F60E011C0A2
:10BA5000862F90E08C9FF0018D9FF00D9C9FF00D44
:10BA60001124EC50F84D848195816F5F8417950700
:10BA700019F36A3069F72093D8113093D9111092D5
:10BA8000DA1140E06DE070E01CC0542F5F5F842F3E
:10BA900090E0869FF001879FF00D969FF00D112496
:10BAA000EC50F84D84819581892B51F44093DA1143
:10BAB0008DE0489FF0011124EC50F84D49F41EC070
:10BAC000452F4A3010F34093DA11E0E0F0E016C061
:10BAD0003483258317830683109729F410821182FB
:10BAE0001282138209C08D919D910D90BC91A02D61
:10BAF00080839183A283B38380E48087CF01DF9129
:10BB0000CF911F910F910895EF92FF920F93DF93C2
:10BB1000CF93CDB7DEB760970FB6F894DEBF0FBEF8
:10BB2000CDBFA82F002309F461C07E010894E11C59
:10BB3000F11C88E0F70111928A95E9F729833A838D
:10BB40004B835C836D837E83AF83988780E2801B09
:10BB5000E82FFF27E7FDF09549815A816B817C81B1
:10BB6000181684F019861A861B861C868827992742
:10BB70008E1B9F0B04C0440F551F661F771F8A95AD
:10BB8000D2F728C0202F332727FD3095DB01CA01CB
:10BB9000022E04C0880F991FAA1FBB1F0A94D2F758
:10BBA00089879A87AB87BC8704C076956795579538
:10BBB0004795EA95D2F78D819E81AF81B88504C003
:10BBC000880F991FAA1FBB1F2A95D2F7482B592B04
:10BBD0006A2B7B2B4D875E876F87788B29853A850B
:10BBE0004B855C856D857E85AF8598898A2F6096AB
:10BBF0000FB6F894DEBF0FBECDBFCF91DF910F918E
:10BC0000FF90EF900895A0E1B0E0E9E0FEE50C942C
:10BC10005C64A8E04E010894811C911CF401BA2FC9
:10BC20001192BA95E9F729833A834B835C836D833C
:10BC30007E838F839887CE010996FC011192AA9585
:10BC4000E9F7A986BA86CB86DC86ED86FE860F8765
:10BC5000188B2D813E814F8158858D859E85AF85BE
:10BC6000B889281739074A075B07C8F08217930776
:10BC7000A407B507B0F029813A814B815C818985A1
:10BC80009A85AB85BC85281739074A075B0738F0CA
:10BC900082179307A407B50720F081E003C080E076
:10BCA00001C082E06096ECE00C9478642F923F92A1
:10BCB0004F925F926F927F928F929F92AF92BF92BC
:10BCC000CF92DF92EF92FF920F931F93DF93CF9368
:10BCD000CDB7DEB761970FB6F894DEBF0FBECDBF0C
:10BCE0003C017F876E876A01FC011782168283817F
:10BCF00081FD03C06FEF7FEF71C39E012F5F3F4F48
:10BD0000398B288BF3012381EE85FF8523FD8591F7
:10BD100023FF8191FF87EE87882309F45CC3853276
:10BD200051F4EE85FF8523FD859123FF8191FF87E7
:10BD3000EE87853229F490E0B3010E947E67E2CF5E
:10BD4000982F10E0882499241032B0F49B3269F0C7
:10BD50009C3228F4903251F0933271F40BC09D3232
:10BD600039F0903349F4116028C01260146025C086
:10BD7000186023C0106121C017FD2AC0892F80538D
:10BD80008A3078F416FF06C0FAE09F9E902C1124AA
:10BD9000980E13C03AE0839E802C1124880E106206
:10BDA0000CC09E3221F416FD16C3106406C09C36EA
:10BDB00011F4106802C0983659F4EE85FF8523FD12
:10BDC000959123FF9191FF87EE87992309F0BCCFCE
:10BDD000892F8554833020F4812F8061905E07C0C5
:10BDE000892F8556833008F0A1C1812F8F7E86FD73
:10BDF00002C076E0972E6FE3F62EF822953619F4FE
:10BE0000F0E4FF2A07C0963619F420E8F22A02C0AF
:10BE100091109A94F7FE0BC03BE3391520F427E00C
:10BE20005CE3B52E0EC0B92CB39427E00AC047E0FE
:10BE3000491528F427E0BB2447E0942E02C0292DA1
:10BE4000BB24C60104969D878C87F60160817181B1
:10BE500082819381AE014F5F5F4F0B2D0E94306650
:10BE60006C010981202E332400FF04C003FD02C0B1
:10BE70001DE209C0F1FE02C01BE205C0F2FC02C0D7
:10BE800010E001C010E2C1018C709070892BB9F1F3
:10BE9000112311F483E001C084E0881510F0882498
:10BEA0000AC0881AF3FC07C080E290E0B3010E9448
:10BEB0007E678A94C9F7112329F0812F90E0B3019E
:10BEC0000E947E6723FE03C001E71BE00EC005E76A
:10BED0001BE00BC0E114F10409F0805290E0B301C3
:10BEE0000E947E670F5F1F4F05C0EF2CFF24F0E11B
:10BEF000EF22FF24F8018491882361F714C1F7FE33
:10BF000012C0BC0C24FE04C08A81813309F4BA94A7
:10BF10001B141CF0BB24B3942DC0F8E0FB1550F5A6
:10BF200038E0B32E27C0F6FC25C0892D90E08C1593
:10BF30009D054CF02CEFC2162FEFD20624F030E80E
:10BF4000F32A01C09A94992049F0E2E0F0E0EC0F66
:10BF5000FD1FE90DF11D80818033A1F3F7FE0AC0BA
:10BF6000B92CB394892D90E0C816D90614F0992401
:10BF700001C09C18F7FC03C025E030E009C01C1488
:10BF80001D041CF021E030E003C096012F5F3F4FFD
:10BF9000112311F02F5F3F4F992029F0892D90E058
:10BFA0000196280F391F882D90E02817390714F0C3
:10BFB000882401C0821A4F2C5524C20189709070C8
:10BFC000892B39F008C080E290E0B3010E947E67BF
:10BFD0008A948820C1F7112329F0812F90E0B301C2
:10BFE0000E947E6743FE07C008C080E390E0B30173
:10BFF0000E947E678A948820C1F7F7FE46C08601BA
:10C00000D7FE02C000E010E076010894E11CF11CAC
:10C01000E01AF10A41E050E04C0F5D1FE40EF51EFE
:10C0200026014B185108892D90E0AA24BB24A81A98
:10C03000B90A5FEF0F3F150729F48EE290E0B301D4
:10C040000E947E67C016D10634F0401651061CF4DB
:10C05000F701808101C080E3015010400894E11C89
:10C06000F11C0A151B052CF090E0B3010E947E67BD
:10C07000E0CF0C151D0539F49A81963318F49533E9
:10C0800011F424FE81E390E04BC08A81813309F0F2
:10C090000F7E90E0B3010E947E679920A1F08EE2AE
:10C0A00090E0B3010E947E6712E0E1E0F0E0EC0F67
:10C0B000FD1FE10FF11D1F5F808190E0B3010E9421
:10C0C0007E679A9491F744FC03C085E690E002C035
:10C0D00085E490E0B3010E947E67D7FC05C0C114DF
:10C0E000D10441F404FF06C0D094C194D108D39484
:10C0F0008DE201C08BE290E0B3010E947E6780E395
:10C1000005C08F5F26EF3FEFC20ED31E3AE0C31685
:10C11000D104BCF790E0B3010E947E67C601C096CF
:10C12000B3010E947E67CC84DD8452C1933631F026
:10C13000933799F0933509F059C023C0F6018081F7
:10C1400089835E010894A11CB11C22E030E0C20E7C
:10C15000D31E21E0E22EF12C12C0F601A080B180A6
:10C1600016FD03C06FEF7FEF02C0692D70E022E083
:10C1700030E0C20ED31EC5010E9439677C011F77D3
:10C1800013C0F601A080B18016FD03C06FEF7FEFF2
:10C1900002C0692D70E022E030E0C20ED31EC5015E
:10C1A0000E9410677C01106813FF07C01BC080E26B
:10C1B00090E0B3010E947E678A94882D90E0E81693
:10C1C000F906A8F30FC0F50117FD859117FF8191BE
:10C1D0005F0190E0B3010E947E6781108A94089409
:10C1E000E108F108E114F10471F7F2C0943611F09E
:10C1F000993689F517FF08C0F60120813181428107
:10C20000538184E090E00AC0F601808191819C0115
:10C21000442737FD4095542F82E090E0C80ED91E88
:10C220009FE6F92EF12257FF09C0509540953095B1
:10C2300021953F4F4F4F5F4F90E8F92ACA01B9014E
:10C24000AE014F5F5F4F2AE030E00E949068E82E19
:10C25000E889EE1A41C0953721F41F7E2AE030E0CC
:10C260001CC0197F9F3661F0903720F4983509F093
:10C27000B2C00FC0903739F0983709F0ACC004C095
:10C2800028E030E00AC0106114FD146020E130E0C5
:10C2900004C014FD166020E132E017FF08C0F6016B
:10C2A000608171818281938144E050E008C0F60191
:10C2B00080819181BC0180E090E042E050E0C40EBA
:10C2C000D51EAE014F5F5F4F0E949068E82E5889DF
:10C2D000E51A8FE7F82EF122F6FE0BC08EEFF8225A
:10C2E000E91438F4F4FE07C0F2FC05C09FEEF92211
:10C2F00002C01E2D01C0192DF4FE0DC0FE01EE0D71
:10C30000F11D8081803319F4E9EEFE2208C01F5F21
:10C31000F2FE05C003C08F2D867809F01F5F0F2D38
:10C32000F3FC14C0F0FE0FC0181510F09E2C0BC0CB
:10C330009E2C980C911A182D06C080E290E0B30153
:10C340000E947E671F5F1815C0F304C0181510F413
:10C35000811A01C0882404FF0FC080E390E0B3017C
:10C360000E947E6702FF1DC001FD03C088E790E0C8
:10C370000EC088E590E00BC0802F867891F001FF19
:10C3800002C08BE201C080E2F7FC8DE290E0B301D5
:10C390000E947E6706C080E390E0B3010E947E6742
:10C3A0009A94E914C0F3EA94E1E0F0E0EC0FFD1F89
:10C3B000EE0DF11D808190E0B3010E947E67EE20BA
:10C3C00091F706C080E290E0B3010E947E678A94F4
:10C3D0008820C1F797CCF30166817781CB01619604
:10C3E0000FB6F894DEBF0FBECDBFCF91DF911F9186
:10C3F0000F91FF90EF90DF90CF90BF90AF909F9004
:10C400008F907F906F905F904F903F902F90089506
:10C410005058BB27AA270ED044C135D130F03AD1AD
:10C4200020F031F49F3F11F41EF42AC10EF4E09580
:10C43000E7FB20C1E92F46D180F3BA1762077307E3
:10C440008407950718F071F49EF55EC10EF4E0952F
:10C450000B2EBA2FA02D0B01B90190010C01CA01BE
:10C46000A0011124FF27591B99F0593F50F4503E69
:10C4700068F11A16F040A22F232F342F4427585F5B
:10C48000F3CF469537952795A795F0405395C9F773
:10C490007EF41F16BA0B620B730B840BBAF091502B
:10C4A000A1F0FF0FBB1F661F771F881FC2F70EC0CA
:10C4B000BA0F621F731F841F48F48795779567959D
:10C4C000B795F7959E3F08F0B3CF9395880F08F086
:10C4D0009927EE0F979587950895A8D008F481E0E5
:10C4E00008950CD0DEC0D6D040F0CDD030F021F48D
:10C4F0005F3F19F0BFC0511108C1C2C0E3D098F32B
:10C500009923C9F35523B1F3951B550BBB27AA27D4
:10C5100062177307840738F09F5F5F4F220F331F46
:10C52000441FAA1FA9F333D00E2E3AF0E0E830D012
:10C5300091505040E695001CCAF729D0FE2F27D015
:10C54000660F771F881FBB1F261737074807AB07E3
:10C55000B0E809F0BB0B802DBF01FF2793585F4F58
:10C560002AF09E3F510568F085C0CFC05F3FECF3D5
:10C57000983EDCF3869577956795B795F7959F5F1D
:10C58000C9F7880F911D9695879597F90895E1E071
:10C59000660F771F881FBB1F621773078407BA07D0
:10C5A00020F0621B730B840BBA0BEE1F88F7E0952B
:10C5B0000895E89409C097FB3EF490958095709596
:10C5C00061957F4F8F4F9F4F9923A9F0F92F96E9DF
:10C5D000BB279395F695879577956795B795F11154
:10C5E000F8CFFAF4BB0F11F460FF1BC06F5F7F4FF1
:10C5F0008F4F9F4F16C0882311F096E911C0772303
:10C6000021F09EE8872F762F05C0662371F096E80B
:10C61000862F70E060E02AF09A95660F771F881FDA
:10C62000DAF7880F9695879597F90895990F00087E
:10C63000550FAA0BE0E8FEEF16161706E807F907F4
:10C64000C0F012161306E407F50798F0621B730B8F
:10C65000840B950B39F40A2661F0232B242B252B10
:10C6600021F408950A2609F4A140A6958FEF811DB3
:10C67000811D089597F99F6780E870E060E0089554
:10C680009FEF80EC089500240A94161617061806EA
:10C690000906089500240A941216130614060506C6
:10C6A0000895092E0394000C11F4882352F0BB0F57
:10C6B00040F4BF2B11F460FF04C06F5F7F4F8F4FBA
:10C6C0009F4F089557FD9058440F551F59F05F3FF5
:10C6D00071F04795880F97FB991F61F09F3F79F0A4
:10C6E00087950895121613061406551FF2CF469526
:10C6F000F1DF08C0161617061806991FF1CF8695A8
:10C700007105610508940895E894BB27662777278B
:10C71000CB0197F908950BD0C4CFB5DF28F0BADF6D
:10C7200018F0952309F0A6CFABCF1124EECFCADFC6
:10C73000A0F3959FD1F3950F50E0551F629FF00134
:10C74000729FBB27F00DB11D639FAA27F00DB11D8D
:10C75000AA1F649F6627B00DA11D661F829F222716
:10C76000B00DA11D621F739FB00DA11D621F839F9D
:10C77000A00D611D221F749F3327A00D611D231F73
:10C78000849F600D211D822F762F6A2F11249F57C1
:10C7900050408AF0E1F088234AF0EE0FFF1FBB1FE4
:10C7A000661F771F881F91505040A9F79E3F510583
:10C7B00070F060CFAACF5F3FECF3983EDCF3869534
:10C7C00077956795B795F795E7959F5FC1F7FE2B2E
:10C7D000880F911D9695879597F90895629FD001CE
:10C7E000739FF001829FE00DF11D649FE00DF11D2C
:10C7F000929FF00D839FF00D749FF00D659FF00DDB
:10C800009927729FB00DE11DF91F639FB00DE11DC7
:10C81000F91FBD01CF0111240895AA1BBB1B51E1D3
:10C8200007C0AA1FBB1FA617B70710F0A61BB70BA0
:10C83000881F991F5A95A9F780959095BC01CD0145
:10C84000089597FB092E07260AD077FD04D0E5DF6F
:10C8500006D000201AF4709561957F4F0895F6F781
:10C86000909581959F4F0895A1E21A2EAA1BBB1B9C
:10C87000FD010DC0AA1FBB1FEE1FFF1FA217B307AC
:10C88000E407F50720F0A21BB30BE40BF50B661FC2
:10C89000771F881F991F1A9469F760957095809586
:10C8A00090959B01AC01BD01CF0108952F923F925D
:10C8B0004F925F926F927F928F929F92AF92BF92B0
:10C8C000CF92DF92EF92FF920F931F93CF93DF935C
:10C8D000CDB7DEB7CA1BDB0B0FB6F894DEBF0FBEB9
:10C8E000CDBF09942A88398848885F846E847D8406
:10C8F0008C849B84AA84B984C884DF80EE80FD8008
:10C900000C811B81AA81B981CE0FD11D0FB6F8947D
:10C91000DEBF0FBECDBFED010895AF92BF92CF92A3
:10C92000DF92EF92FF920F931F93CF93DF93EC016F
:10C93000A880B980CA80DB80A114B104C104D104ED
:10C9400041F484E2A82E89EDB82E8BE5C82E87E04D
:10C95000D82EC601B5012DE133EF41E050E00E9431
:10C96000B26A27EA31E440E050E00E94EE637B01C6
:10C970008C01C601B5012DE133EF41E050E00E948A
:10C98000B26ACA01B9012CEE34EF4FEF5FEF0E949B
:10C99000EE636E0D7F1D801F911F97FF04C06150D5
:10C9A000704080409048688379838A839B839B0191
:10C9B0003F77C901DF91CF911F910F91FF90EF90C9
:10C9C000DF90CF90BF90AF9008950E948D6408953E
:10C9D0008FEC95E00E948D640895A0E0B0E0809314
:10C9E000CF059093D005A093D105B093D2050895BB
:10C9F0003F924F925F926F927F928F929F92AF92EF
:10CA0000BF92CF92DF92EF92FF920F931F93CF933B
:10CA1000DF93EC012B016A016115710519F0FB012F
:10CA200091838083C114D10449F0C6010297839792
:10CA300028F020E030E040E050E0DCC0A9908A2DF2
:10CA400090E00E940867892BC9F7FDE2AF1621F438
:10CA5000A9903324339405C08BE2A81609F4A99059
:10CA60003324C114D10421F0E0E1CE16D10411F534
:10CA7000F0E3AF1669F48881883711F0883541F406
:10CA8000A980229682E0382A20E1C22ED12C12C041
:10CA9000C114D10479F4E0E3AE1659F199E9E92E15
:10CAA00099E9F92E99E9092F99E1192F8AE0C82E01
:10CAB000D12C3AC0FAE0CF16D10491F080E1C8162B
:10CAC000D10429F0E8E0CE16D104F9F415C0BFEF87
:10CAD000EB2EBFEFFB2EBFEF0B2FBFE01B2F24C0B1
:10CAE000A9E9EA2EA9E9FA2EA9E90A2FA9E11A2F44
:10CAF0001BC0F8E0CF2ED12CEFEFEE2EEFEFFE2E85
:10CB0000EFEF0E2FEFE11E2F0FC09601442737FDE8
:10CB10004095542F6FEF7FEF8FEF9FEF0E943464AB
:10CB2000C901DA017C018D0120E030E040E050E0F5
:10CB300060E03601882477FC8094982C70EDB72E45
:10CB4000BA0CF9E0FB1570F48A2D81548A3118F47F
:10CB500099ECB92E06C08A2D81568A3148F589EAAA
:10CB6000B82EBA0C8B2D90E08C159D050CF56F3FFF
:10CB7000E9F0E216F30604071507B8F0CA01B90197
:10CB8000A40193010E94EE639B01AC018B2D90E008
:10CB9000A0E0B0E0280F391F4A1F5B1F2817390794
:10CBA0004A075B0710F061E001C06FEFA990C6CFA4
:10CBB0004114510451F0662311F0219703C031FE56
:10CBC00004C02297F201D183C08330FE07C0509584
:10CBD0004095309521953F4F4F4F5F4F67FF0AC0FB
:10CBE00082E290E090937D2880937C282FEF3FEFA6
:10CBF0004FEF5FEFB901CA01DF91CF911F910F9104
:10CC0000FF90EF90DF90CF90BF90AF909F908F906C
:10CC10007F906F905F904F903F90089566277727A1
:10CC20000C942969FC0188279927E89421912032E6
:10CC3000E9F3293010F02E30C8F32B3241F02D32B9
:10CC400039F4689404C00E947667820F911D219187
:10CC500020532A30C0F31EF4909581959F4F08957C
:10CC6000283008F027E03327DA01990F311D87FDBE
:10CC7000916000966105710539F432602E5F3D9335
:10CC800030E32A95E1F708959F3F30F08038710531
:10CC9000610509F03C5F3C5F3D93913008F080688E
:10CCA000911DDF93CF931F930F93FF92EF92192F54
:10CCB000987F9695E92F96959695E90FFF27ED5267
:10CCC000F44F99273327EE24FF24A701E7010590AD
:10CCD0000894079428F4360FE71EF81E491F511DCB
:10CCE000660F771F881F991F0694A1F70590079478
:10CCF00028F4E70EF81E491F561FC11D770F881F25
:10CD0000991F661F0694A1F70590079428F4F80E62
:10CD1000491F561FC71FD11D880F991F661F771FF8
:10CD20000694A1F70590079420F4490F561FC71FDA
:10CD3000D81F990F661F771F881F0694A9F7849143
:10CD40001095177041F0D695C79557954795F7946C
:10CD5000E7941A95C1F7E9E7FBE0689415901591FF
:10CD600035916591959105907FE27395E118F10AEF
:10CD7000430B560BC90BD009C0F7E10CF11E431F42
:10CD8000561FC91FD01D7EF4703311F48A95E6CF6B
:10CD9000E894015030F0080F0AF40027021708F455
:10CDA000202F2395022F7A3328F079E37D932A955B
:10CDB000E9F710C07D932A9589F6069497956795B3
:10CDC000379517951794E118F10A430B560BC90BC9
:10CDD000D00998F023957E9173957A3308F070E32B
:10CDE0007C932013B8F77E9170617D9330F083952A
:10CDF00071E37D9370E32A95E1F71124EF90FF90A2
:10CE00000F911F91CF91DF91992787FD90950895FC
:10CE100091118DC3803219F089508550D0F7089553
:10CE2000FC010590615070400110D8F780959095F5
:10CE30008E0F9F1F08954EED51E10E9444670895A3
:10CE4000FB01DC0102C001900D9241505040D8F727
:10CE50000895DC0101C06D9341505040E0F7089502
:10CE6000FB01DC018D91019080190110D9F3990B20
:10CE70000895FC016150704001900110D8F7809531
:10CE800090958E0F9F1F0895009731F4DA018D91D0
:10CE90009C91009709F40EC0DC01FB013D912191AA
:10CEA000222319F03217C9F3FACF332331F4DA0110
:10CEB0001D921C928827992708951197AF93BF93CD
:10CEC000FB013D912191321771F4332321F488271E
:10CED0009927119702C01E921196FA01A193B0836F
:10CEE0009F918F910895222369F7EACF7AE0979F67
:10CEF000902D879F802D910D112408950F931F93DE
:10CF0000CF93DF938C01EB018B8181FF1BC082FFEC
:10CF10000DC02E813F818C819D812817390764F4D3
:10CF2000E881F9810193F983E88306C0E885F985F2
:10CF3000802F0995892B31F48E819F8101969F83E3
:10CF40008E8302C00FEF1FEFC801DF91CF911F91B9
:10CF50000F910895DF93CF93CDB7DEB7FE013596DD
:10CF6000619171918091782890917928AF010E9408
:10CF7000565ECF91DF910895DF93CF93CDB7DEB7A3
:10CF8000FE01359661917191A0917828B091792830
:10CF900013968C911397886013968C9380917828C0
:10CFA00090917928AF010E94565EE0917828F09127
:10CFB00079282381277F2383CF91DF910895609182
:10CFC0007828709179280E947E6708950F931F93A7
:10CFD000CF93DF938C01E0917828F09179288381B9
:10CFE00081FF21C0C0E0D0E00DC0E0917828F09131
:10CFF000792820853185BF01F9010995892B11F028
:10D00000CFEFDFEFF80181918F01882371F7E09175
:10D010007828F0917928208531858AE0BF01F901CF
:10D020000995892B11F0CFEFDFEFCE01DF91CF9182
:10D030001F910F9108950F931F93DF93CF93CDB757
:10D04000DEB72E970FB6F894DEBF0FBECDBF0D89A9
:10D050001E898F89988D97FF02C080E090E8019724
:10D060009E838D831A83098386E08C839E01255ECF
:10D070003F4FCE010196698D7A8DA9010E94565EBF
:10D080004D815E8157FD0AC02F81388542175307B5
:10D090000CF49A01020F131FF80110822E960FB69E
:10D0A000F894DEBF0FBECDBFCF91DF911F910F91DE
:10D0B00008950F931F93DF93CF93CDB7DEB72E97CD
:10D0C0000FB6F894DEBF0FBECDBF8C0177FF02C054
:10D0D00060E070E8615070407E836D831A8309833D
:10D0E00086E08C83CE010196BA01A9010E94565EAA
:10D0F0002D813E8137FD09C0EF81F8852E173F074E
:10D100000CF4F901E00FF11F10822E960FB6F8947F
:10D11000DEBF0FBECDBFCF91DF911F910F9108955C
:10D12000FA01AA27283051F1203181F1E8946F9358
:10D130006E7F6E5F7F4F8F4F9F4FAF4FB1E03ED0FE
:10D14000B4E03CD0670F781F891F9A1FA11D680F9C
:10D15000791F8A1F911DA11D6A0F711D811D911DCF
:10D16000A11D20D009F468943F912AE0269F112444
:10D170003019305D3193DEF6CF010895462F4770A8
:10D18000405D4193B3E00FD0C9F7F6CF462F4F7003
:10D19000405D4A3318F0495D31FD4052419302D061
:10D1A000A9F7EACFB4E0A695979587957795679507
:10D1B000BA95C9F700976105710508959B01AC0107
:10D1C0000A2E06945795479537952795BA95C9F72E
:10D1D000620F731F841F951FA01D0895DC01CB01F2
:10D1E000FC01F999FECF06C0F2BDE1BDF89A319677
:10D1F00000B40D9241505040B8F70895F999FECF10
:10D2000092BD81BDF89A992780B50895A8E1B0E054
:10D2100042E050E00C94F068DC01CB0103C02D919A
:10D220000E94176941505040D0F70895262FF99970
:10D23000FECF1FBA92BD81BD20BD0FB6F894FA9AF9
:10D24000F99A0FBE019608950E941669272F0C9433
:10D2500017698F929F92AF92BF92CF92DF92EF9217
:10D26000FF920F931F93CF93DF93EC015B01611546
:10D27000710519F0FB0191838083F9908F2D90E067
:10D280000E940867892BC9F7FDE2FF1621F4F99087
:10D29000EE24E39405C02BE2F21609F4F990EE2493
:10D2A0008E0101501040C80163E77CE043E050E08C
:10D2B0000E949A6A892B01F58E010E5F1F4FC801EB
:10D2C00066E77CE045E050E00E949A6A892B19F4F9
:10D2D0008E01095F1F4FA114B10419F0F5011183EC
:10D2E0000083E0FC04C070E090E080E814C070E0CF
:10D2F00090E080E86FEF08C1C8016BE77CE043E095
:10D3000050E00E949A6A892B69F4A114B10429F4AF
:10D3100070E090E080EC6FE7F7C02296F501D183D2
:10D32000C083F6CF8824992440E050E060E070E0AC
:10D33000EF2DE053EA30A0F5F2E0EF2A8E2D90E0D9
:10D340009C0128703070E2FE06C0232B79F508940A
:10D35000811C911C2BC0232B19F008948108910883
:10D36000DB01CA0112E0880F991FAA1FBB1F1A9583
:10D37000D1F7480F591F6A1F7B1F440F551F661FA7
:10D38000771F4E0F511D611D711D483929E9520744
:10D3900029E9620729E1720748F084E0E82A06C01B
:10D3A000EE3F31F4E3FC39C098E0E92AF990C0CFB0
:10D3B000E53311F0E53189F529912D3219F4E0E1D9
:10D3C000EE2A05C02B3219F081E090E003C02991CC
:10D3D00082E090E0E22FE053EA3018F0C81BD90B4E
:10D3E0001CC020E030E0FCE020383F075CF4C901BD
:10D3F000880F991F880F991F280F391F220F331F7D
:10D400002E0F311DE991E053EA3068F3E4FE03C0CA
:10D41000309521953F4F820E931ECE2CDD24E1FEE8
:10D4200007C0A114B10421F02197F501D183C08375
:10D43000CB01BA010E94D9627B018C01F3E0CF22BB
:10D44000DD2423E0C216D10421F417FB109517F94F
:10D45000109557016801C801B70120E030E040E0B5
:10D4600050E00E946D62882309F44AC097FE0DC007
:10D4700022E9E22E2CE0F22E90948194910893946C
:10D48000C0E2D0E000E010E012C09AEAE92E9CE091
:10D49000F92EF6CFF7012591359145915491C601AA
:10D4A000B5010E948B635B016C018C1A9D0A8C167E
:10D4B0009D0684F7D595C7950F5F1F4F0630110560
:10D4C00029F08CEF9FEFE80EF91EF1CFC501D601D0
:10D4D0007C018D018C2D880F8D2D881F8F3F51F081
:10D4E000C601B50120E030E040E050E00E946D62EE
:10D4F000882331F482E290E090937D2880937C2809
:10D500007E2D9F2D802F612F272F392F482F562FAB
:10D51000B901CA01DF91CF911F910F91FF90EF9058
:10D52000DF90CF90BF90AF909F908F9008959927F4
:10D5300088270895FB01DC014150504088F08D910F
:10D5400081341CF08B350CF4805E659161341CF0E5
:10D550006B350CF4605E861B611171F3990B0895B5
:10D56000881BFCCF97FB092E05260ED057FD04D053
:10D570007BD90AD0001C38F4509540953095219500
:10D580003F4F4F4F5F4F0895F6F7909580957095F8
:0ED5900061957F4F8F4F9F4F0895F894FFCF06
:10D59E005363686564756C6564206576656E74208A
:10D5AE006E6F773D256C64206E6578743D256C64D6
:10D5BE000D0A005363686564756C65642065766555
:10D5CE006E74206174203D256C642066756E633D1B
:10D5DE0025780D0A00263A202573205B41444452DB
:10D5EE003D252D642E252D64205345513D252D645A
:10D5FE0020525353493D252D75204C51493D252D23
:10D60E0075204452503D252D642E253032645D0A1E
:10D61E0000656570726F6D007374617475733D3063
:10D62E0078253032780A200049443D002530327882
:10D63E00002050533D25640020543D252D362E32BA
:10D64E0066002054313D252D362E32660020545F63
:10D65E004D43553D252D352E31660020565F4D43E9
:10D66E00553D252D342E3266002050303D252D6C33
:10D67E0058002050305F543D252D372E3366002044
:10D68E0055503D252D6C58002052483D252D342EE9
:10D69E0031660020565F494E3D252D352E326600EF
:10D6AE0020565F41313D252D352E32660020565FC6
:10D6BE0041323D252D352E326600263A2025730A3D
:10D6CE000025303258006C656E3D25640A00002836
:10D6DE004578745077722900312E30204669726D6C
:10D6EE0077617265205665722E20322E35203230CB
:10D6FE0031322D30362D3231006F6E006F6666007E
:10D70E00613100726573657400613200765F696E17
:10D71E00006175746F00666C757368004144445205
:10D72E003D252D642E252D64205345513D252D6418
:10D73E0020525353493D252D75204C51493D252DE1
:10D74E00750A004F6E007472696D0043683D252D99
:10D75E00642054785077723D252D640A000100ED47
:10D76E00478A3C22FFCC3B22FFCC3B1A20090D00FE
:10D77E00DC036162636465666768696A6B6C6D6E13
:10D78E006F708F023C000200636D642070726F63D5
:10D79E00657373000000F803082800000000666F30
:10D7AE006F2070726F636573730000000E049E0E1F
:10D7BE0000000000737464696E2070726F6365738D
:10D7CE00730000002404B80D0000000062726F6147
:10D7DE0064636173742070726F636573730000000D
:10D7EE003C04851200000000536C65657020707259
:10D7FE006F636573730000005804CC0800000000CE
:10D80E0004041A0432044E0466040000980C00004E
:10D81E000D0040000A064A0610000000F828BF2836
:10D82E001810000000004576656E742074696D65F1
:10D83E00720000009604D62D00000000A509020318
:10D84E0006070A0B0E0F020306070A0B0E0F436F95
:10D85E006E74696B6920322E3500000000020000E4
:10D86E0000008C3A00000000C600C500C400C100D4
:10D87E00C200000000CE00CD00CC00C900CA0000DE
:10D88E0000005246323330206472697665720000B1
:10D89E0000F204C24000000000FB40123DC63D22D3
:10D8AE003F9B3F623D563B503B4A3C4A3D52696D61
:10D8BE0065001D0570433B4361646174612E6E7596
:10D8CE006D20776179206F75742074686572653A82
:10D8DE002025640A00DA449A444648AE47ED4600D5
:10D8EE0080C0E0F0F8FCFEFF6E756C6C6D6163003D
:10D8FE005805FE48E348E948EF48F548FB48736988
:10D90E0063736C6F776D6163006E051D4A7E4916F9
:10D91E0049FF48054913494374696D657220707259
:10D92E006F636573730000008705934A0000000063
:10D93E00BA000800670B6F0B350002003F11411152
:10D94E005443502F495020737461636B000000B034
:10D95E0005E04D00000000FFFFFFFF00000000018A
:04D96E0000000000B5
:00000001FF
